:020000040800F2
:1000000000060020E1010008E3010008E301000808
:10001000E3010008E3010008E3010008E301000830
:10002000E3010008E3010008E3010008412F000894
:10003000E3010008E3010008E3010008E301000810
:10004000E3010008E3010008E3010008E301000800
:10005000E3010008E3010008E9310008113200085B
:10006000393200086132000889320008E3010008D3
:10007000E3010008E3010008E3010008E3010008D0
:10008000E3010008E3010008E3010008E3010008C0
:10009000E3010008E3010008E3010008B1320008B1
:1000A000E3010008E3010008E3010008E3010008A0
:1000B00085330008E3010008E3010008E3010008BC
:1000C000E3010008E3010008E3010008E301000880
:1000D000E3010008E3010008E3010008E301000870
:1000E00015330008E3010008E3010008E3010008FC
:1000F000E3010008E3010008E3010008E301000850
:10010000E3010008E3010008E3010008E30100083F
:10011000E3010008E3010008E3010008E30100082F
:10012000E3010008E3010008E3010008E30100081F
:10013000E3010008E3010008E3010008E30100080F
:10014000E3010008E3010008E3010008F5260008C8
:10015000E3010008E3010008E3010008E3010008EF
:10016000E3010008E3010008E3010008E3010008DF
:10017000E3010008E3010008E3010008E3010008CF
:10018000E3010008E3010008E3010008E3010008BF
:10019000E3010008E3010008E3010008E3010008AF
:1001A000E3010008E3010008E3010008E30100089F
:1001B000E3010008E3010008E3010008E30100088F
:1001C000E3010008E3010008E3010008E30100087F
:1001D000E3010008E3010008E3010008E30100086F
:1001E00002E000F000F8FEE772B6374880F30888B6
:1001F000364880F3098836483649086040F20000E6
:10020000CCF200004EF63471CEF200010860BFF36C
:100210004F8FBFF36F8F40F20000C0F2F0004EF638
:100220008851CEF200010860BFF34F8FBFF36F8F8C
:100230004FF00000E1EE100A4EF63C71CEF20001E4
:100240000860062080F31488BFF36F8F01F01AFF57
:1002500002F014FE4FF055301F491B4A91423CBF3B
:1002600041F8040BFAE71D49184A91423CBF41F896
:10027000040BFAE71A491B4A1B4B9A423EBF51F83E
:10028000040B42F8040BF8E700201849184A914281
:100290003CBF41F8040BFAE701F0F8FE02F042FE21
:1002A000144C154DAC4203DA54F8041B8847F9E7A7
:1002B00000F042F8114C124DAC4203DA54F8041B22
:1002C0008847F9E701F0E0BE000600200022002088
:1002D0000000000808ED00E00000002000060020FB
:1002E0005037000800220020402200204022002039
:1002F000602E0020E0010008E0010008E001000895
:10030000E00100082DE9F04F2DED108AC1F80CD066
:10031000C3689D46BDEC108ABDE8F08F002383F3CF
:1003200011882846A047002001F05AFAFEE701F0A4
:10033000E9F900DFFEE7000038B500F0BBFB01F093
:1003400071FE054601F094FE0446C8B90E4B9D426D
:1003500018D001339D4218BF044641F2883504BFCE
:1003600001240025002001F067FE0CB100F074F8B4
:1003700000F0E8FC284600F0BFF800F06DF8F9E75F
:100380000025EFE70546EDE7010007B008B500F0EE
:1003900063FBA0F120035842584108BD07B541F264
:1003A0001203022101A8ADF8043000F073FB03B082
:1003B0005DF804FB38B5302383F3118817480368D0
:1003C0000BB101F0D9FA164A144800234FF47A71A0
:1003D00001F0C8FA002383F31188124C236813B18B
:1003E0002368013B2360636813B16368013B63606A
:1003F0000D4D2B7833B963687BB9022000F014FCF3
:10040000322363602B78032B07D163682BB902205A
:1004100000F00AFC4FF47A73636038BD402200207C
:10042000B50300086023002058220020084B1870F4
:1004300003280CD8DFE800F008050208022000F0CD
:10044000F1BB022000F0ECBB024B00225A60704767
:100450005822002060230020234B244A10B51C465C
:10046000196801313FD004339342F9D16268A24246
:1004700039D31F4B9B6803F1006303F540439A4255
:1004800031D2002000F030FB0220FFF7CFFF194BE4
:100490001A6C00221A64196E1A66196E596C5A6425
:1004A000596E5A665A6E5A6942F080025A615A6908
:1004B00022F080025A615A691A6942F000521A61A8
:1004C0001A6922F000521A611B6972B64FF0E023DC
:1004D0003021C3F8084DD4E9003281F311889D46DC
:1004E00083F30888104710BD00C0000820C0000832
:1004F00000220020003802402DE9F04F93B0AA4BB3
:1005000000902022FF210AA89D6800F0C5FBA74AA1
:100510001378A3B9A648012103601170302383F337
:10052000118803680BB101F027FAA24AA048002302
:100530004FF47A7101F016FA002383F31188009BBF
:1005400013B19D4B009A1A609C4A009C1378032BB0
:100550001EBF00231370984A4FF0000A18BF536063
:10056000D3465646D146012000F05CFB24B1924BA5
:100570001B68002B00F01182002000F06DFA039040
:10058000039B002BF2DB012000F04AFB039B213B85
:10059000162BE8D801A252F823F000BFF905000895
:1005A00021060008B5060008670500086705000871
:1005B000670500083F0700080F0900082908000820
:1005C0008B080008B3080008D90800086705000870
:1005D000EB080008670500085D0900089906000897
:1005E00067050008A109000805060008990600082B
:1005F000670500088B0800080220FFF7C7FE0028E7
:1006000040F0F581009B0221BAF1000F08BF1C46A3
:1006100005A841F21233ADF8143000F03BFAA2E71E
:100620004FF47A7000F018FA071EEBDB0220FFF798
:10063000ADFE0028E6D0013F052F00F2DA81DFE8A9
:1006400007F0030A0D10133605230593042105A8AE
:1006500000F020FA17E054480421F9E75848042133
:10066000F6E758480421F3E74FF01C08404600F035
:100670003DFA08F104080590042105A800F00AFAE3
:10068000B8F12C0FF2D1012000FA07F747EA0B0B63
:100690005FFA8BFB4FF0000900F04AFB26B10BF02C
:1006A0000B030B2B08BF0024FFF778FE5BE74648DF
:1006B0000421CDE7002EA5D00BF00B030B2BA1D10D
:1006C0000220FFF763FE074600289BD0012000F0C0
:1006D0000BFA0220FFF7AAFE00261FFA86F8404612
:1006E00000F012FA044690B10021404600F01CFAD6
:1006F00001360028F1D1BA46044641F21213022114
:1007000005A8ADF814303E4600F0C4F92BE70120EF
:10071000FFF78CFE2546244B9B68AB4207D9284641
:1007200000F0E4F9013040F067810435F3E7234B32
:1007300000251D70204BBA465D603E46ACE7002E9A
:100740003FF460AF0BF00B030B2B7FF45BAF022089
:10075000FFF76CFE322000F07FF9B0F10008FFF6E1
:1007600051AF18F003077FF44DAF0F4A926808EBC2
:10077000050393423FF646AFB8F5807F3FF742AF9F
:10078000124B0193B84523DD4FF47A7000F064F901
:100790000390039A002AFFF635AF019B039A03F8F2
:1007A000012B0137EDE700BF002200205C23002071
:1007B00040220020B50300086023002058220020BA
:1007C00004220020082200200C2200205C220020AD
:1007D000C820FFF7DBFD074600283FF413AF1F2DAD
:1007E00011D8C5F1200242450AAB25F0030028BF0D
:1007F000424683490192184400F028FA019A804841
:10080000FF2100F049FA4FEAA8037D490193C8F39C
:100810008702284600F048FA064600283FF46DAFEC
:10082000019B05EB830537E70220FFF7AFFD0028AA
:100830003FF4E8AE00F0A4F900283FF4E3AE00274F
:10084000B846704B9B68BB4218D91F2F11D80A9B22
:1008500001330ED027F0030312AA134453F8203CAF
:1008600005934046042205A900F096FA0437804615
:10087000E7E7384600F03AF90590F2E7CDF8148042
:10088000042105A800F006F906E70023642104A866
:10089000049300F0F5F800287FF4B4AE0220FFF7CF
:1008A00075FD00283FF4AEAE049800F051F90590B4
:1008B000E6E70023642104A8049300F0E1F800288F
:1008C0007FF4A0AE0220FFF761FD00283FF49AAE4E
:1008D000049800F04DF9EAE70220FFF757FD0028E1
:1008E0003FF490AE00F05CF9E1E70220FFF74EFD27
:1008F00000283FF487AE05A9142000F057F9042121
:100900000746049004A800F0C5F83946B9E732203C
:1009100000F0A2F8071EFFF675AEBB077FF472AEBB
:10092000384A926807EB090393423FF66BAE022008
:10093000FFF72CFD00283FF465AE27F003074F4476
:10094000B9453FF4A9AE484600F0D0F8042105901F
:1009500005A800F09FF809F10409F1E74FF47A7057
:10096000FFF714FD00283FF44DAE00F009F9002810
:1009700044D00A9B01330BD008220AA9002000F0C2
:1009800093F900283AD02022FF210AA800F084F928
:10099000FFF704FD1C4800F029FF13B0BDE8F08FFD
:1009A000002E3FF42FAE0BF00B030B2B7FF42AAE7F
:1009B0000023642105A8059300F062F8074600288B
:1009C0007FF420AE0220FFF7E1FC804600283FF4D0
:1009D00019AEFFF7E3FC41F2883000F007FF0598FD
:1009E00000F0D8F9464600F0A3F93C46BBE50646C0
:1009F00052E64FF0000905E6BA467EE637467CE649
:100A00005C22002000220020A086010070B50F4B60
:100A10001B780133DBB2012B0C4611D80C4D296831
:100A20004FF47A730E6AA2FB03320146224628462F
:100A3000B047844204D1074B00221A70012070BDD8
:100A40004FF4FA7000F0D2FE0020F8E710220020E8
:100A5000082600209423002007B500230246012128
:100A60000DF107008DF80730FFF7D0FF20B19DF89A
:100A7000070003B05DF804FB4FF0FF30F9E700001A
:100A80000A4608B50421FFF7C1FF80F00100C0B29B
:100A9000404208BD30B4054C2368DD69044B0A466A
:100AA000AC460146204630BC604700BF0826002007
:100AB000A086010070B501F0BBF9094E094D3080E8
:100AC000002428683388834208D901F0ABF92B68E9
:100AD00004440133B4F5404F2B60F2D370BD00BF26
:100AE000962300206823002001F050BA00F1006036
:100AF00000F540400068704700F10060920000F58A
:100B0000404001F0DBB90000054B1A68054B1B881B
:100B10009B1A834202D9104401F084B90020704727
:100B2000682300209623002038B5084D044629B1DB
:100B300028682044BDE8384001F094B92868204472
:100B400001F078F90028F3D038BD00BF68230020F9
:100B500010F003030AD1B0F5047F05D200F1005074
:100B6000A0F51040D0F80038184670470023FBE786
:100B700000F10050A0F51040D0F8100A70470000B6
:100B8000064991F8243033B10023086A81F82430F3
:100B90000822FFF7B1BF0120704700BF6C2300207F
:100BA000014B1868704700BF002004E070B5194B76
:100BB0001D68194B0138C5F30B0408442D0C0422A1
:100BC0001E88A6420BD15C680A46013C824213464D
:100BD0000FD214F9016F4EB102F8016BF6E7013A3A
:100BE00003F10803ECD181420B4602D22C2203F818
:100BF000012B0A4A05241688AE4204D1984284BFCC
:100C0000967803F8016B013C02F10402F3D1581A03
:100C100070BD00BF002004E06834000854340008B0
:100C200070470000704700007047000070B5044630
:100C30004FF47A764CB1412C254628BF412506FB5E
:100C400005F000F0D3FD641BF4E770BD10B5002380
:100C5000934203D0CC5CC4540133F9E710BD0000CB
:100C600010B5013810F9013F3BB191F900409C42A9
:100C700003D11AB10131013AF4E71AB191F9002018
:100C8000981A10BD1046FCE703460246D01A12F926
:100C9000011B0029FAD1704702440346934202D057
:100CA00003F8011BFAE770472DE9F8431F4D14467E
:100CB00095F824200746884652BBDFF870909CB315
:100CC00095F824302BB92022FF2148462F62FFF7E8
:100CD000E3FF95F82400C0F10802A24228BF224693
:100CE000D6B24146920005EB8000FFF7AFFF95F8C2
:100CF0002430A41B1E44F6B2082E17449044E4B2DC
:100D000085F82460DBD1FFF73BFF0028D7D108E04E
:100D10002B6A03EB82038342CFD0FFF731FF002819
:100D2000CBD10020BDE8F8830120FBE76C23002035
:100D3000024B1A78024B1A70704700BF94230020B0
:100D40001022002010B5104C104800F0B5F82146D4
:100D50000E4800F0DDF82468626DD2F8043843F0E4
:100D60000203C2F804384FF47A70FFF75FFF0849B6
:100D7000204600F0D3F9626DD2F8043823F0020364
:100D8000C2F8043810BD00BF343500080826002022
:100D90003C3500087047000030B5094D0A449142C7
:100DA0000DD011F8013B5840082340F30004013BEB
:100DB0002C4013F0FF0384EA5000F6D1EFE730BD7A
:100DC0002083B8ED026843681143016003B11847FE
:100DD0007047000013B5446BD4F894341A68117846
:100DE000042915D1217C022912D1197912890123F4
:100DF0008B4013420CD101A904F14C0001F0FAFE22
:100E0000D4F89444019B21790246206800F0D0F97F
:100E100002B010BD143001F07DBE00004FF0FF3372
:100E2000143001F077BE00004C3001F04FBF0000DD
:100E30004FF0FF334C3001F049BF0000143001F097
:100E40004BBE00004FF0FF31143001F045BE0000F2
:100E50004C3001F01BBF00004FF0FF324C3001F06E
:100E600015BF00000020704710B5D0F894341A6800
:100E700011780429044617D1017C022914D159792B
:100E8000528901238B4013420ED1143001F0DEFD54
:100E9000024648B1D4F894444FF4807361792068D5
:100EA000BDE8104000F072B910BD0000406BFFF7C4
:100EB000DBBF0000704700007FB5124B03600023CA
:100EC0004360C0E90233012502260F4B0574044636
:100ED0000290019300F18402294600964FF480733A
:100EE000143001F08FFD094B0294CDE9006304F545
:100EF00023724FF48073294604F14C0001F056FE32
:100F000004B070BD88340008AD0E0008D50D00088F
:100F10000B68302282F311880A7903EB8202906118
:100F20004A79093243F822008A7912B103EB82032D
:100F300098610223C0F894140374002080F3118890
:100F40007047000038B5037F044613B190F8543061
:100F5000ABB9201D01250221FFF734FF04F1140075
:100F600025776FF0010100F069FC84F8545004F11A
:100F70004C006FF00101BDE8384000F05FBC38BDA7
:100F800010B5012104460430FFF71CFF002323772E
:100F900084F8543010BD000038B5044600251430E4
:100FA00001F048FD04F14C00257701F017FE201DEB
:100FB00084F854500121FFF705FF2046BDE8384072
:100FC000FFF752BF90F8443003F06003202B07D1A5
:100FD00090F84520212A4FF0000303D81F2A06D895
:100FE00000207047222AFBD1C0E90E3303E0034AF8
:100FF00082630722C263036401207047112200202C
:1010000037B5D0F894341A681178042904461AD1F7
:10101000017C022917D11979128901238B401342CF
:1010200011D100F14C05284601F098FE58B101A9F4
:10103000284601F0DFFDD4F89444019B2179024653
:10104000206800F0B5F803B030BD0000F0B500EB4B
:10105000810385B09E6904460D46FEB1302383F3BB
:10106000118804EB8507301D0821FFF7ABFEFB68F4
:101070005B691B6806F14C001BB1019001F0C8FDD3
:10108000019803A901F0B6FD024648B1039B294629
:10109000204600F08DF8002383F3118805B0F0BDE1
:1010A000FB685A691268002AF5D01B8A013B13407D
:1010B000F1D104F14402EAE7093138B550F8214092
:1010C000DCB1302383F31188D4F894241368527967
:1010D00003EB8203DB689B695D6845B104216018FE
:1010E000FFF770FE294604F1140001F0B9FC204618
:1010F000FFF7BAFE002383F3118838BD7047000064
:1011000001F018B8012303700023C0E90133C36163
:1011100083620362C36243620363704738B5044667
:10112000302383F311880025C0E90355C0E9055534
:10113000416001F00FF80223237085F311882846DF
:1011400038BD000070B500EB810305465069DA60D8
:101150000E46144618B110220021FFF79DFDA0692C
:1011600018B110220021FFF797FD31462846BDE84F
:10117000704001F0B9B80000826802F0011282608C
:101180000022C0E90422826101F03AB9F0B400EB18
:1011900081044789E4680125A4698D403D43458168
:1011A00023600023A2606360F0BC01F055B9000029
:1011B000F0B400EB81040789E468012564698D407F
:1011C0003D43058123600023A2606360F0BC01F011
:1011D000CFB9000070B50223002504460370C0E9B2
:1011E0000255C0E90455C564856180F8345001F0AA
:1011F00017F863681B6823B129462046BDE8704094
:10120000184770BD0378052B10B504460AD080F846
:1012100050300523037043681B680BB104219847C5
:101220000023A36010BD00000178052906D190F8C5
:101230005020436802701B6803B1184770470000D4
:1012400070B590F83430044613B1002380F8343080
:1012500004F14402204601F0F5F863689B68B3B9D5
:1012600094F8443013F0600535D00021204601F099
:1012700095FB0021204601F087FB63681B6813B1D2
:10128000062120469847062384F8343070BD204656
:1012900098470028E4D0B4F84A30E26B9A4288BFFD
:1012A000E36394F94430E56B002B4FF0300380F298
:1012B0000381002D00F0F280092284F8342083F3AA
:1012C00011880021D4E90E232046FFF771FF002387
:1012D00083F31188DAE794F8452003F07F0343EAAB
:1012E000022340F20232934200F0C58021D8B3F5C8
:1012F000807F48D00DD8012B3FD0022B00F0938087
:10130000002BB2D104F14C02A2630222E2632364F7
:10131000C1E7B3F5817F00F09B80B3F5407FA4D196
:1013200094F84630012BA0D1B4F84C3043F00203BE
:1013300032E0B3F5006F4DD017D8B3F5A06F31D0C0
:10134000A3F5C063012B90D8636894F846205E68CB
:1013500094F84710B4F848302046B047002884D0AD
:101360004368A3630368E3631AE0B3F5106F36D0F4
:1013700040F6024293427FF478AF5C4BA3630223B2
:10138000E3630023C3E794F84630012B7FF46DAF8D
:10139000B4F84C3023F00203C4E90E55A4F84C30E5
:1013A000256478E7B4F84430B3F5A06F0ED194F813
:1013B000463084F84E30204600F08AFF63681B6890
:1013C00013B1012120469847032323700023C4E969
:1013D0000E339CE704F14F03A3630123C3E7237893
:1013E000042B10D1302383F311882046FFF7C4FE6D
:1013F00085F311880321636884F84F5021701B68BE
:101400000BB12046984794F84630002BDED084F884
:101410004F300423237063681B68002BD6D0022151
:1014200020469847D2E794F848301D0603F00F0194
:1014300020460AD500F0F8FF012804D002287FF4E6
:1014400014AF2B4B9AE72B4B98E700F0DFFFF3E745
:1014500094F84630002B7FF408AF94F8483013F02E
:101460000F01B3D01A06204602D501F0ABFAADE762
:1014700001F09EFAAAE794F84630002B7FF4F5AE0F
:1014800094F8483013F00F01A0D01B06204602D577
:1014900001F084FA9AE701F077FA97E7142284F8CA
:1014A000342083F311882B462A4629462046FFF72D
:1014B0006DFE85F31188E9E65DB1152284F83420CC
:1014C00083F311880021D4E90E232046FFF75EFE46
:1014D000FDE60B2284F8342083F311882B462A463C
:1014E00029462046FFF764FEE3E700BFB834000852
:1014F000B0340008B434000838B590F834300446ED
:10150000002B3ED0063BDAB20F2A34D80F2B32D84C
:10151000DFE803F0373131082232313131313131F6
:1015200031313737C56BB0F84A309D4214D2C368A9
:101530001B8AB5FBF3F203FB12556DB9302383F31D
:1015400011882B462A462946FFF732FE85F311887B
:101550000A2384F834300EE0142384F83430302326
:1015600083F3118800231A4619462046FFF70EFE22
:10157000002383F3118838BD036C03B1984700231F
:10158000E7E70021204601F009FA0021204601F09A
:10159000FBF963681B6813B10621204698470623B0
:1015A000D7E7000010B590F83430142B044629D04A
:1015B00017D8062B05D001D81BB110BD093B022B53
:1015C000FBD80021204601F0E9F90021204601F076
:1015D000DBF963681B6813B1062120469847062390
:1015E00019E0152BE9D10B2380F83430302383F335
:1015F000118800231A461946FFF7DAFD002383F30A
:101600001188DAE7C3689B695B68002BD5D1036C4E
:1016100003B19847002384F83430CEE700230375E4
:10162000826803691B6899689142FBD25A6803601B
:101630004260106058607047002303758268036938
:101640001B6899689142FBD85A6803604260106039
:101650005860704708B50846302383F311880B7D26
:10166000032B05D0042B0DD02BB983F3118808BDB3
:101670008B6900221A604FF0FF338361FFF7CEFFC2
:101680000023F2E7D1E9003213605A60F3E700006B
:10169000FFF7C4BF054BD9680875186802681A605F
:1016A000536001220275D860FEF72CBE98230020FB
:1016B00030B50C4BDD684B1C87B004460FD02B4671
:1016C000094A684600F04EF92046FFF7E3FF009B09
:1016D00013B1684600F050F9A86907B030BDFFF7B4
:1016E000D9FFF9E79823002055160008044B1A6823
:1016F000DB6890689B68984294BF00200120704787
:1017000098230020084B10B51C68D86822681A601E
:10171000536001222275DC60FFF78EFF01462046F0
:10172000BDE81040FEF7EEBD9823002038B5074C09
:1017300007490848012300252370656001F046FB36
:101740000223237085F3118838BD00BF00260020D6
:10175000C03400089823002000F044B9034A5168BF
:1017600053685B1A9842FBD8704700BF001000E036
:101770008B60022308618B82084670478368A3F15F
:10178000840243F8142C026943F8442C426943F85C
:10179000402C094A43F8242CC26843F8182C022232
:1017A00003F80C2C002203F80B2C044A43F8102CED
:1017B000A3F12000704700BF1D03000898230020FC
:1017C00008B5FFF7DBFFBDE80840FFF761BF000089
:1017D000024BDB6898610F20FFF75CBF9823002065
:1017E000302383F31188FFF7F3BF000008B50146EB
:1017F000302383F311880820FFF75AFF002383F377
:10180000118808BD064BDB6839B1426818605A6020
:10181000136043600420FFF74BBF4FF0FF30704769
:10182000982300200368984206D01A68026050602E
:1018300099611846FFF72CBF7047000038B5044681
:101840000D462068844200D138BD036823605C6087
:101850008561FFF71DFFF4E710B503689C68A2429D
:101860000CD85C688A600B604C6021605960996894
:101870008A1A9A604FF0FF33836010BD1B68121BF9
:10188000ECE700000A2938BF0A2170B504460D466E
:101890000A26601901F094FA01F080FA041BA542AF
:1018A00003D8751C2E460446F3E70A2E04D9BDE87A
:1018B0007040012001F0CABA70BD0000F8B5144BA9
:1018C0000D46D96103F1100141600A2A196982604D
:1018D00038BF0A22016048601861A818144601F058
:1018E00061FA0A2701F05AFA431BA342064606D3BF
:1018F0007C1C281901F064FA27463546F2E70A2FC6
:1019000004D9BDE8F840012001F0A0BAF8BD00BF3D
:1019100098230020F8B506460D4601F03FFA0F4A1D
:10192000134653F8107F9F4206D12A46014630469F
:10193000BDE8F840FFF7C2BFD169BB68441A2C1953
:1019400028BF2C46A34202D92946FFF79BFF224617
:1019500031460348BDE8F840FFF77EBF98230020DA
:10196000A823002010B4C0E9032300235DF8044B32
:101970004361FFF7CFBF000010B5194C23699842AF
:101980000DD0D0E90032816813605A609A680A4429
:101990009A60002303604FF0FF33A36110BD23461C
:1019A000026843F8102F53600022026022699A42B5
:1019B00003D1BDE8104001F0FDB9936881680B4484
:1019C000936001F0EBF92269E1699268441AA2423E
:1019D000E4D91144BDE81040091AFFF753BF00BF16
:1019E000982300202DE9F047DFF8BC8008F11007AC
:1019F0002C4ED8F8105001F0D1F9D8F81C40AA6844
:101A0000031B9A423ED81444D5E900324FF0000936
:101A1000C8F81C4013605A60C5F80090D8F8103020
:101A2000B34201D101F0C6F989F31188D5E9033138
:101A300028469847302383F311886B69002BD8D050
:101A400001F0ACF96A69A0EB04094A4582460DD25F
:101A5000022001F0FBF90022D8F81030B34208D17F
:101A600051462846BDE8F047FFF728BF121A224426
:101A7000F2E712EB090938BF4A4629463846FFF714
:101A8000EBFEB5E7D8F81030B34208D01444211A61
:101A9000C8F81C00A960BDE8F047FFF7F3BEBDE839
:101AA000F08700BFA8230020982300200020704763
:101AB000FEE70000704700004FF0FF307047000065
:101AC00002290CD0032904D00129074818BF00209F
:101AD0007047032A05D8054800EBC2007047044848
:101AE00070470020704700BF983500082022002072
:101AF0004C35000870B59AB00546084601A9144651
:101B000000F0C2F801A8FFF7BFF8431C5B00C5E96D
:101B100000340022237003236370C6B201AB023489
:101B20001046D1B28E4204F1020401D81AB070BD41
:101B300013F8011B04F8021C04F8010C0132F0E751
:101B400008B5302383F311880348FFF759FA0023BF
:101B500083F3118808BD00BF0826002090F84430A8
:101B600003F01F02012A07D190F845200B2A03D168
:101B70000023C0E90E3315E003F06003202B08D1E9
:101B8000B0F848302BB990F84520212A03D81F2AF5
:101B900004D8FFF717BA222AEBD0FAE7034A826388
:101BA0000722C26303640120704700BF182200208F
:101BB00007B5052917D8DFE801F019160319192010
:101BC000302383F31188104A01900121FFF7BAFAFC
:101BD00001980E4A0221FFF7B5FA0D48FFF7DCF92C
:101BE000002383F3118803B05DF804FB302383F3F3
:101BF00011880748FFF7A6F9F2E7302383F311882D
:101C00000348FFF7BDF9EBE7EC3400081035000896
:101C10000826002038B50C4D0C4C0D492A4604F11D
:101C20000800FFF767FF05F1CA0204F11000094937
:101C3000FFF760FF05F5CA7204F118000649BDE818
:101C40003840FFF757BF00BFD02A002020220020D5
:101C5000CC340008D6340008E134000870B50446DE
:101C600008460D46FFF710F8C6B220460134037847
:101C70000BB9184670BD32462946FEF7F1FF002821
:101C8000F3D10120F6E700002DE9F04705460C46A8
:101C9000FEF7FAFF2C49C6B22846FFF7DFFF08B16E
:101CA0000836F6B229492846FFF7D8FF08B11036A2
:101CB000F6B2632E0BD8DFF89080DFF89090244FB7
:101CC000DFF898A02E7846B92670BDE8F08729463F
:101CD0002046BDE8F04701F09FBB252E30D10722FA
:101CE00041462846FEF7BCFF80B91A4B224603F155
:101CF0000C0153F8040B42F8040B8B42F9D11988FC
:101D00009B781180937007350F34DBE70822494632
:101D10002846FEF7A5FF98B90F4BA21C19780909B0
:101D20000232C95D02F8041C13F8011B01F00F0117
:101D30005345C95D02F8031CF0D118340835C1E7DA
:101D400004F8016B0135BDE7B8350008E13400083F
:101D5000D0350008C0350008107AFF1F1C7AFF1F1D
:101D6000BFF34F8F024AD368DB03FCD4704700BF38
:101D7000003C024008B5094B1B7873B9FFF7F0FF30
:101D8000074B1A69002ABFBF064A5A6002F188321F
:101D90005A601A6822F480621A6008BD2E2D002055
:101DA000003C02402301674508B50B4B1B7893B9F3
:101DB000FFF7D6FF094B1A6942F000421A611A6810
:101DC00042F480521A601A6822F480521A601A682B
:101DD00042F480621A6008BD2E2D0020003C0240B3
:101DE0000B28F0B516D80C4C0C4923787BB90C4D58
:101DF0000E460C234FF0006255F8047B46F8042B86
:101E0000013B13F0FF033A44F6D10123237051F84C
:101E10002000F0BD0020FCE7602D0020302D0020C8
:101E2000E4350008014B53F820007047E435000802
:101E30000C2070470B2810B5044601D9002010BDB6
:101E4000FFF7CEFF064B53F824301844C21A0BB9E3
:101E50000120F4E712680132F0D1043BF6E700BF3D
:101E6000E43500080B2810B5044621D8FFF778FFA9
:101E7000FFF780FF0F4AF323D360C300DBB243F4C4
:101E8000007343F002031361136943F48033136159
:101E9000FFF766FFFFF7A4FF074B53F8241000F08D
:101EA000D9F8FFF781FF2046BDE81040FFF7C2BF19
:101EB000002010BD003C0240E4350008F8B512F0E7
:101EC0000103144642D18218B2F1016F57D82D4B4D
:101ED0001B6813F0010352D02B4DFFF74BFFF32388
:101EE000EB60FFF73DFF40F20127032C15D824F0EB
:101EF00001046618244C401A40F20117B1422369CC
:101F000000EB010524D123F001032361FFF74CFF0F
:101F10000120F8BD043C0430E7E78307E7D12B69D3
:101F200023F440732B612B693B432B6151F8046B05
:101F30000660BFF34F8FFFF713FF03689E42E9D09F
:101F40002B6923F001032B61FFF72EFF0020E0E750
:101F500023F44073236123693B4323610B882B8067
:101F6000BFF34F8FFFF7FCFE2D8831F8023BADB277
:101F7000AB42C3D0236923F001032361E4E7184691
:101F8000C7E700BF00380240003C0240084908B5DE
:101F90000B7828B11BB9FFF7EDFE01230B7008BDCC
:101FA000002BFCD0BDE808400870FFF7FDBE00BF65
:101FB0002E2D002010B50244064BD2B2904200D123
:101FC00010BD441C00B253F8200041F8040BE0B2ED
:101FD000F4E700BF502800400F4B30B51C6F2404BD
:101FE00007D41C6F44F400741C671C6F44F4004455
:101FF0001C670A4C236843F4807323600244084B37
:10200000D2B2904200D130BD441C00B251F8045B02
:1020100043F82050E0B2F4E700380240007000407E
:102020005028004007B5012201A90020FFF7C2FF98
:10203000019803B05DF804FB13B50446FFF7F2FF07
:10204000A04205D0012201A900200194FFF7C4FF9E
:1020500002B010BD70470000034B1A681AB9034A5A
:10206000D2F874281A607047642D002000300240B6
:1020700008B5FFF7F1FF024B1868C0F3407008BDC8
:10208000642D002070470000FEE700000A4B0B485B
:102090000B4A90420BD30B4BDA1C121AC11E22F0D2
:1020A00003028B4238BF00220021FEF7F5BD53F832
:1020B000041B40F8041BECE790370008602E00205A
:1020C000602E0020602E002070B5D0E915439E6878
:1020D00000224FF0FF3504EB42135101D3F8000901
:1020E0000028BEBFD3F8000940F08040C3F80009C3
:1020F000D3F8000B0028BEBFD3F8000B40F080409F
:10210000C3F8000B013263189642C3F80859C3F8AC
:10211000085BE0D24FF00113C4F81C3870BD00001A
:10212000890141F02001016103699B06FCD4122062
:10213000FFF714BB10B5054C2046FEF7E3FF4FF048
:10214000A0436365024BA36510BD00BF682D00204E
:102150003836000870B50378012B054650D12A4B5C
:10216000446D98421BD1294B5A6B42F080025A634E
:102170005A6D42F080025A655A6D5A6942F08002E7
:102180005A615A6922F080025A610E2143205B692C
:1021900000F022FC1E4BE3601E4BC4F80038002305
:1021A000C4F8003EC02323606E6D4FF40413A36394
:1021B0003369002BFCDA012333610C20FFF7CEFAE0
:1021C0003369DB07FCD41220FFF7C8FA3369002B10
:1021D000FCDA0026A6602846FFF776FF6B68C4F895
:1021E0001068DB68C4F81468C4F81C684BB90A4B63
:1021F000A3614FF0FF336361A36843F00103A36061
:1022000070BD064BF4E700BF682D00200038024087
:102210004014004003002002003C30C0083C30C0A5
:10222000F8B5446D054600212046FFF779FFA96DFA
:1022300000234FF001128F68C4F834384FF0006665
:10224000C4F81C284FF0FF3004EB431201339F42C7
:10225000C2F80069C2F8006BC2F80809C2F8080B9E
:10226000F2D20B686A6DEB65636210231361166925
:1022700016F01006FBD11220FFF770FAD4F80038E0
:1022800023F4FE63C4F80038A36943F4402343F009
:102290001003A3610923C4F81038C4F814380A4B9A
:1022A000EB604FF0C043C4F8103B084BC4F8003B50
:1022B000C4F81069C4F80039EB6D03F1100243F45F
:1022C0008013EA65A362F8BD143600084080001050
:1022D000426D90F84E10D2F8003823F4FE6343EAC2
:1022E0000113C2F8003870472DE9F84300EB810371
:1022F000456DDA68166806F00306731E022B05EBBF
:1023000041130C4680460FFA81F94FEA41104FF015
:102310000001C3F8101B4FF0010104F1100398BF36
:10232000B60401FA03F391698EBF334E06F180566D
:1023300006F5004600293AD0578A04F158014901B0
:1023400037436F50D5F81C180B43C5F81C382B18B1
:102350000021C3F8101953690127611EA7409BB3E0
:10236000138A928B9B08012A88BF5343D8F85C20BC
:10237000981842EA034301F1400205EB8202C8F8D3
:102380005C00214653602846FFF7CAFE08EB89002F
:10239000C3681B8A43EA8453483464011E432E51A8
:1023A000D5F81C381F43C5F81C78BDE8F88305EB49
:1023B0004917D7F8001B21F40041C7F8001BD5F8D6
:1023C0001C1821EA0303C0E704F13F0305EB830374
:1023D0000A4A5A6028462146FFF7A2FE05EB49103B
:1023E000D0F8003923F40043C0F80039D5F81C3880
:1023F00023EA0707D7E700BF0080001000040002AF
:10240000826D1268C265FFF75FBE00005831436DF0
:1024100049015B5813F4004004D013F4001F0CBFB3
:1024200002200120704700004831436D49015B588C
:1024300013F4004004D013F4001F0CBF022001204D
:102440007047000000EB8101CB68196A0B681360CC
:102450004B6853607047000000EB810330B5DD68C6
:10246000AA691368D36019B9402B84BF4023136055
:102470006B8A1468426D1C44013CB4FBF3F4634363
:10248000033323F0030302EB411043EAC44343F058
:10249000C043C0F8103B2B6803F00303012B09B2C3
:1024A0000ED1D2F8083802EB411013F4807FD0F837
:1024B000003B14BF43F0805343F00053C0F8003B8F
:1024C00002EB4112D2F8003B43F00443C2F8003B58
:1024D00030BD00002DE9F041244D6E6D06EB401338
:1024E0000446D3F8087BC3F8087B38070AD5D6F82A
:1024F0001438190706D505EB84032146DB68284606
:102500005B689847FA071FD5D6F81438DB071BD548
:1025100005EB8403D968CCB98B69488A5A68B2FB49
:10252000F0F600FB16228AB91868DA6890420DD2DC
:10253000121AC3E90024302383F311880B48214683
:10254000FFF78AFF84F31188BDE8F081012303FAC5
:1025500004F26B8923EA02036B81CB68002BF3D072
:1025600021460248BDE8F041184700BF682D002011
:1025700000EB810370B5DD68436D6C692668E66029
:102580004A0156BB1A444FF40020C2F810092A68C9
:1025900002F00302012A0AB20ED1D3F8080803EBB5
:1025A000421410F4807FD4F8000914BF40F080502A
:1025B00040F00050C4F8000903EB4212D2F80009C1
:1025C00040F00440C2F80009D3F83408012202FAAE
:1025D00001F10143C3F8341870BD19B9402E84BF0E
:1025E0004020206020682E8A8419013CB4FBF6F458
:1025F00040EAC44040F000501A44C6E72DE9F843D1
:102600003B4D6E6D06EB40130446D3F80889C3F8C2
:10261000088918F0010F4FEA40171AD0D6F8103881
:10262000DB0716D505EB8003D9684B691868DA68B3
:10263000904230D2121A4FF000091A60C3F8049089
:10264000302383F3118821462846FFF791FF89F351
:10265000118818F0800F1CD0D6F834380126A64017
:10266000334216D005EB84036D6DD3F80CC0DCF853
:1026700014200134E4B2D2F800E005EB04342F4416
:102680005168714515D3D5F8343823EA0606C5F8E4
:102690003468BDE8F883012303FA04F22B8923EAA6
:1026A00002032B818B68002BD3D021462846984704
:1026B000CFE7BCF81000AEEB0103834228BF03460E
:1026C000D7F8180980B2B3EB800FE2D89068A0F178
:1026D000040959F8048FC4F80080A0EB0908984455
:1026E000B8F1040FF5D818440B4490605360C7E765
:1026F000682D00202DE9F74FA24C656D6E69AB691E
:102700001E4016F480586E6107D02046FEF762FD29
:1027100003B0BDE8F04F00F047BC002E12DAD5F848
:10272000003E98489B071EBFD5F8003E23F00303E8
:10273000C5F8003ED5F8043823F00103C5F8043885
:10274000FEF772FD370505D58E48FFF7BDFC8D48B5
:10275000FEF758FDB0040CD5D5F8083813F0060F75
:10276000EB6823F470530CBF43F4105343F4A053AD
:10277000EB6031071BD56368DB681BB9AB6923F0DD
:102780000803AB612378052B0CD1D5F8003E7D48BA
:102790009A071EBFD5F8003E23F00303C5F8003E9C
:1027A000FEF742FD6368DB680BB176489847F30299
:1027B00074D4B70227D5D4F85490DFF8C8B10027F5
:1027C0004FF0010A09EB4712D2F8003B03F4402313
:1027D000B3F5802F11D1D2F8003B002B0DDA6289BE
:1027E0000AFA07F322EA0303638104EB8703DB6839
:1027F000DB6813B1394658469847A36D01379B688B
:10280000FFB29F42DED9F00617D5676D3A6AC2F370
:102810000A1002F00F0302F4F012B2F5802F00F05C
:102820008580B2F5402F08D104EB83030022DB68DA
:102830001B6A07F5805790426AD13003D5F81848D3
:1028400013D5E10302D50020FFF744FEA20302D511
:102850000120FFF73FFE630302D50220FFF73AFE97
:10286000270302D50320FFF735FE75037FF550AF30
:10287000E00702D50020FFF7C1FEA10702D5012025
:10288000FFF7BCFE620702D50220FFF7B7FE230761
:102890007FF53EAF0320FFF7B1FE39E7636DDFF848
:1028A000E4A0019300274FF00109A36D9B685FFA34
:1028B00087FB9B453FF67DAF019B03EB4B13D3F8A2
:1028C000001901F44021B1F5802F1FD1D3F8001970
:1028D00000291BDAD3F8001941F09041C3F8001920
:1028E000D3F800190029FBDB5946606DFFF718FC8F
:1028F000218909FA0BF321EA0303238104EB8B03FB
:10290000DB689B6813B15946504698470137CCE7BE
:10291000910708BFD7F80080072A98BF03F8018BFA
:1029200002F1010298BF4FEA182884E7023304EB52
:10293000830207F580575268D2F818C0DCF80820E7
:10294000DCE9001CA1EB0C0C002188420AD104EB4D
:10295000830463689B699A6802449A605A680244D7
:102960005A606AE711F0030F08BFD7F800808C4562
:1029700088BF02F8018B01F1010188BF4FEA1828D6
:10298000E3E700BF682D0020436D03EB4111D1F850
:10299000003B43F40013C1F8003B7047436D03EB69
:1029A0004111D1F8003943F40013C1F800397047E0
:1029B000436D03EB4111D1F8003B23F40013C1F840
:1029C000003B7047436D03EB4111D1F8003923F40C
:1029D0000013C1F80039704700F1604303F561430B
:1029E0000901C9B283F80013012200F01F039A40C5
:1029F00043099B0003F1604303F56143C3F8802161
:102A00001A60704730B5039C0172043304FB032540
:102A1000C0E90653049B03630021059BC160C0E924
:102A20000000C0E90422C0E90842C0E90A1143637A
:102A300030BD0000416A0022C0E90411C0E90A2249
:102A4000C2606FF00101FEF7F9BE0000D0E9043268
:102A5000934201D1C2680AB9181D7047002070471F
:102A600003691960C2680132C260C2691344826995
:102A70000361934224BF436A03610021FEF7D2BE83
:102A800038B504460D46E3683BB16269131D126810
:102A9000A3621344E362002007E0237A33B9294696
:102AA0002046FEF7AFFE0028EDDA38BD6FF00100DA
:102AB000FBE70000C368C269013BC360436913447C
:102AC00082694361934224BF436A43610023836266
:102AD000036B03B11847704770B53023044683F386
:102AE0001188866A3EB9FFF7CBFF054618B186F319
:102AF0001188284670BDA36AE26A13F8015BA362DD
:102B0000934202D32046FFF7D5FF002383F31188B9
:102B1000EFE700002DE9F84F04460E4617469846A9
:102B20004FF0300989F311880025AA46D4F828B05F
:102B3000BBF1000F09D141462046FFF7A1FF20B1AC
:102B40008BF311882846BDE8F88FD4E90A12A7EB69
:102B5000050B521A934528BF9346BBF1400F1BD972
:102B6000334601F1400251F8040B43F8040B914243
:102B7000F9D1A36A40334036A3624035D4E90A2331
:102B80009A4202D32046FFF795FF8AF31188BD428F
:102B9000D8D289F31188C9E730465A46FEF756F86D
:102BA000A36A5B445E44A3625D44E7E710B5029C00
:102BB0000172043303FB0421C0E906130023C0E9BA
:102BC0000A33039B0363049BC460C0E90000C0E9AF
:102BD0000422C0E90842436310BD0000026AC260DB
:102BE000426AC0E904220022C0E90A226FF0010112
:102BF000FEF724BED0E904239A4201D1C26822B96B
:102C0000184650F8043B0B60704700231846FAE75B
:102C1000C368C2690133C360436913448269436175
:102C2000934224BF436A43610021FEF7FBBD0000CD
:102C300038B504460D46E3683BB123691A1DA2620C
:102C4000E2691344E362002007E0237A33B929469E
:102C50002046FEF7D7FD0028EDDA38BD6FF0010001
:102C6000FBE7000003691960C268013AC260C269EB
:102C7000134482690361934224BF436A03610023C2
:102C80008362036B03B118477047000070B53023AF
:102C90000D460446114683F31188866A2EB9FFF764
:102CA000C7FF10B186F3118870BDA36A1D70A36AB7
:102CB000E26A01339342A36204D3E16920460439F6
:102CC000FFF7D0FF002080F31188EDE72DE9F84FE2
:102CD00004460D46904699464FF0300A8AF3118813
:102CE0000026B346A76A4FB949462046FFF7A0FF22
:102CF00020B187F311883046BDE8F88FD4E90A0780
:102D00003A1AA8EB0607974228BF1746402F1BD94F
:102D100005F1400355F8042B40F8042B9D42F9D1EE
:102D2000A36A4033A3624036D4E90A239A4204D30B
:102D3000E16920460439FFF795FF8BF3118846457A
:102D4000D9D28AF31188CDE729463A46FDF77EFFAE
:102D5000A36A3B443D44A3623E44E5E7D0E9042333
:102D60009A4217D1C3689BB1836A8BB1043B9B1A0B
:102D70000ED01360C368013BC360C3691A44836902
:102D800002619A4224BF436A0361002383620123E4
:102D9000184670470023FBE700F030B94FF080433E
:102DA000586A70474FF08043002258631A6102222C
:102DB000DA6070474FF080430022DA60704700000D
:102DC0004FF0804358637047FEE7000070B51B4B1F
:102DD00001630025044686B0586085620E4600F007
:102DE000BFF804F11003C4E904334FF0FF33C4E922
:102DF0000635C4E90044A560E562FFF7CFFF2B4626
:102E00000246C4E9082304F134010D4A25658023F4
:102E10002046FEF7ADFC0123E0600A4A03750092EC
:102E200072680192B268CDE90223074B6846CDE98A
:102E30000435FEF7C5FC06B070BD00BF00260020BB
:102E40004436000849360008C92D0008024AD36AF2
:102E50001843D062704700BF982300204B6843603E
:102E60008B688360CB68C3600B6943614B69036205
:102E70008B6943620B6803607047000008B5264BFE
:102E800026481A6940F2FF110A431A611A6922F4AE
:102E9000FF7222F001021A611A691A6B0A431A635F
:102EA0001A6D0A431A651E4A1B6D1146FFF7D6FFBD
:102EB00002F11C0100F58060FFF7D0FF02F138013C
:102EC00000F58060FFF7CAFF02F1540100F5806051
:102ED000FFF7C4FF02F1700100F58060FFF7BEFF4D
:102EE00002F18C0100F58060FFF7B8FF02F1A80144
:102EF00000F58060FFF7B2FF02F1C40100F58060C9
:102F0000FFF7ACFF02F1E00100F58060FFF7A6FFDC
:102F1000BDE8084000F0EEB8003802400000024072
:102F20005036000808B500F059FAFEF7FFFBFFF72E
:102F300093F8BDE80840FEF76DBE00007047000042
:102F4000EFF3098305494A6B22F001024A636833B3
:102F500083F30988002383F31188704700EF00E0B2
:102F6000302080F3118862B60C4B0D4AD96821F4E9
:102F7000E0610904090C0A43DA60D3F8FC2009492E
:102F800042F08072C3F8FC200A6842F001020A6035
:102F90002022DA7783F82200704700BF00ED00E0BE
:102FA0000003FA05001000E010B5302383F3118808
:102FB0000E4B5B6813F4006314D0F1EE103AEFF39C
:102FC0000984683C4FF08073E361094BDB6B236637
:102FD00084F30988FEF78AFB10B1064BA36110BD8C
:102FE000054BFBE783F31188F9E700BF00ED00E034
:102FF00000EF00E02F030008320300080F4B1A6CAB
:1030000042F001021A641A6E42F001021A660C4A7A
:103010001B6E936843F0010393604FF0804353228B
:103020009A624FF0FF32DA6200229A615A63DA60E4
:103030005A6001225A611A60704700BF003802408E
:10304000002004E04FF0804208B51169D3680B40BE
:10305000D9B2C9439B07116107D5302383F3118887
:10306000FEF77AFB002383F3118808BD1F4B1A6912
:103070006FEAC2526FEAD2521A611A69C2F30802A9
:103080001A614FF0FF301A695A69586100215A6974
:1030900059615A691A6A62F080521A621A6A02F019
:1030A00080521A621A6A5A6A58625A6A59625A6A8D
:1030B0001A6C42F080521A641A6E42F080521A66FC
:1030C0001A6E0B4A106840F480701060186F00F49C
:1030D0004070B0F5007F1EBF4FF48030186719674D
:1030E000536823F40073536000F054B90038024071
:1030F00000700040334B4FF080521A64324A4FF454
:10310000404111601A6842F001021A601A68910782
:10311000FCD59A6822F003029A602A4B9A6812F052
:103120000C02FBD1196801F0F90119609A601A6864
:1031300042F480321A601A689203FCD55A6F42F04A
:1031400001025A671F4B5A6F9007FCD51F4A5A60FD
:103150001A6842F080721A601B4A53685904FCD501
:10316000184B1A689201FCD5194A9A60194B1A68D3
:10317000194B9A42194B21D1194A1168194A9142A7
:103180001CD140F205121A60144A136803F00F03B1
:10319000052BFAD10B4B9A6842F002029A609A68AA
:1031A00002F00C02082AFAD15A6C42F480425A64A6
:1031B0005A6E42F480425A665B6E704740F2057266
:1031C000E1E700BF003802400070004008544007AB
:1031D00000948838002004E011640020003C024084
:1031E00000ED00E041C20F41074A08B5536903F002
:1031F0000103536123B1054A13680BB15068984726
:10320000BDE80840FFF7D0BE003C0140E02D0020A3
:10321000074A08B5536903F00203536123B1054A15
:1032200093680BB1D0689847BDE80840FFF7BCBE73
:10323000003C0140E02D0020074A08B5536903F027
:103240000403536123B1054A13690BB150699847D0
:10325000BDE80840FFF7A8BE003C0140E02D00207B
:10326000074A08B5536903F00803536123B1054ABF
:1032700093690BB1D0699847BDE80840FFF794BE49
:10328000003C0140E02D0020074A08B5536903F0D7
:103290001003536123B1054A136A0BB1506A984772
:1032A000BDE80840FFF780BE003C0140E02D002053
:1032B000164B10B55C6904F478725A61A30604D504
:1032C000134A936A0BB1D06A9847600604D5104A36
:1032D000136B0BB1506B9847210604D50C4A936BC6
:1032E0000BB1D06B9847E20504D5094A136C0BB1BA
:1032F000506C9847A30504D5054A936C0BB1D06C6C
:103300009847BDE81040FFF74FBE00BF003C0140AA
:10331000E02D0020194B10B55C6904F47C425A6121
:10332000620504D5164A136D0BB1506D98472305FD
:1033300004D5134A936D0BB1D06D9847E00404D5C2
:103340000F4A136E0BB1506E9847A10404D50C4A76
:10335000936E0BB1D06E9847620404D5084A136F80
:103360000BB1506F9847230404D5054A936F0BB1F6
:10337000D06F9847BDE81040FFF716BE003C0140F3
:10338000E02D002008B5FFF75DFEBDE80840FFF71F
:103390000BBE0000062108B50846FFF71DFB0621FD
:1033A0000720FFF719FB06210820FFF715FB062170
:1033B0000920FFF711FB06210A20FFF70DFB06216C
:1033C0001720FFF709FB06212820FFF705FBBDE8C2
:1033D000084007211C20FFF7FFBA000008B5FFF7DF
:1033E00045FE00F00BF8FDF78BFEFDF763FDFFF7E0
:1033F000A5FDBDE80840FFF7CFBC00000023054A4B
:1034000019460133102BC2E9001102F10802F8D16C
:10341000704700BFE02D0020034611F8012B03F890
:10342000012B002AF9D1704753544D3332463F3FA8
:103430003F0053544D3332463430780053544D33AB
:1034400032463432780053544D3332463434365891
:1034500058000000012033000010410001105A0004
:103460000310590007103100000000002834000844
:103470001304000032340008190400003C34000832
:10348000210400004634000800000000310E00084E
:103490001D0E0008590E0008450E0008510E0008C8
:1034A0003D0E0008290E0008150E0008650E0008E4
:1034B0000000000001000000000000006330000078
:1034C000BC340008F02300200026002041726475FF
:1034D00050696C6F740025424F415244252D424C77
:1034E000002553455249414C2500000002000000D0
:1034F000000000004D100008B91000084000400016
:10350000A02A0020B02A00200200000000000000D5
:103510000300000000000000FD1000080000000093
:1035200010000000C02A0020000000000100000080
:1035300000000000682D002001010200B11B0008FE
:10354000C11A00085D1B0008411B00084300000071
:103550005435000809024300020100C0320904008A
:1035600000010202010005240010010524010001F0
:10357000042402020524060001070582030800FF57
:1035800009040100020A00000007050102400000D2
:10359000070581024000000012000000A03500086D
:1035A00012011001020000400912415700020102FD
:1035B000030100000403090425424F415244250041
:1035C0004D616D62614634303555532D49324300AB
:1035D0003031323334353637383941424344454649
:1035E000000000000040000000400000004000001B
:1035F0000040000000000100000002000000020086
:1036000000000200000002000000020000000200B2
:10361000000002000000000041120008F914000838
:10362000A515000840004000C82D0020C82D00202E
:1036300001000000D82D00208000000040010000A3
:10364000030000006D61696E0069646C6500000034
:103650000000800200000000AAAAAAAA0000000040
:10366000FFFF00000000000000A00A0000000000B2
:1036700000000000AAAAAAAA00000000FFFF0000A4
:1036800000000000000000000000005000000000EA
:10369000AAAAAAAA00000000FF3F00000000000044
:1036A000000000000000000000000000AAAAAAAA72
:1036B00000000000FFFF000000000000000000000C
:1036C0000000000000000000AAAAAAAA0000000052
:1036D000FFFF0000000000000000000000000000EC
:1036E00000000000AAAAAAAA00000000FFFF000034
:1036F00000000000000000000000000000000000CA
:10370000AAAAAAAA00000000FFFF00000000000013
:103710000000000000000000000000000A0000009F
:103720000000000003000000000000000000000096
:103730000000000000000000000000000000000089
:103740000000000000000000000000000000000079
:103750000E0400000000000000400F000000000008
:10376000FF0096000000000800960000000008001E
:1037700004000000B4350008000000000000000054
:103780000000000000000000000000000000000039
:10379000FFFFFFFFFFFFFFFFFFFFFFFFFFFFFFFF39
:1037A000FFFFFFFFFFFFFFFFFFFFFFFFFFFFFFFF29
:1037B000FFFFFFFFFFFFFFFFFFFFFFFFFFFFFFFF19
:10C000000006002099D2000811EC09086DEB090820
:10C01000D9EB09086DEB0908A5EB09089BD20008CC
:10C020009BD200089BD200089BD20008F1360C0876
:10C030009BD200089BD200089BD200089BD200082C
:10C040009BD200089BD200089BD200089BD200081C
:10C050009BD200089BD200080D490C0835490C08FA
:10C060005D490C0885490C08AD490C08A9F20B087C
:10C07000D1F20B08FDF20B0829F30B0855F30B085E
:10C080007DF30B08A9F30B082DF20B089BD20008D7
:10C090009BD200089BD200089BD20008D5490C080F
:10C0A000214B0C08254B0C08394B0C083D4B0C0858
:10C0B0009BD20008414B0C08554B0C0835F90B0876
:10C0C000DDFA0B089BD200089BD200089BD2000827
:10C0D0009BD20008A94A0C08BD4A0C08D14A0C089A
:10C0E000394A0C089BD200089BD200089BD200085A
:10C0F0009BD200089BD200089BD20008D5F30B0806
:10C100009BD200089BD20008694B0C089BD2000808
:10C11000E54A0C08F94A0C089BD200089BD200089B
:10C1200001F40B0829F40B0855F40B0881F40B08F3
:10C13000ADF40B089BD200089BD200089BD20008EC
:10C140009BD200089BD200089BD200081D3E0C0821
:10C15000D5F40B0801F50B082DF50B080D4B0C0859
:10C160009BD200089BD200089BD200089BD20008FB
:10C170009BD200089BD200089BD200089BD20008EB
:10C180009BD200089BD200089BD200089BD20008DB
:10C190009BD200089BD200089BD200089BD20008CB
:10C1A0009BD200089BD200089BD200089BD20008BB
:10C1B0009BD200089BD200089BD200089BD20008AB
:10C1C0009BD200089BD200089BD200089BD200089B
:10C1D0009BD200089BD200089BD200089BD200088B
:10C1E0001DF50008B9290108215C01087DBB010883
:10C1F00039040208F97C0208EDFD030815C10508A1
:10C200001DC70508BD250608E9790608AD810608A1
:10C21000E584060859EA0608F90A070855C7070819
:10C22000113F0808C5E40908210B0B08856D0B08B0
:10C2300055940B08799E0B08D5CD0B08FDD30B0840
:10C2400081F0004102E000BF83F0004330B54FEAC7
:10C2500041044FEA430594EA050F08BF90EA020F34
:10C260001FBF54EA000C55EA020C7FEA645C7FEAC7
:10C27000655C00F0E2804FEA5454D4EB5555B8BFEA
:10C280006D420CDD2C4480EA020281EA030382EA5B
:10C29000000083EA010180EA020281EA0303362DED
:10C2A00088BF30BD11F0004F4FEA01314FF4801CC0
:10C2B0004CEA113102D0404261EB410113F0004FD2
:10C2C0004FEA03334CEA133302D0524263EB430389
:10C2D00094EA050F00F0A780A4F10104D5F1200E27
:10C2E0000DDB02FA0EFC22FA05F2801841F1000182
:10C2F00003FA0EF2801843FA05F359410EE0A5F156
:10C3000020050EF1200E012A03FA0EFC28BF4CF086
:10C31000020C43FA05F3C01851EBE37101F000453C
:10C3200007D54FF0000EDCF1000C7EEB00006EEB49
:10C330000101B1F5801F1BD3B1F5001F0CD34908D3
:10C340005FEA30004FEA3C0C04F101044FEA44522A
:10C3500012F5800F80F09A80BCF1004F08BF5FEAB1
:10C36000500C50F1000041EB045141EA050130BD91
:10C370005FEA4C0C404141EB0101013C28BFB1F5A3
:10C38000801FE9D291F0000F04BF01460020B1FAEE
:10C3900081F308BF2033A3F10B03B3F120020CDAC1
:10C3A0000C3208DD02F1140CC2F10C0201FA0CF09F
:10C3B00021FA02F10CE002F11402D8BFC2F1200C04
:10C3C00001FA02F120FA0CFCDCBF41EA0C019040BA
:10C3D000E41AA2BF01EB0451294330BD6FEA040403
:10C3E0001F3C1CDA0C340EDC04F11404C4F12002EE
:10C3F00020FA04F001FA02F340EA030021FA04F300
:10C4000045EA030130BDC4F10C04C4F1200220FA56
:10C4100002F001FA04F340EA0300294630BD21FA94
:10C4200004F0294630BD94F0000F83F4801306BF5A
:10C4300081F480110134013D4EE77FEA645C18BF4E
:10C440007FEA655C29D094EA050F08BF90EA020FE5
:10C4500005D054EA000C04BF1946104630BD91EADD
:10C46000030F1EBF0021002030BD5FEA545C05D1E0
:10C470004000494128BF41F0004130BD14F580041F
:10C480003CBF01F5801130BD01F0004545F0FE4193
:10C4900041F470014FF0000030BD7FEA645C1ABFC8
:10C4A000194610467FEA655C1CBF0B46024650EAFF
:10C4B000013406BF52EA033591EA030F41F400212B
:10C4C00030BD00BF90F0000F04BF0021704730B5B1
:10C4D0004FF4806404F132044FF000054FF0000186
:10C4E00050E700BF90F0000F04BF0021704730B547
:10C4F0004FF4806404F1320410F0004548BF40421C
:10C500004FF000013EE700BF42004FEAE2014FEA70
:10C5100031014FEA02701FBF12F07F4393F07F4F4B
:10C5200081F06051704732F07F4208BF704793F04E
:10C530007F4F04BF41F40021704730B54FF4607461
:10C5400001F0004521F000411CE700BF50EA010264
:10C5500008BF704730B54FF000050AE050EA01020D
:10C5600008BF704730B511F0004502D5404261EB7D
:10C5700041014FF4806404F132045FEA915C3FF4BE
:10C58000D8AE4FF003025FEADC0C18BF03325FEA5B
:10C59000DC0C18BF033202EBDC02C2F1200300FA0C
:10C5A00003FC20FA02F001FA03FE40EA0E0021FA31
:10C5B00002F11444BDE600BF70B54FF0FF0C4CF41F
:10C5C000E06C1CEA11541DBF1CEA135594EA0C0FD1
:10C5D00095EA0C0F00F0DEF82C4481EA030621EA0C
:10C5E0004C5123EA4C5350EA013518BF52EA033547
:10C5F00041F4801143F4801338D0A0FB02CE4FF0F9
:10C600000005E1FB02E506F00042E0FB03E54FF028
:10C610000006E1FB03569CF0000F18BF4EF0010E20
:10C62000A4F1FF04B6F5007F64F5407404D25FEA1C
:10C630004E0E6D4146EB060642EAC62141EA5551CF
:10C640004FEAC52040EA5E504FEACE2EB4F1FD0C11
:10C6500088BFBCF5E06F1ED8BEF1004F08BF5FEA8F
:10C66000500E50F1000041EB045170BD06F0004641
:10C6700046EA010140EA020081EA0301B4EB5C04EE
:10C68000C2BFD4EB0C0541EA045170BD41F48011E6
:10C690004FF0000E013C00F3AB8014F1360FDEBF0B
:10C6A000002001F0004170BDC4F10004203C35DAE7
:10C6B0000C341BDC04F11404C4F1200500FA05F36A
:10C6C00020FA04F001FA05F240EA020001F000420B
:10C6D00021F0004110EBD37021FA04F642EB060181
:10C6E0005EEA430E08BF20EAD37070BDC4F10C04AB
:10C6F000C4F1200500FA04F320FA05F001FA04F26F
:10C7000040EA020001F0004110EBD37041F100015A
:10C710005EEA430E08BF20EAD37070BDC4F1200565
:10C7200000FA05F24EEA020E20FA04F301FA05F2CD
:10C7300043EA020321FA04F001F0004121FA04F275
:10C7400020EA020000EBD3705EEA430E08BF20EA45
:10C75000D37070BD94F0000F0FD101F0004640007F
:10C7600041EB010111F4801F08BF013CF7D041EA01
:10C77000060195F0000F18BF704703F00046520005
:10C7800043EB030313F4801F08BF013DF7D043EAD6
:10C790000603704794EA0C0F0CEA135518BF95EA8C
:10C7A0000C0F0CD050EA410618BF52EA4306D1D113
:10C7B00081EA030101F000414FF0000070BD50EA32
:10C7C000410606BF1046194652EA430619D094EABC
:10C7D0000C0F02D150EA013613D195EA0C0F05D1A6
:10C7E00052EA03361CBF104619460AD181EA0301FA
:10C7F00001F0004141F0FE4141F470014FF00000B2
:10C8000070BD41F0FE4141F4780170BD70B54FF04C
:10C81000FF0C4CF4E06C1CEA11541DBF1CEA1355CC
:10C8200094EA0C0F95EA0C0F00F0A7F8A4EB0504AE
:10C8300081EA030E52EA03354FEA013100F08880A5
:10C840004FEA03334FF0805545EA131343EA12636E
:10C850004FEA022245EA111545EA10654FEA002623
:10C860000EF000419D4208BF964244F1FD0404F5DC
:10C87000407402D25B084FEA3202B61A65EB030538
:10C880005B084FEA32024FF480104FF4002CB6EBF5
:10C89000020E75EB030E22BFB61A754640EA0C0075
:10C8A0005B084FEA3202B6EB020E75EB030E22BFB5
:10C8B000B61A754640EA5C005B084FEA3202B6EBF6
:10C8C000020E75EB030E22BFB61A754640EA9C00B5
:10C8D0005B084FEA3202B6EB020E75EB030E22BF85
:10C8E000B61A754640EADC0055EA060E18D04FEA43
:10C8F000051545EA16754FEA06164FEAC30343EAE3
:10C9000052734FEAC2025FEA1C1CC0D111F4801FAF
:10C910000BD141EA00014FF000004FF0004CB6E7A8
:10C9200011F4801F04BF01430020B4F1FD0C88BF47
:10C93000BCF5E06F3FF6AFAEB5EB030C04BFB6EB52
:10C94000020C5FEA500C50F1000041EB045170BD45
:10C950000EF0004E4EEA113114EB5C04C2BFD4EB72
:10C960000C0541EA045170BD41F480114FF0000EF6
:10C97000013C90E645EA060E8DE60CEA135594EA72
:10C980000C0F08BF95EA0C0F3FF43BAF94EA0C0F75
:10C990000AD150EA01347FF434AF95EA0C0F7FF4EA
:10C9A00025AF104619462CE795EA0C0F06D152EA3E
:10C9B00003353FF4FDAE1046194622E750EA410622
:10C9C00018BF52EA43067FF4C5AE50EA41047FF433
:10C9D0000DAF52EA43057FF4EBAE12E74FF0FF3C98
:10C9E00006E000BF4FF0010C02E000BF4FF0010C69
:10C9F0004DF804CD4FEA410C7FEA6C5C4FEA430CE2
:10CA000018BF7FEA6C5C1BD001B050EA410C0CBF30
:10CA100052EA430C91EA030F02BF90EA020F002092
:10CA2000704710F1000F91EA030F58BF994208BFF9
:10CA300090422CBFD8176FEAE37040F001007047B6
:10CA40004FEA410C7FEA6C5C02D150EA013C07D10D
:10CA50004FEA430C7FEA6C5CD6D152EA033CD3D058
:10CA60005DF8040B704700BF8446104662468C4652
:10CA70001946634600E000BF01B5FFF7B7FF002885
:10CA800048BF10F1000F01BD4DF808EDFFF7F4FFAE
:10CA90000CBF012000205DF808FB00BF4DF808ED39
:10CAA000FFF7EAFF34BF012000205DF808FB00BF5C
:10CAB0004DF808EDFFF7E0FF94BF012000205DF87E
:10CAC00008FB00BF4DF808EDFFF7CEFF94BF012033
:10CAD00000205DF808FB00BF4DF808EDFFF7C4FF2C
:10CAE00034BF012000205DF808FB00BF4FEA410C75
:10CAF0007FEA6C5C02D150EA013C0AD14FEA430C58
:10CB00007FEA6C5C02D152EA033C02D14FF0000094
:10CB100070474FF0010070474FEA410212F50012D2
:10CB200015D211D56FF47873B3EB625212D94FEA74
:10CB3000C12343F0004343EA505311F0004F23FA5E
:10CB400002F018BF404270474FF00000704750EAB3
:10CB5000013005D111F0004008BF6FF00040704770
:10CB60004FF00000704700BF4A0011D212F50012CA
:10CB700011D20DD56FF47873B3EB62520ED44FEA35
:10CB8000C12343F0004343EA505323FA02F07047B5
:10CB90004FF00000704750EA013002D14FF0FF30F3
:10CBA00070474FF0000070474FEA4102B2F1E04396
:10CBB00024BFB3F5001CDCF1FE5C0DD901F0004C84
:10CBC0004FEAC0024CEA5070B2F1004F40EB8300D4
:10CBD00008BF20F00100704711F0804F21D113F100
:10CBE0003872BCBF01F00040704741F480114FEA39
:10CBF0005252C2F11802C2F1200C10FA0CF320FAC2
:10CC000002F018BF40F001004FEAC1234FEAD323DE
:10CC100003FA0CFC40EA0C0023FA02F34FEA430348
:10CC2000CCE77FEA625307D150EA01331EBF4FF0D1
:10CC3000FE4040F44000704701F0004040F0FE40EC
:10CC400040F40000704700BF80F0004002E000BFE9
:10CC500081F0004142001FBF5FEA410392EA030FE7
:10CC60007FEA226C7FEA236C6AD04FEA1262D2EB31
:10CC70001363C1BFD218414048404140B8BF5B4236
:10CC8000192B88BF704710F0004F40F4000020F0CF
:10CC90007F4018BF404211F0004F41F4000121F0E5
:10CCA0007F4118BF494292EA030F3FD0A2F101022F
:10CCB00041FA03FC10EB0C00C3F1200301FA03F16D
:10CCC00000F0004302D5494260EB4000B0F5000F90
:10CCD00013D3B0F1807F06D340084FEA310102F14F
:10CCE0000102FE2A51D2B1F1004F40EBC25008BF01
:10CCF00020F0010040EA03007047490040EB0000CB
:10CD0000013A28BFB0F5000FEDD2B0FA80FCACF1CB
:10CD1000080CB2EB0C0200FA0CF0AABF00EBC250F8
:10CD200052421843BCBFD0401843704792F0000FE6
:10CD300081F4000106BF80F400000132013BB5E739
:10CD40004FEA41037FEA226C18BF7FEA236C21D0AF
:10CD500092EA030F04D092F0000F08BF0846704714
:10CD600090EA010F1CBF0020704712F07F4F04D1E2
:10CD7000400028BF40F00040704712F100723CBFF5
:10CD800000F50000704700F0004343F0FE4040F41F
:10CD9000000070477FEA226216BF08467FEA2363DD
:10CDA0000146420206BF5FEA412390EA010F40F4C8
:10CDB000800070474FF0000304E000BF10F0004314
:10CDC00048BF40425FEA000C08BF704743F09643FB
:10CDD00001464FF000001CE050EA010208BF704716
:10CDE0004FF000030AE000BF50EA010208BF70479D
:10CDF00011F0004302D5404261EB41015FEA010CB2
:10CE000002BF84460146002043F0B64308BFA3F1A9
:10CE10008053A3F50003BCFA8CF2083AA3EBC2538B
:10CE200010DB01FA02FC634400FA02FCC2F12002AA
:10CE3000BCF1004F20FA02F243EB020008BF20F0E1
:10CE40000100704702F1200201FA02FCC2F1200247
:10CE500050EA4C0021FA02F243EB020008BF20EA3C
:10CE6000DC7070477BB972B90029BEBF00204FF05B
:10CE7000004106E008BF00281CBF6FF000414FF0E2
:10CE8000FF3000F007BAADF1080C6DE904CE0029BF
:10CE900009DB002B1ADB00F095F8DDF804E0DDE992
:10CEA000022304B07047404261EB4101002B1BDBC1
:10CEB00000F088F8DDF804E0DDE9022304B0404228
:10CEC00061EB4101524263EB43037047524263EB13
:10CED000430300F077F8DDF804E0DDE9022304B055
:10CEE000404261EB41017047524263EB430300F063
:10CEF00069F8DDF804E0DDE9022304B0524263EB97
:10CF00004303704753B94AB9002908BF00281CBF22
:10CF10004FF0FF314FF0FF3000F0BCB9ADF1080C1D
:10CF20006DE904CE00F04EF8DDF804E0DDE90223FF
:10CF300004B07047430803F05533C01A830803F068
:10CF4000333300F03330184400EB101000F00F3092
:10CF500000EB002000EB0040000E704707EE900A47
:10CF6000F5EEC07AF1EE10FA01D400F00BB8F1EE54
:10CF7000677A08B517EE900A00F004F8404261EBBA
:10CF8000410108BDD0B5FFF7BFFA0C4B00220646A1
:10CF90000F46FFF711FBFFF7E7FD0446FFF792FA94
:10CFA000074B0022FFF708FB02460B463046394686
:10CFB000FFF74AF9FFF7D8FD2146D0BD0000F03D4C
:10CFC0000000F0412DE9F047089D04468E46002BF5
:10CFD0004DD18A42944669D9B2FA82F252B101FA2D
:10CFE00002F3C2F1200120FA01F10CFA02FC41EA3D
:10CFF000030E94404FEA1C48210CBEFBF8F61FFAC2
:10D000008CF708FB16E341EA034306FB07F199425C
:10D010000AD91CEB030306F1FF3080F01F8199420F
:10D0200040F21C81023E63445B1AA4B2B3FBF8F0E9
:10D0300008FB103344EA034400FB07F7A7420AD970
:10D040001CEB040400F1FF3380F00A81A74240F298
:10D0500007816444023840EA0640E41B00261DB103
:10D06000D4400023C5E900433146BDE8F0878B4238
:10D0700009D9002D00F0EF800026C5E900013046F7
:10D080003146BDE8F087B3FA83F6002E4AD18B42D1
:10D0900002D3824200F2F980841A61EB030301207B
:10D0A0009E46002DE0D0C5E9004EDDE702B9FFDE67
:10D0B000B2FA82F2002A40F09280A1EB0C014FEA12
:10D0C0001C471FFA8CFE0126200CB1FBF7F307FB6F
:10D0D000131140EA01410EFB03F0884208D91CEB12
:10D0E000010103F1FF3802D2884200F2CB804346AF
:10D0F000091AA4B2B1FBF7F007FB101144EA01448E
:10D100000EFB00FEA64508D91CEB040400F1FF311C
:10D1100002D2A64500F2BB800846A4EB0E0440EA0A
:10D1200003409CE7C6F12007B34022FA07FC4CEA13
:10D13000030C20FA07F401FA06F31C43F9404FEA06
:10D140001C4900FA06F3B1FBF9F8200C1FFA8CFE1B
:10D1500009FB181140EA014108FB0EF0884202FA6F
:10D1600006F20BD91CEB010108F1FF3A80F0888030
:10D17000884240F28580A8F102086144091AA4B2ED
:10D18000B1FBF9F009FB101144EA014100FB0EFE6E
:10D190008E4508D91CEB010100F1FF346CD28E459D
:10D1A0006AD90238614440EA0840A0FB0294A1EB2E
:10D1B0000E01A142C846A64656D353D05DB1B3EB8B
:10D1C000080261EB0E0101FA07F722FA06F3F140BB
:10D1D0001F43C5E9007100263146BDE8F087C2F162
:10D1E0002003D8400CFA02FC21FA03F391400143DA
:10D1F0004FEA1C471FFA8CFEB3FBF7F007FB103613
:10D200000B0C43EA064300FB0EF69E4204FA02F4BE
:10D2100008D91CEB030300F1FF382FD29E422DD911
:10D22000023863449B1B89B2B3FBF7F607FB163346
:10D2300041EA034106FB0EF38B4208D91CEB0101C6
:10D2400006F1FF3816D28B4214D9023E6144C91A46
:10D2500046EA004638E72E46284605E70646E3E656
:10D260001846F8E64B45A9D2B9EB020864EB0C0E60
:10D270000138A3E74646EAE7204694E74046D1E76F
:10D28000D0467BE7023B614432E7304609E764441D
:10D29000023842E7704700BF02E000F000F8FEE706
:10D2A00072B6374880F30888364880F309883648D4
:10D2B0003649086040F20000CCF200004EF63471AE
:10D2C000CEF200010860BFF34F8FBFF36F8F40F2C3
:10D2D0000000C0F2F0004EF68851CEF20001086066
:10D2E000BFF34F8FBFF36F8F4FF00000E1EE100AD6
:10D2F0004EF63C71CEF200010860062080F31488DF
:10D30000BFF36F8FB6F052FAB7F09CF94FF055307B
:10D310001F491B4A91423CBF41F8040BFAE71D49E3
:10D32000184A91423CBF41F8040BFAE71A491B4ADC
:10D330001B4B9A423EBF51F8040B42F8040BF8E72E
:10D3400000201849184A91423CBF41F8040BFAE703
:10D35000B6F030FAB7F0CAF9144C154DAC4203DA06
:10D3600054F8041B8847F9E702F052F8114C124DAB
:10D37000AC4203DA54F8041B8847F9E7B6F018BA50
:10D38000000600200022002000C0000808ED00E098
:10D390000000002000060020580F0F080022002087
:10D3A000302C0020302C0020704D0120E0C10008FE
:10D3B00040C2000840C2000840C200082DE9F04FFA
:10D3C0002DED108AC1F80CD0C3689D46BDEC108AC3
:10D3D000BDE8F08F002383F311882846A047002082
:10D3E000B5F066F9FEE7B4F0C3FF00DFFEE700002A
:10D3F00001F0FF01102A2BDB10F0070F08D010F806
:10D40000013B013A8B422DD010F0070F42B3F6D109
:10D41000F0B441EA012141EA014122F007047FF022
:10D4200000070023F0E80256083C85EA010586EA79
:10D43000010685FA47F5A3FA87F586FA47F6A5FAB5
:10D4400087F68EB9EED1F0BC01F0FF0102F00702C1
:10D4500032B110F8013B013A83EA010313B1F8D16C
:10D460000020704701387047002D06BF354603384D
:10D47000073815F0010F07D1013015F4807F02BF86
:10D48000013015F4C03F0130F0BC0138704700BFD7
:10D4900010F8012B11F8013B012A28BF9A42F7D05E
:10D4A000D01A7047034613F8012B002AFBD1181A33
:10D4B0000138704738B50022002304460D46FFF7B7
:10D4C000EDFA28B920462946BDE8384000F00AB8F0
:10D4D000204605F1004100F005F8404261EB4101B2
:10D4E00038BD00BFD0B50C4B002206460F46FFF7F3
:10D4F00063F8FFF739FB0446FEF7E4FF074B002211
:10D50000FFF75AF802460B4630463946FEF79CFEB6
:10D51000FFF72AFB2146D0BD0000F03D0000F0419E
:10D52000036800221B6818477FB503914021054618
:10D530007FF0CCFA039A18B90124204604B070BDDC
:10D54000134E039296F94232002BF5D061F0BAFCEB
:10D55000437A039A53B961F0B5FC847A039A2CB9E3
:10D560000C4B402128467FF0B9FAE6E7D6F8F43BA9
:10D57000B6F94412B3F906309942DDDD064B00934B
:10D580004021064B28467FF0A9FA0024D5E700BFCA
:10D59000384C002064C00C0883C00C0871C00C0813
:10D5A0002DE9F0410D46B4B0202104467FF08EFAFB
:10D5B000002800F0AE80584E96F94232ABB1D6F852
:10D5C000F42BB6F94432B2F90A1003F10A0291427F
:10D5D00003DD40F28D32934207DC504B2A46202176
:10D5E00020467FF07BFA002090E096F93132022B42
:10D5F00005D14B4B2A46202120467FF06FFAB6F822
:10D600000432A3F57A739BB241F6583293420DD897
:10D61000444F96ED9C7AD7F8343CD3ED097AB4EEBA
:10D62000E77AF1EE10FA03DD3F4BD7E73F4BD5E742
:10D6300096ED9D7AD3ED0B7AB4EEE77AF1EE10FA1F
:10D64000F2DCB6F93E32002B01DC394BC6E7002193
:10D65000602203A80DF108080291BAF0D5F86422FF
:10D66000414607F6E85085F027FF40B9314BCDF829
:10D6700000802A46202120467FF030FAB3E761F08F
:10D6800021FC202162F022FC08B92B4BA6E72B4895
:10D690000FF048FD012806D1D7F8400C86F0C2FBF8
:10D6A00098B1012815D0002160221CA81B91BAF066
:10D6B000ABF82349D7F83C0C64231BAA85F0BCFDCA
:10D6C000D8B91BAB00931F4BD3E71F4B00931F4BE5
:10D6D000CFE796F8083C73B11D4819214FF01EFAA8
:10D6E00048B11B48D6F81C6219214FF03DFA86421A
:10D6F000D9DD184BEAE7184BE8E71849D7F8340C9E
:10D7000064231BAA82F058FC0028DAD034B0BDE8AC
:10D71000F0810120FAE700BF384C002090C00C08CF
:10D72000A3C00C08386C0020DBC00C08CBC00C0870
:10D73000F5C00C084E1B0D080AC10C08A883002078
:10D7400083C10C0887C10C084EC10C0829C10C0804
:10D75000783900206DC10C085EC10C0899C10C0815
:10D7600007B5044887F0B6FE00F0010003B05DF88D
:10D7700004FB00BF507800202DE9F043DFF844910E
:10D780000446D9F804000368A5B01B690D46984704
:10D79000804614F04BFF0021074660220CA80B9135
:10D7A000BAF032F864230BAA4146384614F046FA20
:10D7B000064648B93A4A0BAB294620467FF096FB0D
:10D7C000304625B0BDE8F083A9F575606DF040FAEC
:10D7D000B8F1000F03D194F91E30012B0AD1314862
:10D7E00011F052FF80B9304A294620467FF07EFB77
:10D7F0000026E5E710F0060FE2D0A9F5405011F041
:10D8000043FF08B9294AEFE703A9384614F048F85E
:10D8100028B19DF80D305B0601D5254AE4E7DFF815
:10D82000A880D8ED987AF5EEC07AF1EE10FA4FF0B4
:10D830000003C5DD089309930A930DF1200907AB96
:10D84000019305AA06AB04A9CDF80090384614F060
:10D8500009FC48462FF0B8FAD8ED987AB4EEE70AFA
:10D86000F1EE10FA01DB134ABEE79DED057AF4EE06
:10D87000C77AF1EE10FA01D80F4AB5E79DED047AA8
:10D88000F4EEC77AF1EE10FA01D80C4AACE79DED40
:10D89000067AF4EEC77AF1EE10FA91D8084AA3E7B7
:10D8A000A0C10C08382C0020A9C10C08C0C10C086C
:10D8B000E6C10C08F4C10C0809C20C081FC20C0810
:10D8C00035C20C08385C0020384C002008B5054BE8
:10D8D0005B7F9B0704D5044A7FF008FB002008BD4E
:10D8E0000120FCE7385C00204CC20C0870B50C4CE1
:10D8F0000546606803685B690E46984710B10124CD
:10D90000204670BDA4F5405011F0D0FE044600281A
:10D91000F5D1044A314628467FF0E8FAF0E700BF27
:10D92000385C00205CC20C082DE9F046454EB36A15
:10D9300093F8CB509BB081468A4665B9424B1B6831
:10D94000986A03685B6B9847044640B93F4A514662
:10D9500048467FF0CBFA28461BB0BDE8F08661F060
:10D96000B1FA202162F0B2FA58B161F0ABFA1F218E
:10D9700062F0ACFA88B3364A514648467FF0B6FAB0
:10D980000024344B93F8FA3F03F01403142B05D111
:10D99000314A514648467FF0A9FA0024514648468C
:10D9A00080F03EF9002188424FF0600202A808BFD3
:10D9B0000C460191B9F028FFB06A036801AA1B6800
:10D9C00064219847054680B9244A01AB5146484630
:10D9D0007FF08CFA2C462546BDE761F073FAA5214D
:10D9E00062F074FA0028C6D1CBE7002CF3D0D9F846
:10D9F00008303BB9D9F8003051465B6B4846984730
:10DA00000446E8E751464846FFF7CAFD5146074637
:10DA10004846FFF75BFF3840C4B251464846FFF71F
:10DA200083FD514604404846FFF760FF51460440DD
:10DA300048467FF083FA51460440484680F008F992
:10DA40000440C8E7385C00203086002070C20C0813
:10DA500087C20C08384C0020A1C20C08B9C20C08BF
:10DA600008B5FFF761FF054A92F8F81F60F304114B
:10DA700082F8F81F024A907108BD00BF384C0020A0
:10DA80000D880020F7B505460F467FF05BF8044689
:10DA900078B1022128467FF019F8064648B11548AA
:10DAA00087F018FDC205C0F30723C0F3002403D597
:10DAB0003446204603B0F0BD9B07F9D50D4887F0EA
:10DAC00017FD0D4B03F6E433D3ED007AF8EEE77A59
:10DAD00030EE670ADFED097AB0EEC00AB4EEE70A6D
:10DAE000F1EE10FAE4DD064B3A46022128467EF0BC
:10DAF000F5FFDEE750780020386C00200000C842B7
:10DB0000C4C20C08F8B504460F467FF0B7FA1021DE
:10DB1000054620467EF0DAFF58B12046FFF720FE8A
:10DB2000064630B9044B3A46102120467EF0D6FF17
:10DB300035462846F8BD00BFD8C20C0870B505466A
:10DB40000E467EF06BFF044678B1802128467EF0B9
:10DB5000BDFF50B1074B93F8C53543B1064B324674
:10DB6000802128467EF0BAFF0024204670BD04467E
:10DB7000FBE700BF385C0020ECC20C0838B50D4D47
:10DB80000446D5F8400C86F04DF9012810D0D5F8A0
:10DB9000400C86F047F9022804D02046BDE8384002
:10DBA0007EF03EBF04480FF0BDFA0128F5D138BD24
:10DBB0000020FCE7386C0020A8830020F0B5114C51
:10DBC00085B0D4F8EC3B0093D4F8F03B0193D4F843
:10DBD000F43B02936A46D4F8F83B039306460F469B
:10DBE0007FF0D0FF3946054630467EF0D1FF94F8ED
:10DBF000F83F284060F3C303C3F3C00084F8F83F44
:10DC000005B0F0BD384C00202DE9F8430646274802
:10DC1000DFF8A890DFF8A8800F466DF019F80446E9
:10DC2000D9F8040003681B699847054630B914F019
:10DC3000060F03D1D9F83830022B09D139463046C6
:10DC40007FF078F8054618B9002488F807400AE004
:10DC500039463046FFF790FD04460028F4D02DB930
:10DC6000012388F807302046BDE8F88308213046B4
:10DC70007EF02CFF0028F3D00D4822F02BF900286D
:10DC8000EED00C4B93F81424B02101FB023203F5C3
:10DC90000053B2F81E22B3F932329A42E0DD064B4D
:10DCA0003A46082130467EF019FFCDE7E84C0020C7
:10DCB000582D0020382C002000C30C08385C0020B0
:10DCC0000D8800202DE9F3410E46054614F0AEFC08
:10DCD000804613F0A7FD044640B9454A0121284675
:10DCE0007FF004F9204602B0BDE8F081414F78682A
:10DCF000036831469B699847044650B978680368C1
:10DD00005B6C98473C4A0346012128467FF0EEF8B9
:10DD1000E8E7AB68002BE5D0102128467EF0D6FE60
:10DD200020B3D8ED937A98ED920A20EE270AB7F047
:10DD300073FADFED327AA7F5805320EE270AB3F9A4
:10DD40000432DFED2F7A20EE270A07EE903AF8EE44
:10DD5000E77AB4EEE70AF1EE10FA07DD294B01226B
:10DD6000102128467EF0BAFE0024BBE74021284659
:10DD70007EF0ACFE30B3012E1ED0232E1CD0042E1C
:10DD80001AD02148D0F8F43BB3F9083000EE103A2D
:10DD9000A0F50050B8EEC00A00F08EFBB5EEC00A48
:10DDA000F1EE10FA0EDD194B00930122184B4021C1
:10DDB00028467EF093FED7E778680368DB6B9847C8
:10DDC0000028DED0134B1B68D86A0368DB699847CC
:10DDD0000128014604D1104A28467FF087F8C3E79E
:10DDE0003146284602B0BDE8F0417FF00FBC00BFCD
:10DDF00010C30C08385C002021C30C08E02E6542DB
:10DE00000000C84235C30C08384C002083C00C0801
:10DE10003DC30C083086002049C30C0870B5054688
:10DE20000E46FFF7A9FC084B0446D8713146284638
:10DE3000FFF75CFD31460028284608BF00247FF02C
:10DE400089FD204070BD00BF0D880020F8B54B4F04
:10DE50003B78002B40F08F80494DAC6A94F8CB4062
:10DE600001263E7014B13B702046F8BD7FF098FF4C
:10DE7000044630B9434A3870137843F001031370F5
:10DE8000F2E756F021FA314655F058FBA5F540501F
:10DE900006F076F93C4B1E710B2649F067FD013EFA
:10DEA00049F01AFD16F0FF06F7D1384800F00CFFD4
:10DEB00014F0BCFBD0F800222A6590F87C32DA0717
:10DEC00049D413F031FF56F0FFF93C2156F038F9F0
:10DED00000232B6100212D4800F078FF2B4811F022
:10DEE000D3FB01462A488BF05FF92A4B1B68D86A9E
:10DEF000036801211B689847A86A03689B6A9847D2
:10DF00000121A86A8AF070F956F0DEF906466868C1
:10DF1000214D03681B68984795F8C4210146304697
:10DF200055F0E4FCA5F5005006F01CF953F0C4FBD5
:10DF300052F004FF00233B7090F0A0FE05F5005363
:10DF4000C3F84C0CB5F8FA3F23F4087343F02003F0
:10DF5000A5F8FA3F88E79B07BCD431460B4804F08C
:10DF60001BFF0E4887F0C4FADFED0D7A20EE270A7A
:10DF700085ED040AAEE7002476E700BF302C0020D0
:10DF8000385C00202C8800200D880020382C0020D0
:10DF90003456002030860020384C00205078002075
:10DFA0000AD7233C2DE9F043DFF8F880D8F8283071
:10DFB00093F8CB3087B0002B67D06AB1012901D02C
:10DFC000232909D1324B93F9F83F002B04DB0024BD
:10DFD000204607B0BDE8F0837FF08EFF044600289E
:10DFE000F5D014F023FB06461AF012FC0746304623
:10DFF00013F022F9D8B197F92430022B17D100255C
:10E000004FF00009E9B203AA30460191CDF80C9017
:10E01000CDF81090CDF8149013F0ACFC019918B124
:10E0200003AA38461AF0F2F80135032DEAD119484F
:10E03000012106F081FC1748012106F053FC002164
:10E04000D8F828008AF0D0F8134831F0C7FB56F012
:10E050003BF9002155F072FA104B1B68D86A03682F
:10E0600000211B6898470A4B93F8FA2F6FF345126B
:10E0700083F8FA2FD8F80410094BCA1A51425141BB
:10E0800003F13C008EF0CCFFA2E70124A0E700BF23
:10E09000384C0020382C0020407B002030860020A7
:10E0A000DC7C0020385C002010B5054C60680368FB
:10E0B0005B6A984710B1A36A93F8CB0010BD00BF0C
:10E0C000385C002030B52DED028B89B00C46B0EEE7
:10E0D000408AFFF7E9FF0546002838D0B4EE488AA9
:10E0E000F1EE10FA7CBFDFED1C8ADFED1C7A2268AE
:10E0F00063689FED1A0A68BFDFED198A029278BF44
:10E1000068EE288A02A878BF68EEA78AD4ED027A62
:10E110000393F1EE677ACDED047A2EF057FAB4EE60
:10E12000488A00220123F1EE10FACDE900238DED9B
:10E13000050ACDED060A9FED0A0A0A488DED071A79
:10E14000F0EE680A68BF134605A90DF0CDF8284621
:10E1500009B0BDEC028B30BDE02E65420000C84224
:10E16000000000004C82002007B50191FFF79CFFE2
:10E1700030B10199044803B05DF804EB00F0D6BA61
:10E1800003B05DF804FB00BF382C002001486CF0A0
:10E19000EBBE00BFE84C002008B500F5005090F839
:10E1A000F83FC3F340128A420BD061F3451380F865
:10E1B000F83F31B156F088F8BDE808400F2155F01E
:10E1C000BFBF08BD70B500F540560546B36B8B4226
:10E1D0000C4611D0012910D0022915D059B956F09A
:10E1E00073F81B2155F0ACFF0C4A05F5375006219A
:10E1F000103058F089FAB46370BD56F065F81A21F2
:10E2000055F09EFF064AF0E7012100F0DFFD56F0D1
:10E210005BF81D2155F094FF024AE6E7B4C30C08F1
:10E22000C9C30C08C4C30C0810B500F540520C4615
:10E23000537F03F00101A14208D064F30003537738
:10E24000DB0704D405F092FB024B9C7210BD05F075
:10E250005DFDF9E70D88002000F54050437F61F334
:10E2600041034377014B1973704700BF0D880020AD
:10E2700000F5005090F8FA3F43F0040380F8FA3FAD
:10E280007047000010B5044653F016FA04F54052EA
:10E29000436F926A04F58044D360D4F8342C9366BB
:10E2A000D4F83C2CC2F8FC32D4F8340C03685B6D13
:10E2B0009847D4F8340C0368BDE810409B6D1847AC
:10E2C00070B52DED028B00F540550446AB6A93F80E
:10E2D000CB30002B6ED000F5005393F9F83F002BA4
:10E2E00068DB00F5804696F82C3E002B62D168680A
:10E2F00003685B69984700285CD1304B5868036815
:10E300001B6898470B2855D0D6F83C3C9FED2C7ADB
:10E31000D3EDDB7AF0EEE77AF4EEC77AF1EE10FA9D
:10E3200048D5A86A443057F003FC0346DFED250AC0
:10E3300093ED000A9F20B7EE001A2AF0C7FEB5EE53
:10E34000C00AF1EE10FA35DD04F59840183087F078
:10E35000DBF8DFED1D7AB0EEC00AB4EEE70AF1EEAD
:10E3600010FA27D5D6F8340C04F580540368D4EDA0
:10E37000FC7AD3F89830B8EEE78A984738EE400A2E
:10E38000DFED127AB0EEC00AB4EEE70AF1EE10FA51
:10E3900010D5D4F8F43340F2E63203F2F31393428B
:10E3A00008D8BDEC028BA86A9FED090ABDE8704051
:10E3B00087F00ABBBDEC028B70BD00BF385C00204B
:10E3C0000000003400000000000070420000FA432A
:10E3D0000AD7233C08B500F54050806A03681B69E2
:10E3E0009847F6EE007A20EE270AB5EEC00AF1EE65
:10E3F00010FA48BF9FED010A08BD00BF00000000F1
:10E4000038B52DED028B00F580450446D5F8343C37
:10E41000DFED100A93ED370A04F540547120B7EE92
:10E42000001A2AF053FEA06AD5F83C5C03681B6909
:10E43000B0EE408A984738EE400ABDEC028BDFED23
:10E44000067A05F50575284620EE270ABDE838400E
:10E4500077F044BC0000000000007A4400F58050D2
:10E4600000F5896300F25440D3ED005AD2ED007AF2
:10E47000D0ED006A91ED006A26EEE77A67EEA57AA4
:10E48000A6EE257AE6EE267A81ED007AC2ED007AD4
:10E490007047000000F50050B0F9AC3A33B9B0F95C
:10E4A0003E020028B8BF404280B2704783EAE37062
:10E4B000A0EBE370F8E7000070B52DED028B00F5DE
:10E4C000405382B0597F11F00106044605D09FEDFC
:10E4D0002E0A02B0BDEC028B70BD8DED010A60F01A
:10E4E000F1FC037F002BF2D0DFED288ADFED260A56
:10E4F0009DED010AB0EE681A4E202AF0E7FD04F502
:10E5000000554FF4C8723146B5F94602B0EE408A64
:10E510002AF01AFEA5F84602204610F03BFEB5F997
:10E52000463207EE900AB8EEE77A07EE903AF8EE38
:10E53000E77A77EE676AB4EEE68AF1EE10FA0DD567
:10E540002046FFF7A7FF07EE900A38EE668AB8EE7E
:10E55000E70A20EE088A88EE260ABAE777EE877A7D
:10E56000B4EEE78AF1EE10FAB1DDB5F93E3200EE15
:10E57000103A38EE678AB8EEC00A78EEE77A20EEF5
:10E58000088A88EE270AA4E70000000000007A4409
:10E5900000207047002070477047000000F50950C8
:10E5A000143070470048704720F40C0800F54050C4
:10E5B000406803681B6818470348086034211170DD
:10E5C00008221A60704700BFBCC70C0800F5405015
:10E5D000406803681B6D184700F5405040680368A9
:10E5E000DB6C184700F5405300F59D405B684C30EC
:10E5F0001B1A58425841704710B500F540500C4660
:10E60000406803681B6E984707EE900A9FED047AF6
:10E61000F8EE677A012067EE877AC4ED007A10BDC4
:10E620000AD7233C10B500F540500C4640680368FB
:10E63000DB6D984707EE900A9FED047AF8EEE77AD3
:10E64000012067EE877AC4ED007A10BD0AD7233C1B
:10E6500010B500F540500C46406803685B6E984763
:10E66000DFED037A20EE270A012084ED000A10BDB9
:10E670000AD7233C65F0B6BF62F00EBD52F066BF0C
:10E6800028F07CBC55F0D8B817F092BE63F084B87F
:10E6900060F072B85EF07AB910F050BA10F070BE47
:10E6A00006F08ABB11F0D0BE05F0B0B905F09EB8F7
:10E6B00004F0C6BF05F098BE67F014BD0FF0D0BBE4
:10E6C000FFF7FEBD10F076BB10F0B2BD03F06EBADE
:10E6D00010F0FCBA10F078BA60F042BB4AF06EBBA2
:10E6E00022F0A6BE05F0B6BD02F0ECBC63F064B843
:10E6F00010F0BCBD06F016BB04F03CBB06F066BCD7
:10E7000005F02EB806F068B805F0F4BE10F0A2B916
:10E7100006F00CB8FFF7B6BD28F04EBF05F070BB91
:10E720000AF042B90AF02EB809F0C2BF1FB500F5D1
:10E73000405304465868039103685B6A984760B188
:10E74000DFED070A0399002304F5AC400093B0EE17
:10E75000600A1A4614300CF01DFC04B010BD00BF56
:10E760000000000010B52DED028B00F5405304466B
:10E77000586803685B6AB0EE408A984720B9002465
:10E78000BDEC028B204610BD9FED080A04F5AC409D
:10E7900028EE000A14300BF0C7FE04460028EED025
:10E7A00003480121FFF7F8FCEAE700BF0000C84278
:10E7B000382C00200A4A92F9F82F002A0B4605DA75
:10E7C00000228A604A600A600120704700F580409C
:10E7D000D0F8342C783207CA83E80700F4E700BF8A
:10E7E000384C002038B54C4B044640F8043B66F0EA
:10E7F00019F804F1100017F081FA04F1680052F0E2
:10E8000033FC04F5907021F075FA04F58C6015F076
:10E8100099FF04F2845019F083FA04F6C80028F036
:10E8200051FA04F5476065F0DBFD04F554604EF0E5
:10E830009BF804F57F6054F0E1FD04F58550083045
:10E840006BF0E8FC04F58650043062F041FE04F5FC
:10E8500088507DF075FB04F588501C3052F0C6FFDF
:10E8600004F58B50103067F087F904F580530025CC
:10E870002A4A83F8945104F58D5004F58C531433CF
:10E880000430136048F09CFE04F58F502946183080
:10E8900012F0C2F904F5C250083077F05DFC04F5BF
:10E8A000E8500C307AF06CFB04F5F15004307CF049
:10E8B000A1FC04F5F45008307DF0D6F804F5F750CB
:10E8C00011F0ACFF04F5015078F028F904F502507E
:10E8D000134918304CF064FE04F5025030306CF0EF
:10E8E0005BF804F505502C307DF0C6FE04F50053AE
:10E8F00004F5075083F8C4510A4D1C307DF0DEFF4B
:10E900002B6813B1084890F087F9204607494CF06E
:10E9100047FE2C60204638BD48BE0D08BC91002043
:10E92000F8830E08EC880020D8C30C0850BD0D08F1
:10E9300010B510F0A5FB60F0C5FA0368BDE8104003
:10E940005B681847FFF7F4BF10B5044605F0E2FF17
:10E95000204610F0C3FE204605F09AFE204605F042
:10E9600023FF204604F056F82046BDE8104004F08E
:10E97000B9B90000FFF7E8BF70B500F5415514358F
:10E980000446284617F094F819F042FF90F9213018
:10E990008BB390F8403373B304F5405304F28456BC
:10E9A000986A443057F0C4F80346DFED130A93ED3C
:10E9B000000A9F20B7EE001A2AF088FB94F9B835B8
:10E9C000012B284608BF86ED0E0A002116F004FE32
:10E9D000DFED0A7A04F2DC7494ED287A20EE270A3F
:10E9E000DFED077AA7EE270A304684ED280ABDE856
:10E9F000704019F01DBE70BD00000000CDCCCC3DB4
:10EA00006666663FFFF7B8BF10B50121044610F0F7
:10EA10009FFE58B1114B586803689B6A984728B904
:10EA2000204602F05DFA204602F06AFA4FF4001127
:10EA3000204610F08DFE18B129F01AFE28F01EF8BD
:10EA40004FF48021204610F083FE28B129F010FEFB
:10EA5000BDE8104027F020BF10BD00BF385C00208B
:10EA6000FFF7D2BF70B500F580450446D5F8340CE9
:10EA70009FED530A86B06C302DF0A8FD04F58F5041
:10EA800003A918308DED030ACDED040A8DED051AAA
:10EA900011F06EFF0221204610F05AFE68B10121EC
:10EAA000204610F055FE40B9464B586803689B6AF3
:10EAB000984710B9204602F013FA0121204610F0C1
:10EAC00047FE40B93F4B586803689B6A984710B9A6
:10EAD000204602F015FA0121204610F039FE10B947
:10EAE000204602F065FA04F54056B06A03685B6C94
:10EAF00098474021204610F02BFE60B104F57F605E
:10EB0000019054F039F804F58053019893F9C4301A
:10EB10000BB154F073F94FF48061204610F018FEE9
:10EB200018B104F57F6054F0C1F82021204610F0A0
:10EB30000FFE40B1706803681B69984718B3D5F899
:10EB40003C0C83F0B5FA8021204610F001FE30B372
:10EB500029F08EFD27F0C4FE1021204610F0F8FDAC
:10EB600018B1D5F8340C80F047F94FF40041204635
:10EB700010F0EEFD10B304F59940543006B0BDE836
:10EB8000704062F04BBF20460DF0BCF80028D6D193
:10EB9000706803685B6998470028D0D0D3E74FF4CA
:10EBA0008021204610F0D4FD0028D1D14FF400215F
:10EBB000204610F0CDFD0028CAD1CDE706B070BDCB
:10EBC000E02E6542385C0020FFF74CBF10B50121F4
:10EBD000044610F0BDFD10B1204602F0E9F9802195
:10EBE000204610F0B5FD58B14FF48021204610F0BA
:10EBF000AFFD28B929F03CFDBDE8104027F04CBE20
:10EC000010BD0000FFF7E2BF10B5044605F0C6F9DD
:10EC1000204605F01FF8204605F006FA204611F0C0
:10EC200017FC2046BDE8104003F0D0BEFFF7ECBF54
:10EC300070B54FF6FF71044610F08AFD04F50055DB
:10EC400028B1D5F8F82F0721204602F0E1F904F5A4
:10EC50004056B36A93F8CB3053B92046FFF708FB10
:10EC6000B06A95F85A22036895F894121B6A98477F
:10EC700061F03CFF61F0EEFB204611F0E7FB95F8F8
:10EC8000F83F0F4A04F58044DB43D4F8345CC3F307
:10EC9000C01353712B681E6F52F00EFD52F076F9BF
:10ECA0002846B047D4F83C4C52F006FD04F50574F4
:10ECB00052F06CF92046BDE8704076F075BE00BF9A
:10ECC0000D880020FFF7B4BF70B500F5805606F53B
:10ECD000896300F540541B68E36306F2544305461C
:10ECE0001B682364D6F8F80300F58C4050302AF0F6
:10ECF000C1F9E36BA364236C6064E3644FF6FF71B6
:10ED0000284610F025FD38B1D6F8F8232846092109
:10ED1000BDE8704002F054B970BD000030B500F598
:10ED20004052946B002C50D000F5005393F8F91F1B
:10ED3000CD074AD56FF3000183F8F91FD3F8EC1B18
:10ED4000D3F8F05B012CB1F908400BBFD2ED105A9B
:10ED5000D2ED135AD2ED0F7AD2ED127A07EE104AA5
:10ED6000B5F9084006EE904A0CBFF8EEE66AF8EEF8
:10ED7000E66AB8EEC77A25EEE66A00F58050A7EE9F
:10ED8000276A00F5896200F2544067EEA67AD2ED58
:10ED9000006AE7EE257A90ED007A27EE877AA6EEF4
:10EDA000267ABDEEC77A17EE104A0C8192ED007AF2
:10EDB000D3F8F03B67EE877A90ED007AE6EE477A7B
:10EDC000FDEEE77A17EE902A1A8130BD38B5054678
:10EDD0002DED028B00F5405469B1284610F00AF879
:10EDE000636C1B1A03F2F31340F2E63293420BD822
:10EDF000BDEC028B38BDA36B022BF9D10FF0DEFF07
:10EE0000B0F57A7FE9D2F3E7606400F58C405030CA
:10EE1000642390FBF3F308EE103ADFED097AB8EEC5
:10EE2000C88A28EE278AB0EE480AB6F03BF884ED8F
:10EE3000120AB0EE480AB6F08BF984ED130AD7E750
:10EE400035FA8E3C00F58F500121183013F066BB67
:10EE5000FFF7F8BF10B5044610F0A2F910212046C4
:10EE600010F076FC70B1204601F096FF4FF40011CF
:10EE7000204610F06DFC28B929F0FAFBBDE81040DF
:10EE800027F0FCBD10BD0000FFF7E4BFF8B5044655
:10EE9000254605F0CDFF224B45F83C3B214BA465B0
:10EEA000C4E91734204BC4E91934204BE36604F15C
:10EEB000800018F0A3FB04F19C0018F09FFB04F104
:10EEC000B80018F09BFB4FF6FF76194BC4F8CC3016
:10EED000A4F8D06004F1D40018F090FB4FF0FF3795
:10EEE000144B1549C4F8307128461D604CF058FB8E
:10EEF000A4F87870A4F8946004F5A27018F07EFB72
:10EF000004F5B07018F07AFB04F5BE7018F076FBCB
:10EF1000002384F89031C4F8B4312046F8BD00BF16
:10EF2000D8210D0821E7000825E7000829E7000897
:10EF30000000FFFFDC870020B88D0D0810B50446E7
:10EF400005F076FF0A4B23600123A38704F14000FC
:10EF500018F054FB04F1500018F050FB04F160006D
:10EF600018F04CFB04F1700018F048FB204610BD6F
:10EF7000AC2A0D082DE9F043044689B0FFF732FCB6
:10EF8000AA4B236004F50A5004F5005502F074F909
:10EF900004F50953083304F53057C5F8003C06233F
:10EFA00085F8043C4FF07C5805A907F11000CDF816
:10EFB000148056F0B9FE07F128008FF009F804F527
:10EFC00098460023183604F5315785F8403C19233C
:10EFD00004A985F84C3CC5F8486C07F11800CDF839
:10EFE000108056F0A1FE07F130008EF0F1FF4FF0D7
:10EFF0000108182304F5325004F5345785F8943C81
:10F00000103785F8888CC5F8906C283061F072FE56
:10F0100038467DF00FFD06AE854BC5F8103D3146F4
:10F02000381D8DF818804DF0EFF804F53550083094
:10F0300049F082FE04F5365008307DF0E5FC7D4B4A
:10F040007D4FC5F8883D04F536503146203006978F
:10F0500056F06AFE04F5365031462C30069756F0CD
:10F0600063FE04F536503146383004F537580697BC
:10F0700008F1100856F058FE704BC5F8D03D08F165
:10F0800014008EF0A5FF04F5385704F539590837F8
:10F0900009F12C09384614375BF040FDB945F9D128
:10F0A0000723C5F8903F0023A5F8943F4FF4CB7099
:10F0B00018F02EFEC5F88C0F04F53E5018308EF077
:10F0C00087FF04F53F501C308EF082FF5C4B1A68BE
:10F0D0000AB9C3F8008004F5405704F5AF48594B0E
:10F0E000C5F8D03D384608F17C08C7F804800830E0
:10F0F0007EF022FF544B07934FF07E55534BFD6338
:10F10000BD640694009304F5415096E80C004FF45A
:10F110000071143016F012F904F5575008306FF0F2
:10F1200051FE04F5974003A96830039556F03AFE66
:10F1300004F5974003A97C30039556F0F5FD04F5DE
:10F14000984004F58045083018F058FA05F6184341
:10F1500000261E605E609E6005F6244304F598401C
:10F160001E605E609E6004F58F531833C5F8303C16
:10F17000002385F8513C4FF40041543016F09EFEB8
:10F1800004F59940543062F0F1FA04F59A40583091
:10F190006DF01CFD04F59B4014304DF06BF92C4BC9
:10F1A000C5F8943D04F59B402A4B2B49283004F5C3
:10F1B0009B49186009F148094CF0F2F9FF2385F8E2
:10F1C000D83D85F8E03D254948464CF0E9F9244B07
:10F1D0001F6817B123488FF01FFDC3F8009004F596
:10F1E0009B4909F16809204948464CF0D9F905F6D0
:10F1F000E85348465E601D494CF0D2F91C4B1D484F
:10F20000186004F59C4204323B464FF0140C9FB248
:10F210000CFB07010133097C0029F8D1164B1F8034
:10F22000164B1F6877B31648D5E700BFDCCB0C0838
:10F2300060C30C08A0C30C080000A040E8DD0D0866
:10F24000308C00205CCC0C081DE70008CCCB0C08EF
:10F25000B0C30C08C49100202CF00D0884820E0865
:10F2600054920020ECC30C08D8BB0E0818BC0E0842
:10F27000AC880020980F0D08AA880020688800201C
:10F280000DC40C0804F59C40042108301A6056F0A7
:10F29000F5FF04F59C4003A94E4B0393303056F024
:10F2A00043FD04F59C40503005F0C2FD4A4BC5F8C3
:10F2B000503E04F59D40103005F0BAFD04F5A1491B
:10F2C000464BC5F8903E04F59D4009F124094C30A9
:10F2D00004F5A045FFF7DAFD484605F0A9FD404BCF
:10F2E000C5F8A43009F13C008BF084F93D4BC5F81A
:10F2F000E03004F5AA40503005F09AFD3A4BC5F8CD
:10F30000503504F5AB4085F88C75103005F090FD54
:10F31000364BC5F8903504F5AB404C3005F088FD10
:10F32000334BC5F8087604F5AC40C5F8CC3514303D
:10F3300005F07EFD2F4BC5F8143604F5AC40C5F83A
:10F340005076583005F074FD2B4BC5F8583604F54F
:10F35000AD40203005F06CFD284BC5F8A03604F513
:10F36000AD405C3005F064FD254BC5F8DC3605F298
:10F37000547304F5AE401E605E607030FFF7DEFD32
:10F38000404605F055FD1F4BC5F8FC3704F5B0406D
:10F39000383005F04DFD1C4BC5F8383804F5B14048
:10F3A000A5F874780830FFF7C9FD184BC5F8883800
:10F3B000012385F8113905F6181504F5B2402E60C1
:10F3C0006E60AE6024300AF06DF9204609B0BDE8E9
:10F3D000F08300BFCDCC4C3DC81D0D08701E0D083C
:10F3E00080220D0814230D08D0230D0874240D0865
:10F3F000B8260D085C270D08F0270D088C280D088D
:10F4000030290D08102C0D08B02D0D08682B0D08A3
:10F4100038B5054B1C6823680A461D68034B014636
:10F420002046A847002038BD30860020382C002018
:10F4300038B5037904463BB905682DB1284626F056
:10F44000A5FB284618F066FC204638BD2D4B2E4AF9
:10F4500070B5036000F5A04300F5A845C3F8A420EB
:10F460002A4AC3F8E020044605F58A70FFF7E0FF5A
:10F4700005F5867004F5A745FFF7DAFF05F1D8001A
:10F48000FFF7D6FF05F1D000FFF7D2FF04F50053D8
:10F490001F4AD3F88C0FC3F8D02D08B118F03EFCEA
:10F4A0001C4B236004F5805393F87C2E42B9D3F8AB
:10F4B000785E2DB1284626F069FB284618F02AFC14
:10F4C00004F588507CF050FD04F58650043062F05D
:10F4D00017F804F6F44504F69446B54204D0183DF6
:10F4E000284625F0A9FFF8E70B4BC4F8C83804F606
:10F4F000C41055F0F9FF04F5136055F0F5FF2046F0
:10F5000070BD00BFDCCB0C0880220D083CD20E0879
:10F51000E8DD0D0848BE0D08E47F0D0810B58EF03B
:10F52000CDFF064C064B18602046FFF723FD204612
:10F53000044A0549BDE81040B5F08EBB382C0020C8
:10F5400030860020ECE600204DF4000801207047D2
:10F5500090F89C308B4286BF283150F82100002063
:10F560007047000090F89C308B4286BF283150F8DD
:10F570002100002070470000FA207047014B93F8EB
:10F580000A027047384C0020024B986B431E5842C9
:10F5900058417047385C0020024B986B831E5842DC
:10F5A00058417047385C0020034B986A08B188F0D6
:10F5B00017BF0248704700BF385C002048CC0C08D9
:10F5C00038B5C36A2E4D43F4E052C262026B42F476
:10F5D000E0520263426B42F4E0524263D5F83C2CA5
:10F5E0000446E2B143F4F843C362D5F83C0C82F020
:10F5F0001FF938B1236B43F480432363636B43F4F7
:10F6000080436363D5F83C0C82F034FA38B1236B45
:10F6100043F400532363636B43F400536363194B58
:10F620001D6845B1192128464DF078FA18B1E36AF2
:10F6300043F48073E362144B93F8083C6BB1236B83
:10F6400043F48073236345B1192128464DF09EFA97
:10F6500018B1636B43F480736363E36A43F08043E0
:10F66000E362236B43F080432363084B9B6A93F868
:10F67000C1301BB9636B43F08043636338BD00BF87
:10F68000386C0020B8880020384C0020385C0020FE
:10F6900013B54FF44470CDE9002118F033FB044654
:10F6A00028B1DDE900215EF045F9024B23602046D8
:10F6B00002B010BDA0CE0C080020704770470000BB
:10F6C0000320704708207047014B93F80C027047E5
:10F6D000384C0020034B93F98B02003818BF0120EF
:10F6E000704700BF384C0020014B93F90E02704761
:10F6F000384C0020704700007047000008B50C4BE4
:10F70000D3F83C0C68B910230A4A926A43F04000CF
:10F7100022B192F8CB200AB143F0C00040F00100C2
:10F7200008BD82F085F80028EDD01823ECE700BF73
:10F73000386C0020385C002038B5C5780B46352D74
:10F74000044628BF3525352200211846B8F05CF85C
:10F750002A4604F10C01BDE83840B8F00BB80000AF
:10F760001FB5184C94F82E10A4F5907011F040F8C5
:10F7700078B194F82E10A4F5907011F03BF840B1D8
:10F7800094F82E10A4F5907004B0BDE8104011F06C
:10F7900033B8002301930293039312F047FF01A9AA
:10F7A00012F024FD20B101A82DF00EFB04B010BD15
:10F7B00021F07CFE90F8F432B02202FB030090EDC1
:10F7C0003B0AF3E7384C002008B50D4B986AA8B106
:10F7D000443056F0ADF9034693ED000ADFED090A17
:10F7E0009F20B7EE001A29F071FCDFED077A20EEBA
:10F7F000270ABDEEC00A10EE103A18B208BD00BFCD
:10F80000385C0020000000000000C8422DE9F04FE5
:10F81000DFF8D880344F8DB00446042508F5005633
:10F8200017F8019BB8F9643209F1FF3A43FA0AF379
:10F83000D90742D5207C57F031FF8346207C58F011
:10F8400031FE00F121039B4505D2207C0DB0BDE8BF
:10F85000F04F57F079B9BAF1030F2ED8DFE80AF06C
:10F860000234393ED6F8340C03689B68984700F19F
:10F8700094035A69D3F800A0D3F804E0D868196952
:10F88000D3F818C008925A6A1B6ACDF82520CDF823
:10F89000293062222123CDE9003206900791207C95
:10F8A000CDF80CA0192303AAC221CDF810E0CDF8A1
:10F8B00014C08DF8249057F05BFF013D15F0FF0553
:10F8C000AED10DB0BDE8F08FD6F8340C0368DB681C
:10F8D000CCE7D6F8340C03681B69C7E7D6F83C3C84
:10F8E00003F52A73C5E700BF74CF0C08384C00201D
:10F8F00013B504460748019108F08CFE30B9019910
:10F90000204602B0BDE8104059F00CB8042002B007
:10F9100010BD00BF047B0020014808F059BC00BFA7
:10F92000047B002037B504460D4606480192114677
:10F930008AF06CF8019A2946204603B0BDE83040B1
:10F940005CF0C4BEF056002010B588B004465AF0F2
:10F95000E7F90B4B986A38B90A4A0621204608B0E5
:10F96000BDE810405AF0C4B969461E2288F03CFD3B
:10F97000054A6B46062120465AF0BAF908B010BD78
:10F98000385C002094CC0C084E1B0D08034A92F8FA
:10F99000E83B013382F8E83B59F086BA384C002046
:10F9A00007B50846019117F0FFFE38B104480199E8
:10F9B00002F0ACFE002003B05DF804FB0420FAE77F
:10F9C0003C860020F7B58B8BCD2B06460C461746A0
:10F9D0001DD1D1ED067AFCEEE77ACDED017A9DF8E6
:10F9E0000430022B13D10E4D95F84D1D05F6D44071
:10F9F00061F0F2FE58B195F84D1D05F6D44061F066
:10FA0000F3FE20B994ED020A064802F05FFE3A4682
:10FA10002146304603B0BDE8F04059F0D7BA00BFE8
:10FA2000386C00203C860020162A10B40C4605D005
:10FA3000542A03D05DF8044B58F090BF0323237081
:10FA400001205DF8044B704708B559F0E3F940F424
:10FA50001C6040F00D0008BD10B5044618F05AF9BE
:10FA6000204610BD10B50C4C94F9F83F002B0FDB6D
:10FA700004F58054606803681B6D984750B960684E
:10FA80000368DB6C984700280CBF0220032010BDE0
:10FA90000120FCE70420FAE7384C002010B44C6940
:10FAA000012C05D101465DF8044B034803F0BCB9B5
:10FAB0005DF8044B59F012BA382C00202DE9F341BF
:10FAC000B1F90430002B06460C46154635DB4FF0E5
:10FAD0000008CDE900281A4FB1F902209FED190A5C
:10FAE000D7F8EC1B4FF47A735DF0D8F80123CDE919
:10FAF00000539FED140AB4F90020D7F8F01B4FF41F
:10FB00007A7330465DF0CAF89FED0F0AB4F904200D
:10FB1000D7F8F41B43463046CDE900585DF0BEF8F7
:10FB2000CDE900589FED070AB4F90620D7F8F81B75
:10FB30004FF47A7330465DF0B1F802B0BDE8F08161
:10FB4000384C00200000FA4400007A44044B187836
:10FB500020B9044B93F8FA0FC0F38010704700BF30
:10FB6000B0870020384C00200C4B93F8C52582B993
:10FB70005A7F92060DD1A3F5805213F9083C002B51
:10FB800009DB92F8F93F13F0200F14BF0420012085
:10FB90007047052070470320704700BF385C002085
:10FBA00008B5074B93F95832032B03D0BDE8084042
:10FBB0005AF016B9034A02215AF09AF8042008BDF7
:10FBC000384C0020ACCC0C08094BD3F88C2292079F
:10FBD00001D458F0B7BE03F5005303F60C4393ED80
:10FBE000000ADFED047AB8EEC00A20EE270A70475B
:10FBF000384C00200AD7233C10B594B0044603A823
:10FC000017F0FCFC1C4B5868036803A99B6D9847D0
:10FC100078B3002103A817F089FD50B3247C8FF03E
:10FC20002DF8059BDDED047A0893069B09930023CC
:10FC3000F8EEE77A9FED117A0B930C930D930E93E8
:10FC40000F931093119312934FF6F853ADF84C3075
:10FC50000023962267EE877A8DF84E303323CDE964
:10FC60000032079007AA57212046CDED0A7A57F0B7
:10FC70007FFD14B010BD00BF385C00200AD7233CC4
:10FC800030B52DED0A8B764C05466068036899B057
:10FC90005B6A984700285BD004F50054D4F85036CE
:10FCA000062B00F2C980DFE803F00404045788AB98
:10FCB00053006C489FED6C8A0BF034FB9FED6B0A90
:10FCC0000168426883680D930BA80B910C922CF08D
:10FCD0007DFCF0EE489AB0EE40CAF0EE60BAB0EEAD
:10FCE000419AB0EE48AAF0EE488AF0EE48AAB0EE8B
:10FCF00048BA40F6F8542D7C8EF0C0FF00231593CF
:10FD0000169301238C228DF85E303323CDE9003227
:10FD10000B90B1EE499AF1EE688AB1EE488A0BAACF
:10FD2000552128468DED0CCACDED0DBA8DED0E9AFC
:10FD30008DED0FBACDED10AACDED118A8DED12AA81
:10FD4000CDED139A8DED148AADF85C4057F010FD9F
:10FD500019B0BDEC0A8B30BD42480BF0E3FA9FEDC1
:10FD6000430A0168426883680D930BA80B910C92BB
:10FD70002CF02CFC3B48F0EE60BAB0EE419AB0EEAD
:10FD800040CA0BF0D3FA9FED390A2CF01FFC35481E
:10FD9000B0EE40BAF0EE60AAF0EE418A0BF0CAFA7B
:10FDA0009FED320A2CF012FC4FF44064B0EE40AAF2
:10FDB000F0EE609AB0EE418A9DE72A489FED2A9ABC
:10FDC0000BF0B4FA9FED290A2CF000FC2548B0EEA8
:10FDD00040BAF0EE60AAF0EE418A0BF0ABFA9FED6C
:10FDE000230A2CF0F3FBF0EE49BAB0EE40AAF0EE95
:10FDF000609AB0EE418AB0EE49CA40F607447AE70D
:10FE00001848DFED198A0BF095FA9FED180A2CF0CF
:10FE1000DDFBF0EE68AAB0EE40AAF0EE609AB0EE1C
:10FE2000418AB0EE68BAB0EE689AF0EE68BAB0EE09
:10FE300068CA40F63F445EE79FED0B8A0024F0EE6F
:10FE4000489AB0EE48AAF0EE488AF0EE48AAB0EE22
:10FE500048BAB0EE489AF0EE48BAB0EE48CA4AE75F
:10FE6000385C00204C820020000000000AD7233CB0
:10FE70002DE9F0412DED068B3B4C94F8F93F9906A6
:10FE80008CB005466BD504F500579FED380AD7F8BE
:10FE9000340CDFED378A6C302CF098FB8DED041AB2
:10FEA00021EE281A04F58054BDEEC11A666895F853
:10FEB00010808DED020A11EE103A1DB23368CDEDBF
:10FEC000030ADB6D304660EE289A20EEA89A984728
:10FED00007EE900AF8EEE77A304667EEA87AFDEE74
:10FEE000E77A17EE903A1CB233681B6E984707EE1C
:10FEF000900AB8EE678AD7F83C3CDFED1E7A93EDA6
:10FF00000FAA336828EE288A5B6EB4EEE78AF1EE1A
:10FF100010FA58BFB0EE678A30469847BCEEC88AE0
:10FF20000023089318EE103AB7222AEE28AA20EEF2
:10FF3000280AADF82C301A23CDE900323E2105AA5B
:10FF40004046CDED059A8DED069A8DED07AA8DED13
:10FF5000090AADF82850ADF82A4057F009FC0CB05A
:10FF6000BDEC068BBDE8F081384C00209F0CB345FA
:10FF70000AD7233C00FF7F472DE9F04F2DED028B80
:10FF80001A4B047CD3F8343C8DB0D3F88480D3F87A
:10FF90008870D3F88C60D3F8905093ED258AD3F80D
:10FFA00098B0D3F89CA0D3F8DC908EF067FE0023C5
:10FFB0008DF82C3016222523CDE90032029002AABA
:10FFC000532120468DED078ACDF820B0CDF824A02E
:10FFD000CDF82890CDF80C8004970596069557F03B
:10FFE000C7FB0DB0BDEC028BBDE8F08F386C002074
:10FFF00070B58A7A4B7A43EA0223CA7A43EA02430B
:020000040801F1
:100000009D2B06460C4621D1134D95F84D1D05F646
:10001000D44061F0E1FBC8B195F84D1D05F6D44020
:1000200061F0EEFB022811D195F84D1D05F6D44084
:1000300061F0DAFB50B9D4ED057A9FED080A084863
:10004000F8EEE77A27EE800A02F040FB21463046C0
:10005000BDE8704058F028BE386C00200AD7233C19
:100060003C860020054B9B6A2BB193F8CA00002800
:1000700008BF042070470420704700BF385C002090
:1000800008B5034B586803681B68984708BD00BF54
:10009000385C0020024B93F8F90FC0F34010704712
:1000A000384C002070B52B4E2DED028B0546706844
:1000B00091ED018A036886B05B6A0C46984750B997
:1000C000BDEEC88A18EE103ADB0704D4022006B051
:1000D000BDEC028B70BDD4E904012AF0D1F80028F0
:1000E000F4D002A817F08AFA02AA214628465CF04A
:1000F00045FD0028EAD0184902A817F061FB034625
:100100000028E3D1DFED150A00900246B0EE600A48
:10011000134802A90AF03EFFD0B1706803685B6A19
:100120009847044608B10020D1E70E480222042176
:1001300004F0FAFF60B1DFED090A09480094234694
:10014000B0EE600A224602A90AF024FF0028EAD194
:100150000420BCE7385C002040780020000000004C
:100160004C820020382C002008B591F82030032B59
:100170001BD1D1ED027A9FED0E7A91ED060A0D4B5F
:10018000F0EEE77AF4EEC77ADFED0B7A5868F1EE1D
:1001900010FA4CBF0121002120EE270A0FF018FEB3
:1001A000002814BF0020042008BD0220FCE700BF87
:1001B00000000034385C00200000C84210B52DED6E
:1001C000028BD1ED007AF5EEC07AF1EE10FA82B032
:1001D0000C4604DA042002B0BDEC028B10BD9FED8A
:1001E000197AF4EEC77AF1EE10FAF3D891ED030A1A
:1001F0009FED158AF0EEC07AF4EEC87AF1EE10FAAF
:1002000019D5D4ED037A1148D4ED010A94ED000A12
:10021000F4EEC87AD4ED027AFDEEE77AF1EE10FA48
:10022000CDED017A9DF90410ACBF0122002202F04D
:10023000B1F90020CFE7F7EE000A28F043FE0028CE
:10024000C8D0DEE70000B443000000343C86002044
:1002500091ED010AB5EEC00AF1EE10FA08B501DC25
:10026000042008BD9FED0F7A0F4BD1ED007A58683E
:1002700020EE070A9FED0D7A0368F4EEC77AF1EEDF
:1002800010FA05DD1B6F98470028E9D00020E8E749
:100290009FED077AF4EEC77AF1EE10FACCBFDB6E71
:1002A0009B6EF0E70000C842385C00209A99394004
:1002B0003333F33F08B5D1ED007A9FED157AF0EEB8
:1002C000E77AF4EEC77AF1EE10FA1DD5D1ED017A96
:1002D000F0EEE77AF4EEC77AF1EE10FA14D50D4895
:1002E0000222032104F020FF80B10A480121FDF71A
:1002F00053FF094890F80C3F012B03D000F608701B
:100300002FF0C2FC002000E0022008BD0420FCE722
:1003100000000034382C0020386C002010B5D1EDDE
:10032000007AFCEEE77A17EE903A9CB2012C02D0EC
:10033000022C06D04CB90648214666F055F800203C
:1003400010BD044802F078FFF9E70420F8E700BF89
:10035000E0790020382C00201FB5D1ED017A0B7C0C
:10036000FCEEE77ACDED027AD1ED007A0093FCEE57
:10037000E77AD1ED030ACDED037A91ED020A9DF8FB
:1003800008309DF80C20014602480EF0C9FA05B06D
:100390005DF804FB382C002010B5094C637FDB07A7
:1003A0000CD402220521A4F5405004F0BDFE28B96A
:1003B00002221146A4F5405004F0B6FE002010BD04
:1003C000385C002010B5D1ED007AFCEEE77A0446E7
:1003D00017EE903A13F0FF030ED10E4B58680368E6
:1003E000DB6F984708B1002010BD0B4A204606215C
:1003F00059F07EFC0420F7E7012B09D1054B586822
:100400000368D3F8803098470028ECD1034AEDE721
:100410000220E9E7385C0020D0CC0C08E0CC0C08C6
:100420009FED0B7A01F10C03F1EC017AF4EE677A9F
:10043000F1EE10FA0AD6F0EEE77AF4EEC77AF1EEB2
:1004400010FA03DC9942EFD1012070470020704779
:1004500000007A4430B52DED028B8DB000230546A7
:1004600003930493059312F0E1F803A911F0BEFE83
:1004700058B312F0DBF800F55A7393E8070006ACA6
:1004800084E80700DDED060A9DED070A2D7CF1EEFC
:10049000600AB1EE400AB4F027FF2046B0EE408A71
:1004A0002CF092FCDFED0B7A089B0B93012228EED7
:1004B000278A0C23CDE90032A82109AA28468DED10
:1004C000098A8DED0A0A57F053F90DB0BDEC028B85
:1004D00030BD00BFE02E6542242938B505460FD057
:1004E00003D81B2907D1012412E04029FBD0A1F138
:1004F0004203012BF7D92846BDE838405CF02ABDFD
:100500000C2156F033FB044610B12846FFF7A2FF3A
:10051000204638BD38B5174C637FDB070D4609D43C
:10052000A36A93F8CB303BB901221146A4F53C7085
:10053000FDF78CFC002038BD14F9083C002B4FF06F
:10054000020211DA0521A4F5405004F0EDFD002867
:10055000F0D095ED000ADFED087A606820EE270AFA
:1005600001210FF035FCE5E70921A4F5405004F026
:10057000DBFDDFE7385C00200000C84210B5194CF5
:10058000637FDB070DD4A36A93F8CB304BB114F92A
:10059000083C002B07DA01220821A4F53C70FDF786
:1005A00001FD002010BDD1ED007A9FED0F7AF0EE35
:1005B000E77AF4EEC77AF1EE10FA05D50222114679
:1005C0000A4804F0B1FDECE7606803681B689847CF
:1005D0000428E6D0606803681B6898471428EDD1AA
:1005E000DFE700BF385C002000000034382C00201A
:1005F00073B58B8BC12B05460C4644D8BB2B0DD84D
:10060000202B63D02ED8113B99B2052918D9214649
:10061000284602B0BDE870405DF090BDBC3B052BA4
:10062000F5D801A151F823F0670701087107010807
:100630000F0601080F060108FF0601080B07010855
:10064000052BE4D801A151F823F000BF4D070108A4
:100650000F0601080F06010861070108730601086B
:1006600021070108732B2CD006D8542B58D0552BBA
:10067000CDD1022209216BE0B22BC8D102B0BDE876
:100680007040FFF7E5BD4AF21146B34254D00BD893
:10069000D12B40D0B3F5967F53D0D02BB7D102B039
:1006A000BDE87040FFF73ABE4AF21246B3423ED070
:1006B0004AF21346B342AAD102B0BDE87040FFF738
:1006C0005DBF02B0BDE87040FFF778BDD1ED007AA4
:1006D000F5EEC07AF1EE10FA4FDD9FED297AF4EED7
:1006E000C77AF1EE10FA48D8FCEEE77A254ACDED4C
:1006F000017A9DF80430A2F8BA3A00202EE0214693
:1007000002B0BDE87040FFF7CDBC214602B0BDE8A5
:100710007040FFF757BE02B0BDE87040FFF71CBE47
:100720002146284602B0BDE87040FFF71DBD02B06B
:10073000BDE87040FFF7EEBE02B0BDE87040FFF7C5
:100740002BBE02B0BDE87040FFF7B4BD0222052108
:100750000D4804F0E9FC0028CFD1042002B070BDA0
:1007600002220621F4E70221084806F07DF9F2E7AB
:100770000221064806F042F9EDE70220EEE700BF4D
:1007800000007F43384C0020382C0020047B0020E0
:1007900008B591ED007AF6EE007AB4EEE77AF1EE64
:1007A00010FA06DD044801220521FDF7FBFB0020BD
:1007B00008BD0420FCE700BF4859002030B52DEDEE
:1007C000028BCD7893B0272D28BF27250C462722F2
:1007D000002108A8B7F018F82A4604F10C0108A86F
:1007E000B6F0C8FF414B586803685B6A9847002819
:1007F00041D09DF8465068063DD400244FF07E530A
:100800002906049307940694059427D504A82BF091
:1008100087F9EA0701940294039405F006032ED4A5
:10082000002B2ED10D9B01930E9B02930F9B0393E4
:100830002F480AF05DF99DED100A044630B340F2EE
:10084000ED40B7EE001AFFEE000A28F03FFC284802
:10085000234601AA04A90AF053F90CE0099B04936A
:100860000A9B05930B9B069304A80C9B07932BF004
:100870005DF90028CDD113B0BDEC028B30BD062B45
:10088000D6D001211A480AF0CFF8F4E7DFED190AB3
:100890004FF49E60B7EE001A28F018FCF6EE000A3E
:1008A000B0EE408A28F00EFBE8B9B6EE000A124B13
:1008B000B4EEC08AF1EE10FAD3F8403C08DD38EE11
:1008C000400A30EE008A93ED070A28EE000ABEE7E0
:1008D00030EE480AD3ED087A30EE000AF0EEE77AFF
:1008E00027EEC00AB3E79FED030AB0E7385C0020AB
:1008F0004C82002000000000386C00202DE9F043FD
:100900009DB0814608460EA9FEF716FF844B586835
:1009100003685B6A984750B19DF86C30012B09D091
:10092000DA1F022A06D97F4801210AF07DF81DB09E
:10093000BDE8F083BDF86840A20504F0070604F0A6
:10094000380704F4E07501D5002DF0D04FF0000811
:10095000CDF81480CDF81880CDF81C803EBB9FEDFB
:10096000726A9DED107ADDED117ADDED0F6A27EEEA
:10097000067A67EEC67A66EE866A083B012BCDEDF5
:10098000056A8DED067ACDED077A04D8674806AA88
:1009900005A9FDF763FD9DF86C30073B022B06D8D7
:1009A000634884F0A1FD014605A82BF02FFECDF889
:1009B0002080CDF82480CDF82880F7B9DDED147AB9
:1009C000129B0893F1EE677A139B099308A9484696
:1009D000CDED0A7AFFF724FD0028A4D09FED520A3E
:1009E00008A82BF047FE9DF86C30083B012B04D87B
:1009F0004E4809AA08A9FDF731FDCDF82C80CDF8A5
:100A00003080CDF83480EDB99FED476A9DED167AC0
:100A1000DDED177ADDED156A9DF86C3027EE067A6C
:100A200067EEC67A66EE866A083B012BCDED0B6A4F
:100A30008DED0C7ACDED0D7A04D83C480CAA0BA9AB
:100A4000FDF70CFD14F4806233D1DFED3A7A9DEDB1
:100A5000180A9DF86C1020EE270ADFED337A08396A
:100A6000012920EE270A8CBF0021012114F4006324
:100A700005BFDFED307ADDED190ADFED2F0A60EEFC
:100A8000A70A04BFDFED287A60EEA70AAEB9002FEF
:100A900035D1B3FA83F3B2FA82F25B0952090291BB
:100AA000019300920BAB08AA05A91E480AF02AF987
:100AB0003DE79FED210A0021D8E77FB9B3FA83F320
:100AC0005B0901200093B2FA82F3CDE901105B09C2
:100AD00014480BAA08A90AF0ADFB28E7002D7FF403
:100AE00022AF0120B3FA83F3B2FA82F2CDE900100B
:100AF0005B090C4852090BA90AF044FB17E7002DCB
:100B00003FF411AFB3FA83F3B2FA82F2CDE90016E3
:100B10005B09520905A903480AF076F907E700BF07
:100B2000385C00204C8200200000C842382C002095
:100B300050780020E02E6542000000002DE9F047CB
:100B4000A2B08046084614A9FEF7F6FD7E4B586811
:100B500003685B6A9847C0B1BDF88040A30504F004
:100B6000070904F4E07700D57FB10CAE304616F0EB
:100B700045FDB9F1000F29D1DDE9150129F080FB10
:100B800030B97248012109F04FFF22B0BDE8F0876B
:100B90009DF8841009AA40465BF0DAFF0028F0D0E7
:100BA000DDED177A9FED6A7A099B009367EE877AED
:100BB00010ADFDEEE77ADDE9151217EE903A284602
:100BC00016F03CFD95E80F0086E80F00002514F0B4
:100BD000380A06950795089514D1DDED1A7A189B09
:100BE0000693F1EE677A199B079306A94046CDED6F
:100BF000087AFFF715FC0028C3D09FED550A06A818
:100C00002BF038FD09950A950B959FB99FED506A19
:100C10009DED1C7ADDED1D7ADDED1B6A27EE067A6F
:100C200067EEC67A66EE866A8DED0A7ACDED096AC0
:100C3000CDED0B7A14F4806805BFDFED467A9DEDAB
:100C40001E0A9FED450A20EE270A04BFDFED407A19
:100C500020EE270A14F4006405BFDFED3E7ADDEDD7
:100C60001F0ADFED3D0A60EEA70A04BFDFED387A08
:100C700060EEA70AB9F1000F31D1BAF1000F52D1DD
:100C80003046CDED050A8DED040A16F0E7FC032889
:100C90009DED040ADDED050A3FF473AF10A930465F
:100CA000CDED050A8DED040A10951195129516F0FB
:100CB00035FE00283FF465AFB4FA84F46409B8FA4D
:100CC00088F3DDED050A9DED040ACDF804A000943B
:100CD0005B0906AA10A91D480AF084F855E7BAF185
:100CE000000F0FD10123B4FA84F4CDE901A3640904
:100CF000B8FA88F3154800945B0909AA06A90AF016
:100D000099FA42E7002F7FF43CAF0123CDE900734D
:100D1000B8FA88F2B4FA84F30C485B09520909A9BD
:100D20000AF030FA31E7002F3FF42BAFB4FA84F326
:100D3000B8FA88F2CDF800905B09520931460348B1
:100D40000AF028F921E700BF385C00204C8200201F
:100D50000000C842E02E65420000000010B44B7A4B
:100D60008C7ACA7A43EA042343EA0243542B07D01D
:100D7000562B09D0522B0BD15DF8044BFFF71EBD4B
:100D80005DF8044BFFF7BABD5DF8044BFFF7D6BE24
:100D90005DF8044B5CF0ACBB2DE9F0432DED028B0C
:100DA00000F5405604467068DFED4A8A036891B04A
:100DB0005B69984704F580490027002840F085804A
:100DC000D9F83C3CD3EDDE7A93EDD88AFDEEE77A94
:100DD00028EE288A17EE903A1DB204F5325808F131
:100DE000180801A940460EF045FB18B953F06CFAFB
:100DF000394B01933722002102A8B6F005FDA32349
:100E00008DF8083095238DF809308DF03FFFD9F823
:100E1000343CCDF80B00B06AD3F8DC20D3F8E030D6
:100E2000CDF80F104430CDF81320CDF8173054F022
:100E30007FFE0346DFED290A93ED000AB7EE001AA4
:100E40009F2028F043F910EE103AB06ACDF81B301D
:100E500003681B69984710EE103A04F59846CDF8E0
:100E60001F30183618EE103A3046CDF8233084F093
:100E70003FFB20EE280A404610EE103ACDF827300E
:100E8000D9F8E43BCDF82B30019BCDF82F300EF094
:100E900013FB10EE103A3046CDF83330CDF83770F2
:100EA000ADF83B5084F030FBBDEEC00A372210EEA7
:100EB000103A02A904F57F60ADF83D3052F056FBC0
:100EC00011B0BDEC028BBDE8F08308EE107A00256E
:100ED00083E700BF0AD7233C2292CA7F00000000AC
:100EE00010B500F58044D4F8340C7DF01BFED4F826
:100EF0003C1CD4F8340CBDE810407DF079BE0000F5
:100F000070B54FF4805104460EF022FC00284DD0FD
:100F100004F5804604F57F65D6F8340C03689B68B9
:100F20009847692100F19402284652F0B7F9D6F8A3
:100F3000340C0368DB6898476A2100F19402284664
:100F400052F0ACF9D6F8340C03681B6998476B2152
:100F500000F19402284652F0A1F9D6F83C2C6C21FD
:100F6000284602F52A7252F099F9202120460EF007
:100F7000EFFBD8B104F54053586803681B699847E4
:100F800078B1D6F83C2C284690326E2152F086F982
:100F9000D6F83C2C2846BC32BDE870406F2152F098
:100FA0007DB920460AF0AEFE0028EAD170BD0000EF
:100FB00008B511F03BFBBDE8084011F0C9B80000CE
:100FC0007FB50E464FF6FF71044615460EF0C0FB86
:100FD000E0B1102200216846B6F016FCA3238DF87C
:100FE000003095238DF8013003238DF802308DF009
:100FF0004DFE1022CDF80300CDF8071004F57F60F8
:1010000069468DF80B60039552F030FB04B070BD5B
:101010007FB50E464FF6FF71044615460EF098FB5D
:10102000E0B1102200216846B6F0EEFBA3238DF854
:10103000003095238DF8013004238DF802308DF0B7
:1010400025FE1022CDF80300CDF8071004F57F60CF
:1010500069468DF80B60039552F008FB04B070BD33
:1010600030B52DED048B87B004460D4618220021C3
:101070006846B0EE409AF0EE608AB0EE418AB6F073
:10108000C3FBA3238DF8003095238DF80130062390
:101090008DF802308DF0FAFD1822CDF80300CDF85E
:1010A000071004F57F6069468DF80B508DED039AAB
:1010B000CDED048A8DED058A52F058FA07B0BDECEB
:1010C000048B30BD10B54FF4801104460EF040FB88
:1010D00030B104F58F501830BDE810400FF022BD3C
:1010E00010BD00002DE9F0438FB014460546894637
:1010F0003122002101A8DDE916769846B6F084FB7E
:10110000A3238DF8043095238DF8053008238DF83E
:1011100006308DF0BBFD2368049363680593A368D4
:1011200006933B68CDF81D307B68CDF82130BB6855
:10113000CDF825303368CDF829307368CDF8070035
:10114000CDF80B10CDF82D303122B3688DF80F900B
:1011500001A905F57F608DF81C80CDF8313052F083
:1011600005FA0FB0BDE8F08370B52DED068B8CB09D
:10117000144605460E462C22002101A8B0EE409AE6
:10118000F0EE608AB0EE418AB0EE61AAF0EE429ACB
:10119000B6F03AFBA3238DF8043095238DF8053083
:1011A0000B238DF806308DF071FDDFED1A7A94ED8A
:1011B000007ACDF8070027EE277A29EE279A8DEDE1
:1011C000077A94ED017ACDF80B1027EE277A68EEB6
:1011D000A78A8DED087A94ED027A8DF80F6028EEDB
:1011E000278A67EE277A2C2201A905F57F608DED0D
:1011F000049ACDED058A8DED068ACDED097A8DED47
:101200000AAACDED0B9A52F0B1F90CB0BDEC068BE9
:1012100070BD00BFE02E6542A020704730B5144B72
:1012200089B004466946986A04F57F651E2287F0F6
:10123000DBF86A460F49284652F034FB04F5405368
:10124000586803681B68984704F50053014693F8F3
:10125000C421284652F04AFB04F58F50183011F093
:101260004BFC04F590701FF08BF909B030BD00BF46
:10127000385C00204E1B0D08274B70B543600446B8
:1012800018305DF09FFC254E254BA3616825601941
:101290005DF04EFE66513035B5F55A7FF7D1214DE0
:1012A00004F55A705FF0FAFA002104F27C7087F0BE
:1012B000AFFCC4F8305804F63800A5F6440588F0B1
:1012C0007DF99FED191ADFED190A9FED190AC4F88F
:1012D000C85804F6DC007DF07FFD9FED131A9FEDEA
:1012E000150AF0EE410A04F6F4007DF075FD9FED5D
:1012F0000E1A9FED100AF0EE410A04F60C107DF074
:101300006BFD20460C494AF04BF920460B494AF048
:1013100047F9204670BD00BFA8380020C0190D084D
:10132000D4190D085C850020000000009A99993EB0
:101330000000B44300804A43B80C0D08180F0D0894
:1013400070B5514D5149FAB0D022064646A8B6F0C4
:1013500011FA0FCD0EAC0FC40FCD0FC40FCD0FC4BB
:1013600095E80F0084E80F00002446AB181900210F
:10137000B7EE000A103449F049FCD02CF5D1444BAB
:101380000FCB02AC84E80F0001A9204649F0F2FB24
:1013900090B19DF90430DFED3F6AE06807EE103A46
:1013A000B8EEC77AF0EE007AE7EE267AB7EE000ADA
:1013B00080EE270A4AF09CFC00240EAB181900218D
:1013C0001034B7EE000A49F021FC402CF5D1324C24
:1013D00032480F214AF0CAFC0FCC1EAD0FC50FCC0E
:1013E0000FC50FCC0FC594E80F0085E80F00002251
:1013F00004211EA849F0B6FC96F9A469D6B91034A8
:101400000FCC2EAD0FC50FCC0FC50FCC0FC594E878
:101410000F0085E80F00324604212EA849F0A2FCF7
:101420009FED1F0A1F484AF063FC1F48B7EE000AF1
:101430004AF05EFC1D4C9FED1E0A0FCC06AD0FC599
:1014400094E80F0085E80F00002106A849F0DEFBB4
:101450009FED170A0021284649F0D8FB04F110013E
:1014600060222EA8B6F086F900242EAB18190021B0
:10147000B7EE000A103449F0C9FB602CF5D15EF0DC
:1014800073FF7AB070BD00BFECBA0C081CBA0C0830
:101490002CBB0C08CDCCCC3D3CBB0C08F0160D0889
:1014A00000000000880B0D08970B0D08BCBB0C0852
:1014B000000034422DE9F04790B00DF106011D20E7
:1014C0005FF022F8002800F09E809DF80630614A07
:1014D0000133DBB211210BA88DF806308CF09EFD94
:1014E00000220DF107010BA849F0CAF89DF806305B
:1014F000594A112105460BA88CF090FD00220DF1F0
:1015000007010BA849F0BCF89DF80630534A112199
:1015100006460BA88CF082FD00220DF107010BA8F6
:1015200049F0AEF89DF806304D4A03F03F03112113
:1015300007460BA88CF072FD00220DF107010BA8E5
:1015400049F09EF88046002D5DD0002E5BD0002F24
:1015500059D0002857D0284649F0AAFA002852D17D
:10156000304649F0A5FA00284DD1384649F0A0FA96
:10157000002848D1404649F09BFA002843D1394C15
:1015800094E80F000DF10C0C10348CE80F0094E877
:101590000F000DF11C0989E80F0002A9604649F00F
:1015A000E9FA98B3BDF8084002A9484649F0E2FAC2
:1015B00000284AD0BDF8083054BB23B340F2E244BF
:1015C0009C420FFA84FA0FFA83F927D80DF10A0129
:1015D0003046ADF80A904AF097FE0DF10A01284610
:1015E000ADF80AA04AF090FE0DF10A013846ADF8B8
:1015F0000AA04AF089FE00230DF10A014046ADF829
:101600000A304AF09BFE10B0BDE8F0870024CBE71B
:1016100040F2D662002B08BF1346D1E70DF10A0154
:101620003046ADF80AA04AF06FFE0DF10A012846D7
:10163000ADF80A904AF068FE0DF10A013846ADF89F
:101640000A904AF061FE0123D6E7002CDBD040F27D
:10165000D663B5E7A80B0D08B40B0D08C00B0D0839
:10166000CD0B0D083CBC0C0837B500F508517822AD
:101670000831044650F044FB00220C21254849F073
:1016800071FB2046FFF716FF04F508500022B7EE65
:10169000000A02211C3049F0EDFB012504F502513E
:1016A0001D4A009500233031452049F05FFB1B4A5D
:1016B0001368D90708D41A49156004F501530B6063
:1016C00004F585530833CB601549022204F50A500E
:1016D000012549F09DFB134A0095002304F57F6125
:1016E000FD2049F043FB104B1A68D20705D40F4A7E
:1016F0001D6004F588541C3414600C48012149F025
:10170000A3FB4AF053F90A4A138843F001031380FC
:1017100003B030BDF80B0D08EC7C0E0834860020B9
:1017200000220020E0C40D08388600201822002086
:101730009C8800202DE9F04F2DED028B00F5005024
:10174000D1B090F99432062B40F0BA8095495022DE
:1017500028A8B6F00FF828AD002428460021B7EEDF
:10176000000A013449F052FA052C05F11005F4D1B4
:1017700005A928A849F0FEF906A980462CA849F039
:10178000F9F907A9074630A849F0F4F908A906466F
:1017900034A849F0EFF9844B05460FCB18AC84E828
:1017A0000F0003A9204649F0E5F9002870D0002178
:1017B000B7EE000A204649F029FA7C499FED7C8A61
:1017C000802228A8B5F0D6FF28AC002520460021AD
:1017D000B0EE480A013549F019FA082D04F1100459
:1017E000F4D1744D0FCD08AC0FC40FCD0FC40FCD85
:1017F0000FC495E80F00002584E80F0008AC2046D0
:101800000021B7EE000A013549F000FA042D04F179
:101810001004F4D16848002207A948F031FFB8B19C
:10182000B0F90030642B13DD07EE903AB8EEE70A0A
:10183000DFED5F7A604820EE270ABCEEC00A10EEAA
:10184000103A9BB200EE103AB8EE400A4AF0CCFAD9
:101850005A4D9FED578A0FCD18AC0FC40FCD0FC452
:101860000FCD0FC495E80F0018AD84E80F000024D9
:1018700028460021B0EE480A013449F0C7F9042C8B
:1018800005F11005F4D151B0BDEC028BBDE8F08F2D
:10189000B8F1000F03D117B90EB9002D8DD048480B
:1018A000002204A948F0ECFE002886D049F000F997
:1018B000002882D19FED430A41484AF095FA7CE71F
:1018C0000B2B7FF47AAFA0223F490DEB0200B5F05D
:1018D00051FF28AD002428460021B7EE000A01344C
:1018E00049F094F90A2C05F11005F4D102A928A8B1
:1018F00049F040F903A983462CA849F03BF904A913
:10190000824630A849F036F905A9814640A849F039
:1019100031F906A9804634A849F02CF907A90746F1
:1019200038A849F027F908A906463CA849F022F949
:1019300018A9054644A849F01DF90446BBF1000F5B
:1019400008D1BAF1000F05D1B9F1000F02D1B8F1F9
:10195000000F0ED01A4800220DF1070148F090FE4A
:1019600038B149F0A5F820B99FED160A14484AF09D
:101970003BFA27B91EB915B9002C3FF41EAF134826
:1019800000220DF1070148F07BFE00283FF415AF5F
:1019900049F08EF800287FF410AF9FED0A0A0B483B
:1019A0008BE700BF5CBC0C08ACBC0C085CBD0C0831
:1019B000CDCCCC3DDCBD0C08EB0B0D081CBE0C08DF
:1019C0006D040D0800000000BCBC0C08E00B0D0805
:1019D0000F299DBF302303FB0100503000207047CA
:1019E000014B93F94F027047384C0020024B587F4F
:1019F00000F00100704700BF385C0020044BB3F8D2
:101A00001432DB075ABF0069C0F340100020704752
:101A1000384C0020014BD3F8F80B7047384C0020AD
:101A200008B503689B68984730B9044B93F91C00CC
:101A3000B0FA80F0400908BD0020FCE7385C0020C7
:101A400038B50D1E2DDB174C94F8042CEBB29A42DE
:101A500027D3D4F8003C0122595DA4F5005003F0CF
:101A600063FBF0B15DF02EFA03215EF02FFAC0B9EE
:101A70005DF028FA0D215EF029FA90B994F934321C
:101A8000EB40DB075CBF94F94E12E940A4F500502F
:101A900048BF0221BDE8384058BF01F00101FCF702
:101AA00091BB38BD384C0020022A10B50C4605D138
:101AB000BDE810400848352203F036BB074B586894
:101AC00003681B689847A04205D15DF0FBF9BDE8AB
:101AD00010405DF081B910BD382C0020385C00202A
:101AE00029B1022907D1044BC3F8FC1F7047024BF0
:101AF0000122C3F8FC2F7047384C002029B102297D
:101B000005D1034B01221A707047014B19707047C1
:101B1000385C002010B500F50053DFED186AD3F8EB
:101B2000F02BD3F8EC3BB2F90820B3F908309FED65
:101B3000147A07EE902AF8EEE77A0446C7EEA60A72
:101B400000F58F500121183007EE903AF8EEE77A51
:101B500060EE870A87EEA60A20EE070A10F004FE60
:101B600052F0B2FB262152F0EBFA04F53750054A49
:101B7000BDE810400621103054F0C6BD0000C84238
:101B800035FA8E3C68170D0800F58042002382F874
:101B9000503C044A00F5375013720621024A1030B7
:101BA00054F0B2BD0D88002074170D08F8B500F58B
:101BB0008045044695F8501C002953D02A4B2B4AE7
:101BC0005868904203D19B6A93F8CB3023B92046E2
:101BD000BDE8F840FFF7D8BF254E95F8517C04F5D5
:101BE0000053012093F9F82F3072C7BB002A39DB6C
:101BF00085F8510C0139C9B285F8501CD3F8F02B87
:101C0000D3F8EC3BB2F90820DFED1A6AB3F90830DB
:101C10009FED197A07EE902AF8EEE77AB1FA81F192
:101C2000C7EEA60A04F58F504909183007EE903A1E
:101C3000F8EEE77A60EE870A87EEA60A20EE070A3A
:101C400010F092FD95F8503C63B904F537503372AB
:101C50000A4ABDE8F8400621103054F055BD002A6C
:101C6000C8DAB4E7F8BD00BF385C00203484002037
:101C70000D88002000007A4535FA8E3C88170D0843
:101C80006D2900F3E380012901DC5DF063BF8B1E49
:101C90006B2BFAD80FF2040C5CF823F0AB1E010892
:101CA000A51E0108AB1E0108AB1E01088B1C010814
:101CB000AB1E01088B1C01088B1C0108A51E010826
:101CC0008B1C0108AB1E0108A51E0108A51E0108FA
:101CD0008B1C0108AB1E0108AB1E0108AB1E0108DE
:101CE0008B1C01088B1C0108A51E0108AB1E0108F6
:101CF000A51E01088B1C0108A51E0108A51E0108D0
:101D00008B1C01088B1C01088B1C01088B1C010813
:101D10008B1C0108A51E0108AB1E01088B1C0108C5
:101D20008B1C01088B1C0108AB1E01088B1C0108D1
:101D3000A51E01088B1C01088B1C0108AB1E0108A5
:101D4000A51E01088B1C01088B1C01088B1C0108B7
:101D5000AB1E0108AB1E0108AB1E01088B1C01085D
:101D60008B1C0108AB1E01088B1C01088B1C010891
:101D7000AB1E0108AB1E0108AB1E01088B1C01083D
:101D80008B1C0108AB1E0108AB1E01088B1C01084F
:101D90008B1C01088B1C01088B1C01088B1C010883
:101DA0008B1C0108AB1E0108AB1E0108AB1E01080D
:101DB000AB1E0108AB1E0108AB1E01088B1C0108FD
:101DC000A51E0108A51E01088B1C01088B1C01081B
:101DD0008B1C01088B1C01088B1C01088B1C010843
:101DE000AB1E0108A51E01088B1C01088B1C0108F5
:101DF0008B1C01088B1C01088B1C01088B1C010823
:101E00008B1C01088B1C01088B1C01088B1C010812
:101E10008B1C01088B1C01088B1C01088B1C010802
:101E2000AB1E01088B1C01088B1C01088B1C0108D0
:101E30008B1C01088B1C01088B1C01088B1C0108E2
:101E40008B1C01088B1C0108A51E0108A12921DC9F
:101E500096297FF71AAFA1F197030A2B3FF615AF2A
:101E60000FF2040C5CF823F0AB1E0108AB1E010856
:101E70008B1C0108AB1E01088B1C01088B1C010880
:101E80008B1C01088B1C0108A51E0108A51E01085A
:101E9000AB1E0108B42908D0DB2903D0B2297FF496
:101EA000F4AE704700235DF027BE704770B563291C
:101EB0008AB000F3D180012904DC0AB0BDE870408B
:101EC0005DF0A6BB8B1E612BF7D801A454F823F05C
:101ED000D1200108E5200108052101080D21010894
:101EE000BB1E01083F210108BB1E0108BB1E0108E3
:101EF000ED210108BB1E0108BB1E0108F3200108EB
:101F000013220108BB1E0108E92101084D22010826
:101F10005B220108BB1E0108BB1E01086B220108E1
:101F20007922010887220108BB1E0108A9220108A5
:101F3000BB220108BB1E0108BB1E0108BB1E010815
:101F4000BB1E0108BB1E0108CD220108BB1E0108F3
:101F5000BB1E0108BB1E0108BB1E01081F23010890
:101F6000BB1E0108BB1E0108BB1E0108BB1E0108E9
:101F70002323010827230108BB1E0108BB1E0108FB
:101F8000BB1E0108BB1E0108BB1E0108BB1E0108C9
:101F9000BB1E0108BB1E0108B3230108BB1E0108BC
:101FA000BB1E01085F2201086322010867220108A5
:101FB000BB1E0108BB1E0108BB1E0108BB1E010899
:101FC000BB1E0108BB1E0108BB1E0108BB1E010889
:101FD000BB1E0108BB1E0108A7230108AB23010893
:101FE000AF230108B7230108BB230108BF23010861
:101FF000BB1E010801240108C3230108BB1E010800
:10200000BB1E0108BB1E0108BB1E0108BB1E010848
:10201000BB1E0108BB1E010831240108BB1E0108BC
:10202000BB1E0108BB1E0108BB1E0108BB1E010828
:10203000BB1E0108BB1E0108BB1E0108BB1E010818
:10204000BB1E0108BB1E0108BB1E0108BB1E010808
:10205000BB1E010841240108A1291FDC97297FF735
:102060002CAFA1F19803092B3FF627AF01A454F838
:1020700023F000BF45240108BB1E010859240108B4
:10208000BB1E0108BB1E0108BB1E0108BB1E0108C8
:1020900039240108BB1E0108F3220108B42900F00D
:1020A000D780DB2916D0B2297FF407AF002A00F0D1
:1020B000B881022A0ED1A74B58680368DB6F984796
:1020C00040B95BF0F5F9A44A042154F01DFB01E08E
:1020D000022A01D001242FE035220E219F4803F06F
:1020E00023F8F7E7111E18BF01219C48FCF76AF896
:1020F000F0E7012A04D0022A14BF00210221F4E7EC
:102100001146F2E70621FFF7CFFCE3E7022AE1D10F
:10211000904D68680368DB6A984704460028D9D068
:10212000A5F58053D3F8F43BB3F90830002BD1D197
:10213000A5F54050FFF7EEFC20460AB070BD022A1C
:10214000C8D1844E864A71689142C3D0B26A92F86F
:10215000CB20002ABED006F58054A6F58056B4F9EF
:102160003C2F2AB9D6F8F43BB3F90830002BB1D094
:102170001C22002103A805ADB5F046FB284615F04A
:102180003DFAB4F93C3F93B91623ADF80E30D4F8BC
:102190000C3C7448642BB8BF642303A906932BF04E
:1021A000BFF920B152F090F8272151F0C9FF04F691
:1021B000084494E80F0085E80F00D6F8F43B69481E
:1021C000B3F90830002BCCBF1023152303A9ADF8B9
:1021D0000E302BF0A5F900283FF47CAF52F074F8D4
:1021E000272151F0ADFF75E703218CE7022A5E4DF0
:1021F00003D0002385F8083C6CE71921A5F596501B
:102200004AF08CFC04460028F3D0012385F8083CF2
:1022100092E7012A0BD0022A11D0002A7FF45AAF8C
:10222000514B83F8782252F04FF82B21D9E74E4BCF
:10223000019283F8782252F047F82C21D1E74A4BDB
:1022400083F8782252F040F82D21CAE70F215AE78F
:10225000464811468BF0E0F83CE7092153E704219A
:1022600051E705214FE717214DE7901E41424141BB
:102270003F4864F0B9F82DE7022A7FF42BAF3748C6
:1022800000F0DAFF26E7012A06D0022A07D0002A4A
:102290007FF420AF1146EBE711460192E8E734489E
:1022A000012164F0A1F8EAE7324B023AD3F8343C5A
:1022B0005442544183F820400CE7931E594259413F
:1022C0002C4BD3F8340C7DF03DFE03E7214B996A8B
:1022D00091F8F51001293FF4FDAE541E012C13F8BE
:1022E000062C8CBF0024012464F3041203F8062C8E
:1022F000F0E65AB1022A7FF4EDAE164B9A6A92F8D4
:10230000A13143F0020382F8A131E3E6114B9B6A4D
:1023100093F8A11162F3410183F8A111DAE61221C9
:10232000F1E61521EFE6002A34D0022A7FF4D2AE7E
:10233000084D686803681B6C98470446E0B105F5D2
:1023400080550121D5F8340C0368D3F8A0309847A4
:10235000F2E600BF385C0020EC170D08382C002096
:10236000047B0020407B0020384C0020187D00209A
:10237000E0790020386C00205BF09AF80446686829
:1023800003685B6C98473D4A03460421204654F09D
:10239000BBF99FE63A4BD3F8340C03681146D3F8E7
:1023A000A030984796E60021ADE61021ABE6022169
:1023B000A9E60121A7E61621A5E60721A3E60B2140
:1023C000A1E6022A2E4B0ED1012483F82C4E51F0A7
:1023D0007BFF4A2151F0B4FE5BF06AF8294A0621DE
:1023E00054F092F9A8E6002283F82C2E51F06CFFED
:1023F0004B2151F0A5FE5BF05BF8234A062164E611
:10240000012A09D0022A0AD0002A7FF463AE0121F2
:102410001E480DF067F85DE601920021F8E71146CD
:10242000F6E71B4B58680368D3F88030984751E6AD
:102430001146FFF755FB4DE61146FFF75FFB49E6F6
:102440001B2160E6022A7FF445AE1248FCF73CFCF3
:102450005BF02EF8104AD1E711465CF0FBFF0F4805
:102460007AF028FB044600283FF434AE0C4A92F878
:10247000FB3F43F0020382F8FB3F5DE6A0170D0827
:10248000386C0020C9170D08DA170D08D058002045
:10249000385C0020382C002005180D084859002011
:1024A000384C002010B50446044883F01FF804F1AE
:1024B0000801BDE8104027F061BE00BF5078002041
:1024C00038B504462DED028B114883F015F805460A
:1024D00029F0BEFD0F48B0EE408A0DF0D5F890B15E
:1024E000DFED0D7AB4EEE78AF1EE10FA0BDDD5EDF3
:1024F000000A95ED010AB2F0F7FEDFED087A20EE52
:10250000270A84ED080ABDEC028B94ED080A38BD59
:1025100050780020382C002000401C46E02E6542F8
:10252000074B93F93502022805D0032806D000385E
:1025300018BF0120704781F00100704704207047E8
:10254000384C002003688B4214D00429C0E90013E2
:1025500002D007290CD07047074B9FED087AD3EDC6
:10256000FE7AF8EEE77A67EE877AC0ED087A704770
:1025700000238362704700BF383C00200AD7233C09
:1025800008B50246FFF7CCFFBDE8084001461046FB
:10259000FFF7D8BF70B52DED048B0446F0EE408AEE
:1025A000B0EE608A0D4616468CF068FB9FED319ABE
:1025B000DFED319AE06166B3236833B92F4BD3ED79
:1025C000FE7AF8EEE77AC4ED097A68EE898A002D82
:1025D000B7EE000AFFEE007AB8BFB0EE670A68EE09
:1025E000808AC4ED058A264BB4EEE98AF1EE10FA32
:1025F000D3F8340C30DA7CF083FC20EE090A84ED49
:10260000060ABDEC048B20460321BDE87040FFF7AD
:1026100099BF94ED090A98EE890A26F001FD002D74
:1026200084ED050A0BDAB4EEE90AF1EE10FADADB12
:10263000DFED147A30EE670A84ED050AD3E7D2D0D5
:10264000DFED117AB4EEE70AF1EE10FACBD8DFED48
:102650000D7A30EE270AEFE77CF052FCB4EE480A20
:10266000F1EE10FA48BFB0EE408A28EE098A84EDF8
:10267000068AC6E70000C84200000034383C00204B
:10268000386C002000A00C47000000B410B52DED00
:10269000028B0446B0EE608AF0EE408A8CF0EEFACF
:1026A000DFED090AE06168EEA08A68EE200AC4ED59
:1026B000098ABDEC028BC4ED0A0A20460621BDE85A
:1026C0001040FFF73FBF00BF0000C84210B52DED1E
:1026D000028B0446B0EE408A8CF0D0FA94ED090AE1
:1026E000DFED097AE061A8EE270A26F083FCBDEC55
:1026F000028B002384ED090AA36220460621BDE86F
:102700001040FFF71FBF00BF0000C84270B54B6804
:10271000154D06460C4673B98B6863B9C96851B943
:102720001248FFF72DFF95F84D1D05F6D440BDE882
:1027300070405FF0B9B995F84D1D0D485FF054F841
:1027400048B906F10801204615F0E8F818B1074825
:102750000221FFF7F7FE95F84D1D05482246BDE81A
:1027600070405FF095B900BF386C00203C860020B7
:102770000C79002008B50721FFF7E4FE80ED0A0A76
:1027800008BD000008B50368032B21D1D0ED057A00
:102790009FED117AF0EEE77AF4EEC77AF1EE10FAD7
:1027A00018D50E4B90ED090AD3EDFE7AF8EEE77AD4
:1027B00037EEC00A26F034FCDFED097AB0EEC00A2D
:1027C000B4EEE70AF1EE10FA94BF0120002008BD34
:1027D0000120FCE70020FAE700000034383C00202C
:1027E0000000484330B50368023B85B00446082B1F
:1027F0006DD8DFE803F0050D30374B613F616100B4
:10280000FFF750FE84ED090A94ED090A05B030BDCA
:102810008CF034FAE369DFED310AE061C31A07EEA8
:10282000903AF8EE677A94ED050A67EEA07AD4ED57
:10283000060AF12020EEA71A67EEE00A26F046FC11
:10284000D4ED057A77EEC07AC4ED057AD4ED097A35
:1028500037EE800AD6E7FFF733FEDFED217A20EE70
:10286000270ACFE71F4BD3ED147AF8EEE77AC0EDD5
:10287000097AC9E71C4DD5F8480C80F0D1FF002833
:10288000C2D0D5F8483C1B6B6362BDE78CF0F6F90B
:10289000E3699FED127AD4ED0A6AE061C31A07EE8C
:1028A000903AF8EE677A67EE877A94ED097AA6EEA9
:1028B000A77A84ED097AA7E70B4B9FED0C0AD3F8B2
:1028C000340C6C3029F082FE84ED091A9CE7064B2B
:1028D000D3F83C3CD3F84433D6E700BF6F12833AB9
:1028E0000000C842385C0020386C00209F0CB345C3
:1028F0000368092B08D8DFE803F0050A050505057C
:10290000070705100023836290ED0A0A7047044B05
:10291000D3F83C3CD3F84833F5E7C36AF3E700BF8C
:10292000386C0020F8B50023204FCB627B7F204E0F
:1029300013F0010F04460D462BD1786803689B6F96
:10294000984730B3786802F0D7FFDFED1A7A85ED4B
:102950000B0AB0EEC00AB4EEE70AF1EE10FA03D4A7
:1029600009213046FFF7EEFD1148FFF73BFF104805
:1029700084ED000AFFF7BCFF336884ED010A0A2BDF
:102980000FD8DFE803F00C1010101010100C100C12
:102990000C003368092BE7D105480021E2E7022348
:1029A000A3602046F8BD0123FAE700BF385C002091
:1029B0003C86002000000034034B01221A600022F4
:1029C0009A60DA601A6170473C86002013B501A94D
:1029D00004460CF0CFFC04F5804320B9012283F8B3
:1029E0007D2D02B010BDDDED017ADFED096A03F542
:1029F0005762B8EEE77AD2ED007A67EEA67AB4EEC7
:102A0000E77AF1EE10FA54BF01220022E7E700BF97
:102A10000000C8422DE9F04F2DED068B00F5005B5C
:102A200000F58F589BF98A328DB0054600F5804439
:102A300008F1180833B100F5405ADAF8283093F855
:102A4000CB707FB90021A4F8201E404610F07CF81E
:102A500094F8211E40460DB0BDEC068BBDE8F04F4A
:102A600010F07CB88CF00AF90190D4F83C0C9FED82
:102A7000958A90EDDBAA7EF0DBFE09AE002800F01F
:102A8000CC80D4F83C3C03F55C7393E8070086E8FF
:102A9000070030468DED0B8A2AF096F9B0EE409A89
:102AA00028460CF0F1FD05F5984909F118090028B0
:102AB00000F0B680484682F01FFD07C886E8070090
:102AC00030468DED0B8A2AF07FF9F0EE409ADAF865
:102AD000040003681B689847122840F0AA8000236E
:102AE00084F8203EDAF8040003685B69984728B14F
:102AF000DBF8F43BB3F90830002B0DDC9BF9F83F11
:102B0000002B09DA019BC4F8243E484682F0F0FC11
:102B100004F6286383ED000A94F8203E5BB1019B24
:102B2000D4F8240E181A41F28833984240F28F806C
:102B3000002384F8203ED4F8340C9FED630A6C30F7
:102B400029F044FD8DED090ACDED0A0A8DED0B1A31
:102B500096E8070006AB03AE9FED5C0A83E807002A
:102B600086E80700304629F031FD2846B0EE408A5D
:102B7000F0EE608A8DED060ACDED070A8DED081A9C
:102B80000CF082FD002874D0DFED517AF4EEE79A64
:102B9000F1EE10FA94BF01250025D4F83C0C7EF02C
:102BA00047FE30B1DFED4A7AB4EEE79AF1EE10FA63
:102BB00009D9002D64D1DAF8040003681B6898472E
:102BC000022864D00027D4F83C0C7EF053FF054661
:102BD000002873D0B5EEC0AAF1EE10FA6DD5DFED86
:102BE0003D7AB4EEE7AAF1EE10FAACBF012600265A
:102BF000484682F089FC5EB9DFED377AB0EEC00A54
:102C0000B4EEE70AF1EE10FA5AD8002D08BF0027FB
:102C100094F8201E84F8217E17E7B0EE489A3FE72B
:102C200028460CF001FD00287FF444AFDFED259A23
:102C30004DE7DAF8283093F8CB30002B3FF452AF51
:102C40009BF9F83F002BBFF64DAF012348E74846FC
:102C500082F04EFC04F62863D3ED007A30EE670A6A
:102C6000DFED1E7AB4EEE70AF1EE10FA3FF760AF3F
:102C700061E728460CF0D8FC0546002884D18CE793
:102C8000D4F83C0C7EF0D4FD002894D19BE7B0EE44
:102C9000680AB2F007F9F0EE408AB0EE480AB2F0E6
:102CA00001F9DFED0F7A20EE280AB4EEE70AF1EE23
:102CB00010FACCBF0127002785E700252E4697E7AD
:102CC0003746A5E7000000009F0CB345D302373913
:102CD0000000FA420000C8C20000704200004842F2
:102CE00055CF7D3F38B504460CF0CEFC04F58F552A
:102CF000183548B920460CF097FC014620B9284603
:102D0000BDE838400FF080B904F5405460680368AE
:102D1000DB6C984718B9606803681B6D98470146DB
:102D2000EDE7000030B5044689B0684604F58F55DC
:102D300014F064FC183504A814F060FC69462846B9
:102D40000FF01CFA98B104A928460FF067FA70B189
:102D5000059B019323680022DB6C69462046984757
:102D600028B104F5275001213C3086F01DFA09B046
:102D700030BD000000F5805292F87424D2070AD4C6
:102D800000F54052926A92F8CB1009B1FFF7CABF22
:102D900003689B6C1847704730B587B0044602A89B
:102DA000019114F02BFC04F58F5002A918300FF09C
:102DB000E5F9019A18B90025284607B030BD236807
:102DC00002A9DB6C2046984705460028F3D004F59D
:102DD000275001213C3086F0E7F9EDE7F0B50446D5
:102DE00085B004F58F56684618360F46154614F020
:102DF00005FC694630460FF011FA10B9002005B005
:102E0000F0BD394630460FF071F80028F6D0002D9D
:102E1000F5D004F58054284694F8743443F0020346
:102E200084F87434EBE7000003207047F0B5524F8C
:102E3000D7F8B83BDA0785B0044600F19A8000F570
:102E40004055AB6A93F8C120002A40F0928093F875
:102E5000CB30002B00F08A8000F5005393F9F83F47
:102E6000002BC0F2838000F5804696F82C3E002BA4
:102E70007FD1D6F8340C9FED410A6C3029F0A6FBC7
:102E8000CDED020A60EEA00ADFED3D7A8DED010A7C
:102E9000E0EE000A8DED031AF4EEE70AF1EE10FA07
:102EA00064DCD6F8343C9FED377AD3ED377AF4EE14
:102EB000C77AF1EE10FA03D5AB6A1B7A002B55D016
:102EC000B5EE007AF4EEC77AF1EE10FA4ED404F5BE
:102ED0009840183082F018FBDFED2B7AB4EEE70A49
:102EE000F1EE10FA42D8D6F8343C9FED287AD3EDB3
:102EF000367A67EE877AB3EE0E7AF4EEC77AF1EEA1
:102F000010FA33DA224AB4F9A410138801339BB2C1
:102F1000138019B9B4F8A210A4F8A410B4F8A4103E
:102F2000994226D80026168051F0CEF901221921A7
:102F300051F026F9A86A03685B699847431C04F5B9
:102F40003750144A3146103053F0DEFBAB6A012291
:102F500083F8C120D7F8B83B5B070AD504F5855044
:102F6000083005B0BDE8F04067F098B9084B002282
:102F70001A8005B0F0BD00BF384C00209F0CB3454F
:102F80004054094A6666663F000000B4E02E654280
:102F900076860020F0190D0870B52DED028B4A4B96
:102FA000D3F8B83B9B0784B004461ED400F5804597
:102FB000DFED468AD5F8340C03681B699847D0EDDD
:102FC000017AF4EEE87AF1EE10FA0EDB04F54053E4
:102FD00004F59C469B6A93F8C12030364AB1002321
:102FE00003A93046039352F0A5FD04B0BDEC028B5B
:102FF00070BD93F8CB30002BF1D004F5005393F95A
:10300000F83F002BEBDB95F82C3E002BE7D1D5F8F1
:10301000340C03681B699847D0F8A430D5F8340CF9
:10302000039303681B69984704F58C7200F1A401AF
:10303000304652F087FEDDED037AB0EEC08AF0EE46
:10304000E77AF4EEC87AF1EE10FA03D503A9304618
:1030500052F070FDD5F8340C03681B699847D0ED29
:10306000040AF4EEE80AF1EE10FABEDBF6EE087A96
:1030700060EEA77AF4EEC87AF1EE10FA1DD58BF067
:10308000FDFDD5F83C3E42F21072C31A9342ACD912
:10309000DFED0F7AC5F83C0E68EE277A04F5375459
:1030A00017EE900AF9F730FA1034CDE90001094A19
:1030B0000021204653F028FB97E79DED030A25F0F9
:1030C00001FF0028DBD190E7384C002000000034DD
:1030D0000000C8420C1A0D0810B5044600F59B40CC
:1030E000283063F093F904F59B400121BDE81040BE
:1030F00048306BF099BA0000F8B500F580450446F9
:1031000095F9A83D53B300F5005695F8BC2D96F8F7
:10311000F83FDB43C3F3C01363F3C30200F59B47DF
:1031200000F5984085F8BC2D183082F0EDF9DFED00
:103130003E7A283720EE670A384663F0E7F995F8BB
:103140002C3E5BB9384663F08DF904F540539A6A1A
:1031500092F8CB201AB9354B00221A80F8BD95F8A9
:10316000BC2DD207FAD4586803689B6B9847002897
:10317000F1D096F9F83F002BEDDB2C4E33884BB99C
:10318000B5F9AE3D33B1642213FB02F3D5F80C2C34
:103190009A42E3DB384663F0D5F9D5F8343C9FED2D
:1031A000247AD3ED367A67EE877AB3EE0E7AF4EEB0
:1031B000C77AF1EE10FA05D83388002BCED0013B48
:1031C0003380CBE7B4F9A4301BB9B4F8A230A4F82B
:1031D000A4303388B4F8A420B4F9A400154993426C
:1031E0003CBF013333803388D5F8E42B012B01D168
:1031F0000A60B3E709689142ADDD18B9B4F8A220BE
:10320000A4F8A420B4F8A4209A42A7D800233380BD
:1032100051F05AF802220C2150F0B2FF2046BDE8CE
:10322000F840FFF759BF00BF0AD7233C748600203F
:10323000E02E65427086002008B500F5804292F9C4
:10324000A83D6BB300F5005393F9F83F002B0EDA5D
:1032500000F53750134A0621103053F055FA51F05B
:1032600033F80322BDE808400F2150F089BFB2F9BE
:10327000AE3D8BB1D2F80C2C642113FB01F39A42C2
:103280000ADA00F53750084A0121103053F03CFAB1
:1032900051F01AF80222E5E7BDE80840FFF71CBF2D
:1032A00008BD00BF241A0D08361A0D08F0B52DED23
:1032B000028B00F54056584DB36A93F8CB308DB071
:1032C000044643B100F5005393F9F82F002A02DBBE
:1032D00093F95E322BB900232B800DB0BDEC028B2D
:1032E000F0BD00F5804797F82C3E002BF3D101F09C
:1032F00013FB002878D1706803689B6B98470028FF
:10330000E9D004F59740683052F074FC29F05CFD78
:10331000F0EE087AB4EEE70AF1EE10FAF0EE408A29
:10332000D9DA04F5A252D2ED017A92ED000A20EE2C
:10333000270AB1F071FFDFED397A20EE270AB2EEED
:103340000E7AB4EEC70AF1EE10FAC4D9D7F8343CBD
:1033500093ED368A28EE278AF3EE0E7AB4EEE78AEA
:10336000F1EE10FAB7D904F58F50002309A91830EF
:1033700009930A930B930EF05DFF00283BD12B8835
:10338000B4F9A42001339BB22B80002A3ED0B4F8BC
:10339000A420B3EB420FA0DB50F096FF01220C21DA
:1033A00050F0EEFE1E4B002218EE900ACDE90623E7
:1033B000F9F7AAF81B4BCDE90401002218EE100A18
:1033C000CDE90223F9F7A0F804F537541034CDE91C
:1033D0000001154A2046002153F096F901220C21E4
:1033E0001248FAF7DFFD78E7706803681B6D9847AD
:1033F000002880D16FE709A829F0E6FCF2EE047AF4
:10340000B4EEE70AF1EE10FAB9DB64E7B4F8A220F3
:10341000A4F8A420BBE700BF6C860020E02E654224
:103420000000084000003E404C1A0D08485900209A
:10343000F0B52DED028B8BB0002307930893099311
:1034400005AB0446019300F58F5007AB009302AA29
:1034500004AB03A918300EF005FE04F5005605462E
:1034600086F8C40D28B9002528460BB0BDEC028BA8
:10347000F0BD8BF0F7FBD6F8C83D9FED327AC31A4A
:1034800007EE903AF8EE677A074667EE877A04F51A
:10349000365006AA02A92030CDED067A52F052FC31
:1034A00004F5365006AA03A92C308DED020A52F01D
:1034B00049FC04F5365006AA04A938308DED030AFC
:1034C00052F040FC96ED988AC6F8C87DB5EEC08AE9
:1034D000F1EE10FAC7D9DDED080A9DED070AB1F04B
:1034E00067FDDDED090AB1F063FDD6F8482DDDED8D
:1034F000037AB4EEC08AF1EE10FA94BF01230023E0
:103500001AB196F84C2DD20712D438EE087AB4EEE0
:10351000E77AF1EE10FA0BD80233DBB2DDED027A76
:10352000B4EEE78AF1EE10FA09D8002B9BD09BE7A6
:10353000B4EEE78AF1EE10FAF0D80133EDE7012B93
:1035400092D890E7BD37863570B500F540550446F2
:103550006B7F43F004036B7750F0B6FE012211211C
:1035600050F00EFEAB6A93F8CB30002B3FD068686A
:1035700003681B68984709280AD1204608F0C2FB57
:1035800030B104F5AC405830BDE8704008F0A2BB43
:10359000174B586803681B69984704F5005340B9F6
:1035A00093F95D32032B22D10621204608F096FBC9
:1035B0000CE093F95D120229F6D16B7FDB07F3D49F
:1035C0000622204601F0B0FD0028EDD0094B6868C6
:1035D00001225A7303685B6C9847034604F5375021
:1035E000054ABDE870400221103053F08DB870BD1F
:1035F000385C00200D880020801A0D0808B500F501
:103600004052537F590716D56FF3820353770A4B05
:103610005A7B42B1002200F537505A730221074A03
:10362000103053F071F850F04FFEBDE80840002212
:10363000112150F0A5BD08BD0D880020A41A0D0869
:10364000F0B5054685B005F58F576846183713F075
:10365000D5FF694638460EF0E1FD80B105F500530F
:10366000D3ED987A374CF5EEC07AF1EE10FA08D81F
:10367000354A002328462380D373FFF7BFFF05B0E8
:10368000F0BD2846FFF7D4FE064628460BF0CCFFD7
:1036900010B928460BF0A4FFA378002E18BF002015
:1036A0000343DBB2A370002BE9D06378A8BB83BBD4
:1036B00023780133DBB2082B237003D14EB3384695
:1036C0000EF03CFD2378092B02D138460EF02EFD7A
:1036D0002378092B1DD94FF48573238050F0F4FD16
:1036E0000222102150F04CFD8BF0C8FA6368C01A1A
:1036F00047F23053984209D905F53750134A022151
:10370000103053F001F88BF0B9FA60602846FFF7EB
:103710001BFF0D4B6278DA73B1E72678002EF8D0E4
:10372000013EF6B22670002BF3D0002EF1D1667068
:1037300050F0CAFD3246102150F022FD2846FFF716
:103740005DFFE6E7788600200D880020BC1A0D0892
:1037500000F540535B7F5B0701D5FFF7F5BE70476F
:1037600073B5044600F58F5001A9183004F50055D3
:103770000EF0C2FAD5F88C3D834206460CD004F513
:103780008043D3F8340C7CF023FEC5F88C6D50F0E8
:103790009BFD3E2150F0D4FC04F5805695F9901D18
:1037A00096F9082596F8083591421BD0FF2B19D0C1
:1037B00004F58043D3F8340C7CF00AFE96F8083503
:1037C00085F8903D50F080FD95F8902D182150F02F
:1037D000D7FC04F5375095F9903D034A0421103089
:1037E00052F092FF02B070BDCC1A0D082DE9F043E3
:1037F0008FB005468BF042FA00230593069307939A
:10380000089309930A930B930C930D9305F58F5826
:1038100004AB019308F1180803AB009306460BAB09
:1038200008AA05A940460EF0FDFBDFED477A9DEDA5
:10383000077AB4EEE77AF1EE10FA074630DB9DED39
:103840000A7AB4EEE77AF1EE10FAACBF0124002454
:1038500005F50059404699F8C43D002B08BF0027E4
:103860000EF0F2FB8046EFB9444699F9543B012B28
:1038700029D164B105F540539A6A92F8CB4034B12E
:10388000586803685B69984780F00100C4B299F8F2
:10389000943DCBBBCCB9C9F8986D0FB0BDE8F083AF
:1038A0000024D5E7002CDFD005F536502C3052F03F
:1038B0003FF990ED007AF7EE007AB4EEE77AF1EE98
:1038C00010FAD2DCD0E70024E1E7D9F8980D301ADD
:1038D000B0F57A7FE1D9C9F89C3D012405F5804314
:1038E00089F8944DD3F83C3C83F80C4450F0ECFC40
:1038F00022461D2150F044FC144A05F537500221A0
:10390000103052F001FFC8E714B1C9F89C6DC4E74C
:10391000D9F89C0D43F69823361A9E42BDD905F579
:103920008043C9F8984D89F8944DD3F83C3C83F80E
:103930000C44C9F89C4D50F0C7FC22461D2150F0A4
:103940001FFC034AD9E700BF00000034E41A0D0849
:10395000FE1A0D087047000000F537500B46024A6A
:103960000421103052F0D0BE1C1B0D0810B50446C7
:1039700050F0AAFC0022052150F002FC04F537505B
:10398000034ABDE810400421103052F0BDBE00BF14
:10399000281B0D0813B50B464AB100F537500092AD
:1039A0000421054A103052F0AFFE02B010BD02B043
:1039B000BDE81040FFF7D0BF401B0D0808B500F56B
:1039C0003750064A0421103052F09EFE50F07CFC25
:1039D000BDE808400022082150F0D2BB541B0D085E
:1039E00038B504460D468BF049F904F5405325B926
:1039F0005A69986102B9586138BD9A69801A642879
:103A000084BF0022C3E90522F6E7000037B504466B
:103A100000F59840183081F05DFD04F50052C0F3C8
:103A2000803592F8FA3FC3F34001A9421DD065F3F7
:103A3000410304F5375482F8FA3F10346DB150F069
:103A400043FC02220B2150F09BFB094A0221204635
:103A500003B0BDE8304052F057BE50F035FC2A4666
:103A60000B2150F08DFB034AF0E703B030BD00BFDF
:103A70006C1B0D08881B0D0838B50A460C4606213C
:103A8000054601F051FB28B1054A137843F00803BD
:103A9000137038BD21462846BDE8384008F01EB9ED
:103AA0002C88002038B50A460D461521044601F041
:103AB0003BFB28B1094A137843F00803137038BD63
:103AC00004F5375004211030054A52F01DFE2946F6
:103AD0002046BDE8384008F001B900BF2C8800201E
:103AE000981B0D0838B50A460D461521044601F00D
:103AF0001BFB28B1094A137843F00803137038BD43
:103B000004F5375004211030054A52F0FDFD2946D6
:103B10002046BDE83840FFF7AFBF00BF2C8800202B
:103B2000C01B0D0838B50A460D461B21044601F09E
:103B3000FBFA28B1094A137843F00803137038BD23
:103B400004F5375004211030054A52F0DDFD2946B6
:103B50002046BDE83840FFF78FBF00BF2C8800200B
:103B6000D61B0D0838B5044600F537500D46103009
:103B70000421044A52F0C8FD29462046BDE83840D9
:103B800008F0ACB8E81B0D0810B500F5005494F827
:103B9000FA3F9A0624D400F54050406803681B6839
:103BA0009847032808D005D802280ED194F8F80FBA
:103BB000C00914E01B28F9D194F8F80F00F0A00018
:103BC000A0F180035842584109E0B4F8F80F20F4FE
:103BD000FE4020F07F0080B2003818BF012010BDE9
:103BE0000120FCE738B500F5405504466B7F184AC4
:103BF00043F0080300F537506B770221103052F084
:103C000083FD50F061FB0122172150F0B9FA2046E4
:103C1000FFF7BAFF40B104F534500122BDE8384047
:103C200015211030FAF7BEB9686803681B68984719
:103C3000062806D104F5AE407030BDE8384009F0E2
:103C400057BA20460B21BDE83840FFF715BF00BF2B
:103C5000FC1B0D0870B500F54055D5E905239B1AEE
:103C600041F28832934206460FD9686803685B6D5B
:103C7000984704466B7FC3F3C003A34211D034B10D
:103C80003046BDE87040FFF7ADBF0024F2E750F0CA
:103C90001BFB2246172150F073FA6B7F64F3C303BA
:103CA0006B7770BD0B4610B511460446072B07D83D
:103CB000DFE803F02A041316191C242708F00EF875
:103CC00004F50053D3F8583B9B061DD504F58550E9
:103CD0000830BDE8104066F0E1BAFFF7CDFEEFE72F
:103CE000FFF700FFECE7FFF7DDFEE9E700F53450F2
:103CF000012214211030FAF755F9E1E7FFF712FF1E
:103D0000DEE7FFF72FFFDBE710BD0000F8B5044644
:103D100004F5005750F0D8FA0122052150F030FA8E
:103D200097F84232072B98BF2E4A204694BFD55CA5
:103D30000125FFF729FF68B12B4A2C492046FFF7E0
:103D400029FE102104F5345001220844FAF72AF91B
:103D5000002513E004F54056706803681B6D984712
:103D600098B196F8C53583B196F9C435012B0CDCB2
:103D70001F4A20492046FFF70DFE0125294620460F
:103D80000322BDE8F840FFF78DBF706803681B6D24
:103D9000984718B1D7F8583B190713D470680368CF
:103DA0001B689847032803D1D7F8583BDA070CD48F
:103DB000706803685B6A984768B90C492046FFF74A
:103DC000CBFDDBE70A4A0949D4E70B4A07492046FD
:103DD000FFF7E0FDBCE7D7F8583B5B07EDD5074A96
:103DE000F4E700BFDC1C0D081C1C0D08E2F00D08F8
:103DF000261C0D08391C0D08491C0D08591C0D08FE
:103E000038B50446154650F05FFA0122062150F0FD
:103E1000B7F92046FFF7B8FE98B104F534500122F7
:103E200007211030FAF7BEF8134A14492046FFF76D
:103E3000B1FD0025294620460422BDE83840FFF7A1
:103E400031BF04F54053EDB2586803681B6D9847C5
:103E500068B104F50053D3F8583B1B0707D535B1BB
:103E6000074A06492046FFF795FD0125E2E7034989
:103E70002046FFF771FDDDE71C1C0D08761C0D08C0
:103E8000261C0D082DE9F041044604F5005750F0BA
:103E90001BFA0122082150F073F95AF013FF97F82A
:103EA0003132072B98BF364A04F5405698BFD55C8F
:103EB000B36A93F8CB8088BF0225B8F1000F0BD10D
:103EC00030492046FFF748FD0025294620460522B7
:103ED000BDE8F041FFF7E6BE2046FFF755FE60B1B2
:103EE00004F53450012212211030FAF75BF8264A0B
:103EF00024492046FFF74EFDE6E7706803681B6D16
:103F0000984768B196F8C53553B196F9C435012B79
:103F100006DC1E4A1E492046FFF73CFD0125D4E77A
:103F2000706803681B6D984718B1D7F8583B19079C
:103F300012D4706803681B689847032803D1D7F828
:103F4000583B9A070BD4D7F8583BDB0609D40D49E8
:103F50002046FFF701FDB8E70C4A0A49DBE70D4AA6
:103F6000C6E770680368DB69984706460028EED10B
:103F7000094A04492046FFF70DFD3546A5E700BF75
:103F8000E41C0D08AB080D081C1C0D08261C0D08B0
:103F9000701C0D087E1C0D08931C0D0870B500F5F3
:103FA0000055044695F93132BBB3D5F8886FA6B3F6
:103FB0008AF064FE05F53B6595ED000ADFED177AA2
:103FC0009FED171ADFED170A861B20EE270A8D20BA
:103FD00025F07CF8BCEEC00A10EE103A9E420DD2DD
:103FE00004F540535B7F9A0717D520460021FAF766
:103FF00033F92046BDE87040FFF7E0BC0DD904F569
:1040000040535B7F9B0708D420460121FAF724F92F
:104010002046BDE87040FFF735BF70BD00007A4410
:104020000000804F000000002DE9F341074600F535
:104030009840183081F04EFA07F54054C0F380489C
:1040400001908AF01BFE94F8203043454546064611
:104050000CD007F5375084F820801030002D3DD06B
:10406000384B394A6662022152F04EFB94F82030F8
:1040700007F500583BB394F8213023BBB8F9C63B91
:104080009FED320A9FED321ADFED320A07EE903AC9
:10409000F8EEE77A40F2571027EE800A25F016F87E
:1040A000BCEEC00A606A10EE103A361A9E420AD977
:1040B000012307F5375084F82130274A214B02218C
:1040C000103052F021FB98F9C53B002B637F0CDCCC
:1040D0006FF34513637702B0BDE8F081194B1F4AB7
:1040E000C4F8248084F82180BDE7C3F34012AA42BB
:1040F000F1D065F3451363779B06ECD5184B5868F0
:1041000003681B6998470028E5D050F0DDF80122CC
:104110001F2150F035F83846FFF736FD48B107F556
:10412000345001222121103002B0BDE8F041F9F7EE
:1041300039BF98F8C51B3222384602B0BDE8F041BD
:10414000FFF7B0BDAC1C0D08BB1C0D0800007A4485
:104150000000804F00000000D11C0D08C61C0D0897
:10416000385C002008B5044B01221A708AF07AFDF1
:10417000024B186008BD00BF8186002084860020A5
:10418000014B00221A707047818600202DE9F04112
:1041900004468AF067FD294BB4F8BE201988284EE2
:1041A000914205460ED01A80264B18603378A3B191
:1041B0000024347050F088F822461321BDE8F04105
:1041C0004FF0DEBF3378204FD3B93B782BB11D4B76
:1041D0001E4A1B68C31A934201D8BDE8F08101232F
:1041E000337004F54053986A90F8CB3013B10368EC
:1041F0009B6A984750F068F8012213214FF0C0FFE6
:104200003B78002BE9D03378002BE6D00D4A1049DB
:104210001368EB1A8B42E0D904F540541560A06A8C
:1042200090F8CB30002BD8D0002183F0DDFFA06ABE
:104230000368BDE8F0415B6A184700BF8286002032
:1042400080860020848600208186002080841E00D5
:1042500040420F002DE9F84300F5405800F50055A5
:104260000446D8F8040095F8EC7003681B6D984775
:10427000014650B995F9F83F002BA5BFD8F8283072
:1042800093F8CB00012180F0010104F5025909F1F6
:104290003009484667F00AF8D8F8283093F8CB3050
:1042A0000646002B7BD0002865D03E4B93F9F83FA3
:1042B000002B04DB02463C49484666F0D1FB95F9E9
:1042C000B67057B195F9F83F002B0EDA04F534506B
:1042D00001220F211030F9F765FE4FF0F5FF32464D
:1042E000BDE8F84309214FF04BBFD8F8040003683C
:1042F0005B69984758B195F9F93F002B07DA98F8B0
:104300001D30DA0703D495F8EC30DB07DED53146F3
:10431000484667F031F8DFED257AB4EEE70AF1EEB2
:1043200010FA05DD0A220921204600F0FDFED4E73F
:10433000023F032F11D801A353F827F025430108AA
:104340004D4301086B430108714301080A221521FE
:10435000204600F0E9FE0028BFD10A2206212046AF
:1043600000F0E2FE0028B8D1DCE70A221121F6E7CE
:104370000A221521F3E797B195F8EC307BB9094B88
:1043800093F9F83F002B06DB04F53750084A052166
:10439000103052F0B9F94FF097FF0022A0E7BDE8C6
:1043A000F88300BF384C0020EC1C0D080000C84208
:1043B000F51C0D0810B500F58044B7EE001A94F80E
:1043C000EA3DDFED080A43F0010384F8EA3D2520C9
:1043D000B0EE410A24F07AFE04F6E85484ED010AB6
:1043E00010BD00BF0000000070B500F54056044647
:1043F000B36A93F8A130032B00F5804509D0384B00
:1044000000221A7095F81C3E62F3000385F81C3EEA
:1044100019E0706803681B6D98470028EFD12046AB
:104420000BF032F980B104F59840183081F068F84B
:10443000DFED2C7AB4EEE70AF1EE10FA20DB95F806
:104440001C2ED1073BD570BDB06A443051F070FBD3
:104450000346DFED250A93ED000A9F20B7EE001A10
:1044600024F034FEDFED217AB4EEE70AF1EE10FA23
:10447000E5DC04F58053D3F8F4231D4B9A42DEDBD0
:1044800004F5005393F8083C6BB104F5546419210A
:10449000204648F039FB042805D11921204648F070
:1044A00053FBC828CBD895F81C3EDA07CBD50C496E
:1044B00091F90020002A10DD013A0A70C3E708498B
:1044C0000B7801335BB2632B0B70BCDD42F0010251
:1044D000642385F81C2E0B70B5E76FF3000395E796
:1044E0008886002000007A4300000000CDCC4C3FBD
:1044F00024FAFFFF2DE9F04100F540560446012162
:10450000B06A81F0ADFA04F58045014604F5005724
:10451000D5F8340C002956D10368D3F89030984769
:10452000B7F8F83F13F48142B36A06D093F8A0219C
:1045300042F0200283F8A02105E093F8A01162F375
:10454000451183F8A01197F9F83FB5F81E0E002B1E
:104550000BDBB36A9FED247AD3ED3E7AF0EEE77A77
:10456000F4EEC77AF1EE10FA3CD5013800B2A5F8A6
:104570001E0EB4F9A4301BB9B4F8A230A4F8A430CC
:10458000B4F9A420002124F0DFFDD5F8343CA5F8CF
:104590001E0E1A68B4F9A410D2F8942007EE900AFF
:1045A000B8EEE70A19B9B4F8A210A4F8A410B4F848
:1045B000A41007EE901AF8EE677ABDE8F04180EE9D
:1045C000270A1846104795F81C1E0368C943D3F8FC
:1045D000903001F001019847B36A93F8A0216FF37E
:1045E0004512A7E70130C1E70000003470B500F5BF
:1045F00040550446686803685B69984708B1002025
:1046000070BD686803681B6898470B28F7D004F5ED
:104610008046D6F8340C0368D3F8A43098470028B5
:10462000EDD1686803681B6D98470028E8D104F550
:10463000005494F9F82F94F8F83F002A07DB9B0602
:1046400005D596F81C0EC04300F00100D8E7012004
:10465000D6E7000010B55AF035FC20215BF036FC9F
:10466000044670B14FF47A715AF072FCB4F9083014
:10467000DFED057A00EE103AB8EEC00A20EE270A08
:1046800010BD9FED020AFBE76F12833A00000000A5
:1046900070B500F540550446AB6A93F8F520012A41
:1046A0000AD0023A022A3BD81A6893F8CC10D26E8C
:1046B00041BB9FED1C0A2FE0FFF7CCFFDFED1A7A1C
:1046C00004F50053B4EEE70AF1EE10FA93F8FA2F6E
:1046D0000EDD42F0100283F8FA2FAD6A2B68DE6E11
:1046E0002046FFF7B7FF28463346BDE8704018471D
:1046F0006FF3041283F8FA2FA86A9FED0A0A036881
:10470000DB6EF2E7B3F9DC109FED070A07EE901AB3
:10471000F8EEE77A27EE800ABDE8704018461047A9
:1047200070BD00BF000000000AD7233C38B500F57B
:10473000405400F50050A56AB0F8F83F03F48143F7
:104740003BB10122002105F1D000BDE838407EF0E8
:1047500079BF95F8CC504DB9606803685B6998479C
:1047600020B1A06A2A460121D030EEE70022A06ADB
:104770001146F9E738B50D4604468AF07FFA002D58
:10478000084B06DD186004F58044002384F81D3EC4
:1047900038BD1B68C01AB0F5C87FF9D904F580444C
:1047A0000123F3E78C86002038B500F5405304461A
:1047B0009D6AFFF71BFF95F8A03160F3000385F8B1
:1047C000A03104F500532046D3F8F43BB3F90810A8
:1047D000BDE83840FFF7CEBF70B500F5005300F5D7
:1047E0009845183586B093F8941D0446284680F005
:1047F0001FFE02A812F002FF04F58F5002A9183024
:104800000DF0BCFC04F58043049AC3F8102C059A03
:10481000C3F8142C284680F05DFE82061AD528467F
:1048200080F066FE04F59845FDEEC07A083504F583
:10483000805417EE901A0222284617EE906A12F062
:10484000E3FE94F87434DB0706D40122314628468F
:1048500012F0DAFE06B070BD0121284612F066FFA4
:104860000028F2D0F6E7000070B500F5804486B06D
:10487000B4F8483E8B420D46164603D1D4F8443E68
:10488000934221D08AF0FAF9D4F8403EC31A132B90
:104890001AD9C4F8446EA4F8485EC4F8400E4FF02C
:1048A00013FD04468AF0F2F9084B094A1B68CDE96A
:1048B0000453084B0193084B0093CDE90201074BC9
:1048C000074920464FF08CFA06B070BD9086002054
:1048D0000C1D0D08241D0D0898F10C08D8D40C08E7
:1048E0001F1D0D0838B500F500540D4694F8F93F2A
:1048F000C3F380138B420BD021B14FF0E5FC1121A3
:104900004FF01EFC94F8F93F65F3861384F8F93FE5
:1049100038BD00007047000010B500F58043044624
:10492000D3F8340C0368D3F8A430984710B904F5D1
:104930004054207810BD0000F8B500F5005406463C
:1049400094F8F83FB1EBD31F0D4643D0224B002221
:104950001A6000293AD04FF0B7FC12214FF0F0FB5B
:1049600094F8F83F65F3C71385F0010784F8F83F22
:1049700072F0D8F9394672F0B1F937B194F8C6310E
:104980001BB98AF07BF9C4F8C80184F8C6710DB36D
:10499000B4F814325B071DD506F54054A36A93F8AA
:1049A000CB30BBB1606803685B69984790B96068B9
:1049B000036820219B69984760B106F534500122B5
:1049C000BDE8F8400D211030F9F7ECBA4FF07CFC4F
:1049D0001C21C3E7F8BD00BF908600202DE9F04FF1
:1049E0002DED088B00F54058C64ED8F8282092F8D7
:1049F000CB908DB0834600F5005A00F58047B9F1A1
:104A0000000F04D10121FFF797FF002423E09AF95A
:104A1000F82F002A18DAD8F804000268D26C904700
:104A200004460028F1D1D8F8282092F8A01111F0FE
:104A3000400100F0638192F8A120032A0BD10146C6
:104A40005846FFF779FF06E097F82C3E0093002BBD
:104A500040D0002434609AF9F82F002AC0F2508127
:104A6000D6ED007ABBF9A420B8EE677A1AB9BBF884
:104A7000A220ABF8A420BBF8A430DFEDA36A07EEB8
:104A8000903AF8EEE77A67EEA67AB4EEE77AF1EEBE
:104A900010FAACBF012100215846FFF723FF9AF915
:104AA000F82F002A9AF8F92FB8BF44F001045306F2
:104AB00097F82C2E48BF44F002040AB144F00804D1
:104AC0003268214658460DB0BDEC088BBDE8F04F6A
:104AD000FFF7CABED8F804000268126D9047051EA1
:104AE000D8F80400026852690CBF002404249047DF
:104AF000002800F0CF80D8F8282092F9A021002AC1
:104B000004DB97F81D2E002A00F0C4800BF58052BC
:104B1000D2EDFF7A9FED7D7AF0EEE77AF4EEC77A78
:104B2000F1EE10FA40F1B68044F400744D460BF5F6
:104B30009B4808F14808404669F096FD0130D7F8D7
:104B4000340C9FED730ADFED73BADFED738A0CBF8F
:104B5000012302236C3008EE103A27F037FD0CAB2E
:104B6000CDED0A0A8DED0B1A8DED090A13E9070048
:104B70000DF10C0E0DF1180C8CE807008EE8070003
:104B8000704627F06FFAD7F8342CDFED647A92ED97
:104B900036AA2AEE27AAB4EEEB0AB3EE0EBAF1EE6D
:104BA00010FA0BF59740B4EECBAACCBF44F4A06446
:104BB00044F480646830F1EE10FAC8BF44F48074A5
:104BC000F0EE40AA51F016F828F0FEF8B8EEC88AC8
:104BD0000BF59840B4EEC80AF1EE10FA00F1180097
:104BE00098BF44F08004F0EE409A80F08DFC68EEAF
:104BF000288AB0EEC09AB4EEE89AF1EE10FA584660
:104C000048BF44F040040AF025FB00285BD144F083
:104C10002004CDF80490404669F026FD012863D1B8
:104C200044F01004CDF80090002D65D0F4EEEBAA0E
:104C3000F1EE10FA60DCB4EECBAAF1EE10FA5BDC18
:104C4000F4EEC89AF1EE10FA56D8B4EEE89AF1EE06
:104C500010FA51D5019B002B4ED0009B002B4BD05E
:104C60003268BBF9A41007EE902AB8EE677A19B93A
:104C7000BBF8A210ABF8A410BBF8A43007EE903A32
:104C8000F8EEE77AB4EEE77AF1EE10FA32D50132B7
:104C90003260E0E65846FFF73FFE10B1002D3FF4CA
:104CA00046AFD8F82820D579002D3FF440AFD7F88B
:104CB0003C2CD2EDDB7AF5EEC07AF1EE10FA3FF53E
:104CC00033AF002533E70BF53050103050F030FF94
:104CD000DFED137A90ED007AB4EEE77AF1EE10FA98
:104CE00095D40023019396E7404669F0BDFC01305E
:104CF0009AD195E70121A3E60022C9E70C46AAE66E
:104D00000121C9E690860020CDCC4C3EDB0FC93F87
:104D10009F0CB3450080BB440000C842E02E6542B2
:104D20000000484330B500F5AA530833044693E821
:104D3000070089B002AD85E807009FED1D7ADDED23
:104D4000047A77EE877A9FED1B7ACDED047AD4ED65
:104D50002B7AF0EEE77AF4EEC77A04F59740F1EE9D
:104D600010FA00F168000BD5B4F9A23007EE903AC2
:104D7000F8EEE77AF7EE006A86EEA77A84ED2B7AF2
:104D8000D4F8AC30019301AA294651F019F8204615
:104D9000FFF724FE2046FEF7AFF92046FEF786FA1D
:104DA0002046FEF743F82046FEF7F6F809B030BD7E
:104DB0000AE81C410000003410B504462DED028BBA
:104DC0001D205BF01BFC58B304F54053586800F0FD
:104DD0002FFC192108EE100A04F5546047F094FEE8
:104DE00002281AD00338012808D804F530501030B2
:104DF00050F09EFE90ED008ABDEEC88AB8EEC88ADB
:104E00009FED090A28EE000ABDEC028B04F59B40D9
:104E10004830BDE8104069F0ADBC9FED048AEDE775
:104E2000BDEC028B10BD00BF0AD7233C0000000080
:104E3000124A0260124A426002F17801816001F573
:104E40002751C16004310161083941612439816110
:104E50000C49C1610C49016202F56261416202F6CE
:104E6000E411816202F6E811C16202F6EC1102F56A
:104E70001F624263054A016382637047B42F0D08C5
:104E8000404E0020303E00206C780020502D002045
:104E900017294BD8DFE801F0100C1418231F2B1C26
:104EA0004A274A2F4A4A4A32364A3A4A4A3E4247F3
:104EB00000F59C405030704700F5AF407C307047A3
:104EC00000F59D401030704700F59D404C30704714
:104ED00000F5AA40EEE700F5AD402030704700F540
:104EE000AC401430704700F5AC405830704700F5C6
:104EF000AE407030704700F5AB40E3E700F5A140ED
:104F00002430704700F5AD405C30704700F5B0408C
:104F10003830704700F5B1400830704700F5005058
:104F2000D0F8B00A704700F5AB40CFE700207047DB
:104F300073B50B6805465B6C08460C4616469847E9
:104F4000034605F537500F4A00960421103051F002
:104F5000DBFB4FF0B9F9236805461B6820469847EC
:104F60000A21024628464FF00BF9074B93F8F93F08
:104F70009B0641BF054A137843F00403137002B047
:104F800070BD00BF281D0D08384C00202C88002063
:104F900038B50C4A182305460C464DF0EDFA78B1A9
:104FA00021462846FFF774FF30B10146064A2846DD
:104FB000FFF7BEFF002038BD28464DF023FAF9E781
:104FC0000120F8E7A81D0D08481D0D0810B500F5D3
:104FD0000053002283F8A42C094B044693F8F81FD1
:104FE00000F5804304F54054D3F8340CC90979F036
:104FF000F7FF60680368BDE81040DB68184700BF32
:10500000384C00202DE9F0410446086803685B69CC
:105010000D461646984798B1306803685B69984713
:1050200070B904F540539B6A93F8CB3043B104F553
:10503000005393F9F83F002B02DB2046F9F7E0F923
:1050400028480AF021FF286803689B68984704F500
:105050009C472B685037BB4210D104F58043002297
:10506000D3F8340C03681146D3F88C30984704F514
:1050700040530021986A03681B6F984728680368AB
:105080005B69984790B9326804F5AF437C339A4224
:105090001CD1B7EE001ADFED140A2520B0EE410A4C
:1050A00024F014F804F59B4383ED1B0A3068036871
:1050B0001B6C9847014698B904F58044D4F8340C29
:1050C0000368BDE8F041D3F8A03018479742EDD10E
:1050D000DFED050A2520B7EE001AB0EE600ADFE723
:1050E000BDE8F0816C8700200000000070B500F57D
:1050F0004055044668680B4E0368DB699847307476
:10510000686803681B689847F070686803689B6C60
:105110009847014604F58D500430BDE8704042F0D8
:105120000DBC00BF0D8800202DE9F34700F5804835
:1051300000F5405998F84C4E88F84C2E0546D9F8A1
:10514000040003681B680F4616469847B8421FD1F3
:1051500005F500551A2E85F8C46107D130B905F65A
:105160008C35D8F8343C2A68C3F8FC20784B93F887
:10517000F93F9D0604D40124204602B0BDE8F08723
:10518000B442F8D0734A137843F002031370F2E785
:10519000022E0AD01B2F10D105F59D4031464C3010
:1051A00002B0BDE8F04701F095BC39462846FFF74C
:1051B000EFFE04460028EDD1DEE739462846FFF72A
:1051C00067FE0446019018B928464DF01BF9D3E755
:1051D000D9F8283093F8CB3083F0010A43B901980D
:1051E000036851465B6898470446A8B95A4A0EE0DE
:1051F00003685B6998470446002840F09A80D9F814
:10520000283093F8A031980700F19380534A019910
:105210002846FFF78DFEAFE705F5405101AA04319E
:10522000284605F50054FFF7EDFE0198C9F8040083
:1052300084F8C46103681B6898473246014605F547
:105240007F604EF053FB05F537500021103058F0C9
:105250004DFF94F9B63023B105F50250303066F0B9
:10526000AFF8D9F8040003681B689847C21E504283
:10527000504104F65C3288F8C40CD8F8343C12680B
:10528000C3F8F82004F68C32D8F8343C1268C3F81E
:10529000FC20012F01D00B2F06D104F67434D8F86E
:1052A000343C2268C3F8FC202846FFF71FFF284B38
:1052B00093F8F93F9B063FF565AF5CE705F50053B2
:1052C00093F8B020002A8AD0B3F8CC20D10786D535
:1052D00093F8EC20002A82D0D9F8282092F8CB202D
:1052E000002A3FF47CAF93F8C4210A2A7FF477AFF9
:1052F00093F9F83F002BFFF672AF194A019928463F
:10530000FFF716FE002437E716480AF0CFF9002809
:10531000D4D1D9F8040003685B6998470028CDD040
:10532000019803685B69984704460028C6D10E4A75
:105330006DE7019803681B6998470028E4D0094885
:105340000AF0A2F904460028DED1084A5FE700BF50
:10535000384C00202C8800200ECC0E08701D0D0843
:10536000951D0D08382C0020831D0D08FE7B0E08AE
:105370000148FFF7D9BE00BF382C002070B52DEDD5
:10538000028B234B5B7FDB0782B006460D4614463B
:10539000B0EE408AF0EE608A06D500232B602360D1
:1053A00002B0BDEC028B70BD59F08CFD037F002B69
:1053B000F3D0F36A9FED171A1B689FED170AB3F934
:1053C000083007EE103AB36A1B68B3F9083007EEED
:1053D000903AB8EEC77AF8EEE77A67EE000A68EE20
:1053E000811A27EE800A28EE011A01A9684624F0E6
:1053F00061FDDFED0A6A9DED007ADDED017A27EEB1
:10540000267A67EEA67A85ED007AC4ED007AC7E7C2
:10541000385C00200AD7233C530469390000C84295
:1054200070B52DED028B88B0002302930393364BA9
:105430005B7F13F0010F0646B0EE408A06AD02AC6A
:1054400003D159F03FFD037F5BB994E8030085E881
:1054500003009DED060ADDED070A08B0BDEC028BE6
:1054600070BDB36ADFED296A1B68B3F9083007EE37
:10547000903AF36A1B68B3F9083007EE103AB8EEB9
:10548000C77AF8EEE77A27EE267A67EEA67AF1EE8B
:10549000476ACDED026ADFED1E6ACDED037AB0EE0C
:1054A000C77AB4EEE67AF1EE10FA06D5F0EEE77AB6
:1054B000F4EEE67AF1EE10FAC7D403AA21461548B5
:1054C000F8F7CCFFDDED027A9DED037AF0EEE77A96
:1054D000B0EEC77AF4EE477AF1EE10FACCBFB0EE38
:1054E000670AB0EE470A204626F00AFD04A88DEDB3
:1054F000040ACDED050A26F0B5FD204688EE000A27
:1055000026F02EFDA1E700BF385C00205304693966
:1055100000000034382C00200A4B93F9F82F002AA1
:105520000DDAB5EEC00AF1EE10FA08D903F5805392
:105530009B6A93F8A100C31E58425841704700204F
:10554000704700BF384C0020436A1B6893F8CB308B
:1055500043B1054B93F8F80F00F0A000203818BFB6
:105560000120704701207047384C002010B5436A75
:1055700004461868D1B1022182F046FE236A9FEDED
:105580000C1A18680368F0EE410ADB6AB0EE410AB3
:105590009847236A074A1868D2ED840A03689FED8A
:1055A000040A5B6EBDE81040002118470121E3E7C3
:1055B00000000000384C002010B5436A044618680B
:1055C000002930D0022182F01FFE236A186879F08A
:1055D000D7FC636A1B6893F8A130012B04D8236AB7
:1055E000012118687AF066FA636918687DF016FA86
:1055F000636918687DF072FA63699FED0C0A186898
:105600007DF098FC636918687DF006FD236A9FEDC4
:10561000071A18680368BDE81040DB6AF0EE410A1B
:10562000B0EE410A18470121CDE700BF000000009D
:1056300013B5044601A90C4809F09CFE10B101986D
:1056400002B010BD636918687CF0F2F818B9074B16
:10565000D3F80C0CF4E7064801AA032112F00AF86B
:105660000028F4D0EBE700BF382C0020386C002075
:105670004078002070B504462DED028B00296AD1D8
:105680008368B3F92E58642DB8BF6425FFF7D0FFA7
:10569000A8426268A4BF324B93F8F95FB2F9343084
:1056A000ACBFC5F380150125002BDBBF63691B6808
:1056B0005B4293EDC48AC8BF07EE903AB2F932302C
:1056C000C8BFB8EEE78A002BB8BF5B429BB25B4213
:1056D00007EE903AA368F8EEE77AB3F92E68F4EE95
:1056E000C87AF1EE10FAD8BFB0EE678A2046642E71
:1056F000B8BF6426FFF79CFF6369A26B1B68D2EDFD
:10570000001A93EDC61AD3ED0E0A311A00EE101AE4
:10571000B8EEC00A23F0BCFF6368B3F93230002B47
:10572000B8BF5B429BB25B4201EE103A40F2972059
:10573000B8EEC11AF0EE480A23F0C8FC63692946A6
:1057400018687CF019F9BDEC028B6369BDE8704004
:1057500018687DF061BC9FED030A0025EEE700BFED
:10576000384C002000000000436A186803681B6979
:105770001847000038B52DED028B03680446D3F8B6
:1057800084309847236B2A481B68F0EE408AB3F9AF
:10579000085009F0FFFC4FF47A72041E4FF000012C
:1057A0002846D8BF4FF4FA7423F0CEFC8442B6EEFC
:1057B000000A2ADD07EE900AB8EEE77A07EE904A73
:1057C00027EE007AF8EEE77A87EE278A4FF46D70BD
:1057D00038EEC00AF5EE087AB1EE400A80EE270AEC
:1057E000B7EE001AFEEE000A23F070FCF7EE007A26
:1057F00077EEC07A28EE000A20EE080A20EE080AAA
:10580000A7EE880ABDEC028B38BD031B07EE103AE9
:10581000C4F57A74B8EEC77A07EE904A27EE007A9C
:10582000F8EEE77A87EE278A38EE008ACEE700BFE7
:10583000382C002013B504468DED010A68F0ACFE4B
:105840006369A26B1B6892ED001A93ED0E0AD3ED0B
:10585000C60A01A967F02EFD9DED010A02B010BD38
:10586000436A186803685B6A1847000038B5436AE2
:105870001C6894F8CB10054661B9204682F0C4FC40
:105880006B6A1B6893F8A10018B1012814BF0320AC
:10589000022038BD164803783BBBFFF73DFE20BB16
:1058A000144A92F8F83F03F0A003202B17D0B5EE6E
:1058B000C00AF1EE10FA10D592F8FA3F5B070CD44B
:1058C0000121204682F0A0FC6B6A1B6893F8A1308E
:1058D000012B0CBF02200320DBE70221F1E7204669
:1058E000022182F091FC0420D3E70120D1E700BF20
:1058F0006C870020384C002010B52DED028B124B28
:105900005B7FDB07044604D59FED100ABDEC028BDC
:1059100010BD59F0D7FA037F002BF5D0636B1868E0
:1059200059F0FAFBA368DFED0A7A03F5116292EDF4
:10593000008A03F61413D3ED000A28EE278A24F018
:1059400073FA28EE000AE1E7385C0020000000004E
:105950000000C8420148F8F7AFBD00BF382C002056
:105960000148F9F7DBB900BF382C00200148FFF7E8
:10597000DBBB00BF382C0020F0B57E4D2DED028B37
:1059800095F8F93F8DB00026044658060496059612
:1059900003D5636918687BF0BFFD774F7B7FD9071C
:1059A0005ED463689B899A071CD5744850F0C0F890
:1059B000DFED737A90ED007AB4EEE77AF1EE10FA4B
:1059C00010DD4EF081FC3D214EF0BAFB092205218D
:1059D000A7F54050FFF7A8FB20B909220221204675
:1059E000FFF7C4FF636893F95430CBB365489FED6C
:1059F000668AF9F793F9E3689FED647A1B68D3ED43
:105A00000A7AF4EEC87AF1EE10FAB8BFF0EE477AEF
:105A1000B6EE000A27EE800A2046FFF701FD8DED65
:105A2000040AB0EEC00AB4EEC80AF1EE10FACDEDE9
:105A3000050A06D5F0EEE00AF4EEC80AF1EE10FA17
:105A40000ED495F8FA3F1B0704D44EF03DFC4921D3
:105A50004EF076FB95F8FA3F43F0080385F8FA3FDD
:105A600095F8FB3F09966FF3820385F8FB3F606969
:105A70000A9609AE324604A9006801237BF0B6FD00
:105A8000636918687DF02AF8636918687CF002F988
:105A9000A3688DED060ACDED070A8DED081AD3ED4A
:105AA000007AF5EEC07AF1EE10FA51DDB5F9043264
:105AB0009FED378A00EE903AF8EEE00A2046CDEDF1
:105AC000030AFFF7B5FDA368DDED030AD3ED001A65
:105AD0009FED2B0AB7EE002A07EE900A31EE822ADC
:105AE000B8EEE71A22EE082A61EE881A23F02EFAA1
:105AF000DFED287A20EE270ADFED277A20EE270A4D
:105B0000AFF026FBDFED257A20EE270A06A820EE6F
:105B1000088A26F0A7FAB4EEC08AF1EE10FA17D57B
:105B2000C8EE006A63699DED067ADDED077A27EE1F
:105B3000267A67EEA67A8DED067ACDED077A1B6898
:105B4000D3F88823C3F89423D3F88C23C3F898237D
:105B5000236A13491C683046FCF7E4FE0B9B009354
:105B600096E80C0006A9204679F0BCFA0DB0BDEC11
:105B7000028BF0BD384C0020385C002034780020C7
:105B800000002F44382C00200000003400007A432D
:105B90000000C8420AD7233C35FA8E3C0AE81C4173
:105BA0003C86002013B504460191FFF7E5FE0199FC
:105BB000204602B0BDE81040FFF75CBD0148FEF78B
:105BC000BBBE00BF382C002000487047085A002098
:105BD0000148F8F75FBC00BF382C002030B50F4DEE
:105BE00087B0002304466946D5F83C0C0093019326
:105BF00002937CF067F8D5F83C0C02A97CF0B6F86B
:105C0000009B0393019B04930222029B059303A92B
:105C1000204611F0FFFF204607B030BD386C002051
:105C2000014B01221A7070479486002000207047B3
:105C30000020704700207047002070470020704708
:105C400000207047002070470020704700207047F8
:105C500000207047002070479FED010A704700BF89
:105C600000000000002070470020704700207047AF
:105C700001207047002070470020704701207047C6
:105C800000207047012070470120704700207047B6
:105C9000012070470120704700207047004870477E
:105CA000BCC70E0800487047BCC70E0890F83C30CF
:105CB00043B9836893F82439DB0742BF034B0122C1
:105CC000C3F8FC2F002380F83C307047384C00208C
:105CD0002DE9F0432DED0C8BF0EE409A20EE000AFA
:105CE00097B00025A0EEA00A04468946B0EE41CA4E
:105CF000F0EE60AA90461F46019502950395049523
:105D000005950695AFF070FCF7EE00CAB4EEEC0A0C
:105D1000F1EE10FAC8BFCCEE807AA36803F50E62EC
:105D200003F6E40392ED009A9FEDC5DAD3ED000A85
:105D3000C4BF69EEA79A6AEEA7AAB0EE690A24F07A
:105D400073F8A36829EE0D9A03F50E6203F6E403D7
:105D5000D2ED008AD3ED000A29EE009AB0EE6A0A6D
:105D600024F062F8A36868EE8D8A03F6F80203F661
:105D7000FC03D3ED000A92ED008A68EE808AB0EE53
:105D80004C0A24F051F8636828EE0D8A93F97030BC
:105D900028EE008A002B00F0D980236A9FEDA90A23
:105DA00018686C3026F012FCB0EE60AACDED080A3F
:105DB0008DED091A8DED070A23F032F9BDEEC0BA58
:105DC000A14940F6B8321BEE100A23F0ADF9434268
:105DD00007EE903A6368F8EEE77A93ED1A7A67EE89
:105DE000877AB0EE4A0ACDED017A23F019F9FDEE7B
:105DF000C0BA40F6B83294491BEE900A23F094F9E9
:105E000042426368039507EE902A93ED1B7A93F95B
:105E10007030F8EEE77A022B67EE877ACDED027AE2
:105E20006ED18A4BB3F904320AEE103AB8EECBBA0F
:105E3000B8EECAAA236AB4EECABAF1EE10FA1A682A
:105E40003DDDA368DFED820AA16B92ED051AD1ED6D
:105E5000001A03F50E6393ED007A27EE0D7A3AEE01
:105E60004B0AC7EE200A23F013FCDDED017A37EE72
:105E7000800A8DED010AB8EEEB0A236AB4EECA0A75
:105E8000F1EE10FA1A6834DDA368A16B92ED061AE0
:105E9000D1ED001A03F50E63D3ED000A20EE8DDA82
:105EA000DFED6B0A3AEE400ACDEE200A23F0F0FB5C
:105EB000DDED027A37EE800A8DED020A20E0B1EEC8
:105EC0004A0AB4EEC0BAF1EE10FAD4D5A368A16BB9
:105ED000DFED5F0AD1ED001A92ED051A03F50E63AE
:105EE00093ED007A27EE0D7A30EE4B0AC7EE200ACA
:105EF000B9E7B1EE4AAAB4EECA0AF1EE10FAC3D479
:105F0000236AD3F800C00CF184030FCB12AD85E8EF
:105F10000F000EAE0AAD86E80F0085E80F0004AB57
:105F200001AA2946604679F079FD636893F97030DB
:105F3000022B16D1DDED047A39EE279ADDED057AD4
:105F400078EEA78ADDED067A38EE278A89ED009A89
:105F5000C8ED008A87ED008A17B0BDEC0C8BBDE858
:105F6000F083F0EEE99AF0EEEAAAF4EEE9AAF1EE97
:105F700010FA48BF6D46CDED009ACDED0AAAD5EDD9
:105F8000007ADFED340AB0EECCCAF4EECC7AF1EE52
:105F900010FAD8BF35468DED0ECA95ED007ADFEDCB
:105FA0002E7A87EE270AAD20B7EE001A3CEEC00A23
:105FB00023F08CF8E369D3ED937A04A820EE270A46
:105FC00026F004FBF0EEC07A8DED061AB0EEC91A89
:105FD00031EE671A8DED040AB0EEC11A39EE000AEF
:105FE000CDED050AB520F1EE410A23F06FF8B0EED1
:105FF000409A9DED050AB0EEE81AF0EEC07A31EE57
:10600000671A38EE800AB0EEC11AF1EE410ABA20E2
:1060100023F05CF8F0EE408A9DED060AB0EEC81A57
:10602000F0EEC07A31EE671A38EE000AB0EEC11A0F
:10603000BF20F1EE410A23F049F8B0EE408A85E72F
:106040000000C8429F0CB34548F4FFFF384C0020C5
:1060500000007A440000000000A08C45836893EDA6
:10606000040AB5EEC00AF1EE10FA01DCFFF77CBBC2
:106070007047000073B5036A1D682B68D3F88C6005
:10608000436A0446186803689B6E9847636A0190E8
:10609000186803689B6F9847019902462846B047E5
:1060A000636A1868036801211B6F9847044B93F8D3
:1060B000EA2D01206FF3000283F8EA2D02B070BDD3
:1060C000386C00202DE9F0412DED048B96B00024B2
:1060D0001E46036A01940294039404940594069462
:1060E00005461868F0EE408A6C309FED2E0A88460F
:1060F0001746B0EE609A26F069FAEB698DED070A53
:10610000D3ED7E7ACDED080AF8EEE77AB0EE608A3C
:1061100030EE670A8DED091A22F082FFEB6920EE5E
:10612000490A8DED010A93ED7F0AB8EEC00A38EEF8
:10613000400A22F075FF20EE680A2B6A03948DED69
:10614000020AD3F800C00CF184030FCB12AD85E82E
:106150000F000EAC0AAD84E80F0085E80F0004AB19
:1061600001AA2946604679F059FCD8ED007A9DEDE8
:10617000047A77EE877A9DED057AC8ED007AD7ED3F
:10618000007A77EE877A9DED067AC7ED007AD6ED34
:10619000007A77EE877AC6ED007A16B0BDEC048BF4
:1061A000BDE8F0819F0CB34530B52DED028B436AFD
:1061B0000446186890F8CB1087B0002940F085801D
:1061C00082F022F8636A186890F8A150012D7ED001
:1061D000032D00F09F8045B9236A294618687AF09C
:1061E000C3F9236A186878F0B5FE636A1868036813
:1061F0009B6E9847A36A002840F09980186858F071
:106200008BFFE36A1868B0EE408A58F085FF636B35
:106210008DED010A186858F07FFF05ABB0EE401A0B
:1062200004AADDED010A03A9B0EE480A2046FFF7F3
:106230004FFD636893F9702092B9534A92F9F82F91
:10624000002AB3BFF0EE080AD3ED1A0A93ED1B0A39
:10625000B0EE600A05AB04AA03A92046FFF732FF9F
:10626000636A186803689B6F984748B1636B186846
:1062700058F008FF07EE900AF8EEE77ACDED057AC0
:10628000236AA268186892F8242903689DED030A1E
:10629000DDED040A9DED051A92074CBFDB6B9B6B8D
:1062A0009847236B39481B68B3F908107DF014F840
:1062B000236A62681868D2ED020A036800215B6EE7
:1062C000984707B0BDEC028B30BD022178E7036828
:1062D000DB6B984768B92C4B93F9F83F002B84DAB5
:1062E000636A012118687FF0BBFB00287FF47DAF53
:1062F00006E0636A294618687FF0B2FB0028EAD0FE
:10630000236A002118687AF02FF9236A186878F058
:1063100037FE6AE71C4B93F9F83F002BBFF665AFD9
:1063200001217FF09DFB00287FF45FAFEDE7186847
:1063300058F0A8FEE36A07EE900A1868B8EEE78AFC
:1063400058F0A0FE636A07EE900A186803689B6F16
:10635000F8EEE78A984788B1636B186858F092FEA8
:1063600007EE900AB8EEE71A236A18680368F0EEA1
:10637000680AD3F89C30B0EE480A91E72046FFF750
:10638000BBFAB0EE401AEFE7384C0020207A00202C
:1063900070470000002070470120704702207047BE
:1063A0000020704700207047012070470020704790
:1063B00081F0010070470000012070470120704704
:1063C0000120704700487047541E0D080048704770
:1063D000601E0D0838B54369044618687BF04AFB17
:1063E00018B9636918687CF0C9FC636920461D68A8
:1063F000FFF7EEFB6368B3F93820B3F9363000EEEF
:10640000903A434201EE102A00EE103AB8EEC11A5B
:10641000F8EEE00AB8EEC00A28467BF017FA636986
:1064200020461D68FFF7D4FB6368B3F93820B3F941
:10643000363000EE903A434201EE102A00EE103A58
:106440002846B8EEC11AF8EEE00AB8EEC00A7BF0B2
:1064500077FA012038BD000030B52DED028B0446DF
:10646000436985B01D68FFF7B3FB6368B3F9382053
:10647000B3F9363000EE903A434201EE102A00EEB6
:10648000103AB8EEC11AF8EEE00AB8EEC00A284693
:106490005B4D7BF0DBF92046FFF762FAB5F9043279
:1064A00008EE103A236A186803689B6E9847B8EEA6
:1064B000C88AF0EE400A02AA01A9B0EE480A2046B6
:1064C000FEF75CFF2046FFF717FA236B1B68B3F952
:1064D0000830F0EE408A00EE103A2046B8EEC00ACE
:1064E000FFF738FA2046B0EE408A8DED030AFFF739
:1064F0006FFB6368B3F9363001EE103A434200EEA9
:10650000903AB8EEC11AF8EEE00A2B20B0EE480A35
:1065100022F0DCFD20468DED030AFFF7A7F90428E1
:1065200013D8DFE800F0032F252A4B00236A1868F0
:1065300078F010FD236A0021186879F0BBFA6369CE
:106540009FED300A18687CF0F5FC236ADDED020A45
:1065500018689DED010A0368B0EE681ADB6A984777
:10656000636918687CF058FD05B0BDEC028B30BD46
:10657000236A0121186879F09DFA236A186878F077
:10658000FFFCDCE7204D2B7863B963689FED1F1A91
:10659000DFED1C0A93ED040A452022F097FD284602
:1065A00009F05AFC20469DED030AFFF743F916480F
:1065B0008DED030A03A909F089FCC6E7636A02218D
:1065C000186881F021FEB5F90432114800EE103A46
:1065D00002AA01A9B8EEC00A66F09CFB20469DED18
:1065E000030AFFF727F90B488DED030A08F0DEFEDA
:1065F00063699DED030A18687BF0AEF9A5E700BF5B
:10660000384C0020000000006C87002000007A4415
:1066100090790020D05800200020704790F8B931C0
:10662000002B14BF1B200320704700000020704780
:106630000120704790F89001062804D0A0F10A03C9
:1066400058425841704701207047000001207047B0
:10665000012070470120704790F8B901034A044BAC
:10666000002814BF10461846704700BFFC1E0D08D6
:1066700032900E0890F8B901034A044B002814BF69
:1066800010461846704700BF081F0D0832900E08CC
:1066900090F890010B3818BF0120704790F8B9317D
:1066A0002BB9044BD3F8A80B00F001007047002071
:1066B000704700BF384C002090F8903123B9034B4D
:1066C000187880F001007047002070475087002044
:1066D00038B590F89041012C054601D0002038BD16
:1066E000C368186803681B6998470028F6D1EB68EF
:1066F0001B68204683F8B848F1E70000C3681B68B0
:10670000002283F8B82801207047000070B52DEDF5
:10671000028B002380F8B931B0F87030012B84B0BF
:1067200004460D4601D8002946D0636A254E1B68F1
:1067300093F8CB3073BB2448072384F89031036867
:10674000022B02D10021FBF7FDFE9FED208AE368BA
:10675000F0EE480A1868B0EE481AF0EE481AB0EEAB
:10676000480A01257EF0F6F884ED738A84ED748A78
:1067700084ED758A84F8B85104F59A7026F00EFC01
:10678000134804F0C5FD96F8FA3F6FF3C30386F88B
:10679000FA3F11E096F9F83F002BCCDA04F13C0007
:1067A00028F0D4FC05460028C5D12046FFF70CFA96
:1067B000084A02214FF0A8FF284604B0BDEC028B26
:1067C00070BD00BF384C00203C8600200000000057
:1067D0004C820020101F0D0838B5094D95F80C3F6C
:1067E000012B044603D105F6087026F03FFC95F80E
:1067F0004D1D04485BF00EF8002384F8B93138BD14
:10680000386C00200C79002010B52DED028B094B5F
:106810000446D3F8400CB0EE408A7DF033FC9FED87
:10682000060A28EE008A012084ED748ABDEC028BF2
:1068300010BD00BF386C00200AD7233C10B52DEDE9
:10684000028B094B0446D3F8400CB0EE408A7DF031
:1068500029FC9FED060A28EE008A012084ED758A46
:10686000BDEC028B10BD00BF386C00200AD7233C62
:1068700010B52DED028B094B0446D3F8400CB0EE59
:10688000408A7DF01DFC9FED060A28EE008A01205B
:1068900084ED738ABDEC028B10BD00BF386C002004
:1068A0000AD7233CC3681B6818697BF025BB00002E
:1068B00038B5D0F8943104460D461BB988F0DEF99E
:1068C000C4F8940188F0DAF9D4F89431C01A4FF47E
:1068D0007A73B0FBF3F0B4F89231984209D32046B2
:1068E000FFF772F92B88044A06214FF00DFF0120B3
:1068F00038BD0020FCE700BF2C1F0D0890F8903138
:10690000052B05D1054BD3F8483CD8687BF06CBA11
:10691000C36818680368DB68184700BF386C00203C
:1069200008B590F89031052B0BD1094BD3F8483CB2
:10693000D868243025F096FBBCEEC00A10EE100A91
:1069400008BDC368186803689B689847F4E700BFF0
:10695000386C002090F890318B4206D00B2B80F8D9
:10696000901102D10148FCF7F3BE7047382C00208B
:10697000F7B501231E4E80F87530736883420546D3
:106980000A46A6F5805713D1012485F8B9417068ED
:10699000019203681B689847019A014615484CF01C
:1069A000A5FF97F8F93F9A061BD4204603B0F0BD27
:1069B00001910321FEF7DAFF019A04460028E3D192
:1069C00085F875004DF080FC1B220A214DF0D8FBA4
:1069D00097F8F93F9B06E8D5074A137843F004037C
:1069E00003E0054A137843F002031370DDE700BFAC
:1069F000385C0020283C00202C88002030B585B071
:106A000004460D4601466846FFF7E8F8694604F17A
:106A10003C0029F04DF9C8B94DF056FC1B220A2163
:106A20004DF0AEFB0D4B93F8F93F9B0604D50C4A95
:106A3000137843F0040313702046FFF7C5F8094AA2
:106A400004214FF061FE002005B030BD29462046EC
:106A500005B0BDE83040FFF78BBF00BF384C0020C9
:106A60002C880020401F0D0830B585B004460D4627
:106A700001466846FFF7B2F8694604F13C0029F088
:106A80003BF9C8B94DF020FC1B220A214DF078FBE0
:106A90000D4B93F8F93F9B0604D50C4A137843F04D
:106AA000040313702046FFF78FF8094A04214FF0C2
:106AB0002BFE002005B030BD2946204605B0BDE8BC
:106AC0003040FFF755BF00BF384C00202C88002015
:106AD0007C1F0D087FB505460E4605F13C040146B6
:106AE0006846FFF77BF86946204629F005F9C0B9EA
:106AF0002046694629F0DCF8044690B94DF0E4FBE5
:106B00001B220A214DF03CFB0D4B93F8F93F9B06ED
:106B10000FD42846FFF758F80A4A04214FF0F4FD35
:106B200004E031462846FFF723FF0446204604B020
:106B300070BD054A137843F004031370E9E700BF02
:106B4000384C0020B41F0D082C88002030B50446B6
:106B500085B00F4808F098FD0546B0B1072384F8CA
:106B600090310023019302930393E36801A918680D
:106B70007DF022FAE3681868036801A95B680022C7
:106B8000984704480021FBF7DDFC284605B030BDDE
:106B9000382C00203C860020F0B5424FD7F8142C4A
:106BA000D7F8103C2DED028B1343D7F80C2C134370
:106BB00087B005460C460CD14BF092FE40F27512A0
:106BC0004FF4801107B0BDEC028BBDE8F0404BF0F4
:106BD0003FBE80697EF08CFC2046B0EE408A10F00B
:106BE0003DFD03283AD1EB6801A918687DF0C0FA91
:106BF000064698B3DDED017A6368009338EE678A44
:106C0000294BDFED2A7A93F9F83F9FED290A2948AD
:106C1000002BA8BFB0EE670A38EE008A009BBDEEDD
:106C2000C88A002118EE102A9342ACBF009300924C
:106C3000FBF788FC6B6918687CF0A0F8DDED007A42
:106C40001D48B8EEE70A314609F0BCFB0021284692
:106C5000FFF780FE07B0BDEC028BF0BD94E80F009B
:106C600002AE86E80F00D7F8103C04936A46D7F8C6
:106C7000143C05930221304610F0FCFC78B94DF02D
:106C800023FB022215214DF07BFADDED037AF8EEAD
:106C9000E77A77EE887AFDEEE77ACDED007A002686
:106CA000AEE700BF386C0020384C00200000000028
:106CB0000000C8423C8600205087002030B52DEDF2
:106CC000028BC36887B0044618680D467DF044FA0D
:106CD00000284BD194F89021002300930193029354
:106CE0006AB93148039303A90493059309F09AFB09
:106CF00028B1039B0093049B0193059B029394EDA1
:106D0000730A9FED2A8AE368DDED000A9DED011A02
:106D1000DDED021A1868B4EEC80AF1EE10FAAABF47
:106D2000DFED237A9FED230A20EE270A7DF012FE85
:106D3000D4ED747AF4EEC87AF1EE10FA07DBE3686A
:106D40009FED1B0A186827EE800A7DF09BF9D4EDB1
:106D5000757AF4EEC87AF1EE10FA07DBE3689FED7E
:106D6000140A186827EE800A7DF09CF9E36829462A
:106D700018687DF017FD054688B10F4B1B68022B84
:106D800009D0032B03D10D4B93F935321BB10A48BF
:106D90000021FBF7F5FB01212046FFF7DBFD28462C
:106DA00007B0BDEC028B30BD5087002000000034DE
:106DB0000000C842000000003C860020384C002043
:106DC00010B52DED028BC368DFED348A1B68426974
:106DD000D3ED0A0A9FED328A93ED060AF4EEE80A33
:106DE0000446F1EE10FA1068B8BFF0EE480A7AF0E7
:106DF00013FBE36862691B681068D3ED0A0A93ED20
:106E0000060AF4EEE80AF1EE10FAB8BFF0EE480A0E
:106E10007AF07AFB636918687AF00AFD18B9636939
:106E200018687BF045FDE36862691B68106893EDA4
:106E3000080A93ED0C1AD3ED070AB0EEC00A7AF0F7
:106E400005FDE36862691B68106893ED080A93ED1D
:106E50000C1AD3ED070AB0EEC00A7AF071FD63692F
:106E600018687AF007FE18B9636918687BF086FF26
:106E700000210C48FBF766FB0B4867F013FD0B4A3B
:106E8000B2F8FA3F23F48163A2F8FA3FBDEC028B1B
:106E900020460221BDE81040FFF75CBD0000003431
:106EA00000007A433C860020007A0020384C002005
:106EB00010B50C4B0446D3F8480C90ED0B0A90F833
:106EC000502000F11C017CF0BFFD07480368022B35
:106ED00002D00821FBF736FB20460521BDE8104013
:106EE000FFF738BD386C00203C860020F0B52DED52
:106EF000028B4A4DDFED4A8AB0EE408A8FB00446DD
:106F0000D5F8480C0E4617467CF014FCF0EEC87A13
:106F1000F4EEE87AF1EE10FA07D49FED420AD5F8C4
:106F2000480C28EE000A7CF06BFCD5F8480C90ED7C
:106F30000B0AB0EEC00A0FB1B1EE400A7CF050FC73
:106F40000023D5F8480C079302AA07A908930993D0
:106F50007CF072FCDFED347A9DED027AB4EEE77AD4
:106F6000F1EE10FA56DD022207A90AA810F052FE2F
:106F700071680191304610F071FB019902460AA830
:106F800010F042FBE3680AA918687DF00BFC10B909
:106F90002648FCF727FEA0697EF0A8FA026843683D
:106FA000D5F8480C049303A91C30039224F08CFFFD
:106FB00005A88DED050ACDED060A25F053F81C4B0A
:106FC0001B68022B1BD0D5F8483C1948D3ED0A7A30
:106FD000F4EEE87AF1EE10FAB8BFD3ED047AF4EEED
:106FE000C07AF1EE10FA4FF0000110D5DFED117A02
:106FF000B4EEE70AF1EE10FA09DDFBF7C1FA04215D
:107000002046FFF7A7FC0FB0BDEC028BF0BDFBF7ED
:1070100099FAF4E72046FFF74BFFF4E7386C0020BD
:10702000000000340000C84200009643382C0020C5
:107030003C8600200000FA4370B52DED028B294BF1
:10704000DFED298AD3F8404CD3F83C5CD4ED0A0A32
:107050009FED268A94ED060AF4EEE80AF1EE10FAA6
:10706000B8BFF0EE480A064628467AF0D5F9D4EDC6
:107070000A0A94ED060AF4EEE80AF1EE10FAB8BF37
:10708000F0EE480A28467AF03FFA28467AF0D0FB1C
:1070900010B928467BF00CFC94ED080A94ED0C1A0C
:1070A000D4ED070AB0EEC00A28467AF0CFFB94ED83
:1070B000080A94ED0C1AD4ED070A2846B0EEC00A6F
:1070C0007AF03EFC28467AF0D5FC10B928467BF0D1
:1070D00055FE07480021FBF735FABDEC028B012372
:1070E000337070BD386C00200000003400007A431B
:1070F0003C86002008B50748D0F8A83B9B0704D57C
:107100000121A0F50050F7F747F8BDE80840024814
:1071100008F0BABF384C00205087002030B589B045
:107120000446FEF711FA30B10021204609B0BDE84F
:107130003040FEF741BA636A0221186881F064F8B2
:10714000E368186803685B69984701461048FCF7D4
:1071500047FC636918687BF05FFF236A1D686369F9
:1071600018687AF097FD05AC20460A498DED020AB1
:10717000CDED030A8DED041AFBF7D4FB079B0093BA
:1071800094E80C0002A9284677F0ACFF09B030BDA6
:10719000382C00203C86002038B50446FEF7D4F990
:1071A000054628B120460021BDE83840FEF704BA64
:1071B000636A0221186881F027F829462046BDE855
:1071C0003840FEF7EFBC00000148002106F0ACBBE0
:1071D000A883002030B5174D9FED170A05F58043B1
:1071E00089B00446D3F8480C7CF08EFC0146284652
:1071F000FCF7F6FB636918687BF00EFF236A1D68D5
:10720000636918687AF046FD05AC20460B498DEDA0
:10721000020ACDED030A8DED041AFBF783FB079BF1
:10722000009394E80C0002A9284677F05BFF09B0B0
:1072300030BD00BF382C0020000000003C8600203C
:1072400030B589B00446FEF77FF930B10021204601
:1072500009B0BDE83040FEF7AFB9636A0221186893
:1072600080F0D2FFE368186803685B6998470146BD
:107270001048FCF7B5FB636918687BF0CDFE236A04
:107280001D68636918687AF005FD05AC20460A4957
:107290008DED020ACDED030A8DED041AFBF742FBDA
:1072A000079B009394E80C0002A9284677F01AFF88
:1072B00009B030BD382C00203C86002030B52DEDC3
:1072C000028B83B00446FEF73FF920B9636A1B685E
:1072D00093F8CC3043B90021204603B0BDEC028BBB
:1072E000BDE83040FEF768B994F89831DA071DD44C
:1072F000E3681D682B6828469B689847D5ED097A96
:1073000094F89831B4EEE70AF1EE10FA4CBF01227E
:10731000002262F3000384F8983107D4204603B0BA
:10732000BDEC028BBDE83040FFF7F8BE94F8983111
:107330009B0734D4E368DFED458A1B686269D3EDAF
:107340000A0A9FED438A93ED060A1068F4EEE80AF4
:10735000F1EE10FAB8BFF0EE480A7AF05DF8E36893
:1073600062691B681068D3ED0A0A93ED060AF4EE11
:10737000E80AF1EE10FAB8BFF0EE480A7AF0C4F865
:10738000636918687AF054FA18B9636918687BF071
:107390008FFA94F8983143F0020384F898312D4B1A
:1073A000D4F8A021D3F80C3C9B1A07EE903AB8EE23
:1073B000E78AF1EE047AB0EEC87AB4EEE77AF1EE3D
:1073C00010FA38D594F8983143F0040384F89831D2
:1073D000204684ED678AFEF7CFFA6369A26B1B68CB
:1073E000D2ED001A93EDC61AD3ED0E0AB1EE480A9B
:1073F00022F04EF963691B6840F2AA4093EDC31A6C
:10740000D3EDC40A21F062FE2046FEF713FA1248BB
:107410008DED010A07F0CAFF63699DED010A186846
:107420007AF09AFA6369186803B0BDEC028BBDE884
:1074300030407BF0F1BDD4ED677A68EE277AF5EE47
:10744000C07AF1EE10FAC3D5BCE700BF00000034EB
:1074500000007A43386C0020D058002030B52DED64
:10746000028B83B00446FEF76FF820B9636A1B688D
:1074700093F8CC3043B90021204603B0BDEC028B19
:10748000BDE83040FEF798B86369DFED347A1B68D9
:1074900094ED710A93EDC31AD3EDC40A20EE270AC6
:1074A00040F2C44021F012FE2046FEF7C3F9236AE1
:1074B000186803689B6EB0EE408A9847284BB3F972
:1074C000043207EE903AB4F8BC316425F8EEE77A5E
:1074D00013FB05F3B4EEE70A07EE103A94F9BE3158
:1074E000F1EE10FAD8BFF0EE407A13FB05F39FEDF2
:1074F0001D0AF8EEC76A07EE103AF4EE407AB8EECD
:10750000C77AF1EE10FA58BFB0EE670A6846CDEDC3
:10751000006A8DED017A24F0F7FD236ADDED010AA2
:107520001868B4F8C03102689DED000A126B13FBB5
:1075300005F301EE103A0121B8EEC11A90476369D4
:10754000B0EE480A18687AF007FA636918687BF0A9
:1075500063FD03B0BDEC028B30BD00BF0000C8422C
:10756000384C002000007A442DE9F0432DED028BC9
:10757000DFF89C8385B00446D8F80400FDF7E4FFEB
:1075800048B1D8F80400002105B0BDEC028BBDE87D
:10759000F043FEF711B808F58057D8F8280002210B
:1075A00080F032FEA8F58056D7F8343C93ED378A48
:1075B00087F064FBB6F8F83F03F4814305467BB1DE
:1075C000D7F83C0C79F0A8FF2378022B08D155F0AE
:1075D0006FFFC04BC04A06214FF096F8032323707B
:1075E00062F082FE62F06CFE48B162F07DFE62F0F5
:1075F00071FE20B12378012B10D9022B1DD02378E6
:10760000082B00F28781DFE813F0210039006200C7
:1076100006011F0126013C013E012A0055F048FFEA
:10762000AC4BAE4A06214FF06FF8D7F83C3CD3F88C
:107630005433636108232370E1E755F039FFA54B0C
:10764000A74A06214FF060F80323F4E7D7F8400C6F
:1076500003681B69984710B12046FFF7EDFC2378BB
:10766000082B00F27581DFE813F05E016601660108
:107670007C017C017C017C0184018401A560D7F838
:107680003C3C9FED987AD3F85433636106F6E433BB
:10769000D3ED007AF4EEC77AF1EE10FA4EDB9FEDEF
:1076A000927A67EE877AD7F8403C93ED087AB0EE8D
:1076B000C77AF4EE477A4FF07E53F1EE10FA48BFE6
:1076C000B0EE677A2361022384ED067A2370D4ED4D
:1076D000016A9FED847AD7F83C3CF0EEE67AF4EE4E
:1076E000C77AF1EE10FA0AD4D4ED057A93EDD56A93
:1076F00077EEC67AF4EEE76AF1EE10FA29D4DFED00
:107700007B6AD4ED067A67EEA67AD3EDDB6AF4EEF7
:10771000E76AF1EE10FA26DCA368D4ED047AEB1ADE
:10772000B3F5FA6F21D2B4EE678AF1EE10FAC8BF52
:10773000B0EE678A84ED048AE56090E7B6F93A32E4
:10774000002BB8BF5B429BB207EE903AF8EEE77AA7
:10775000A9E70623237055F0ABFE5E4B644A042173
:107760004EF0D2FF7BE7A56079E706F6D833D3ED7C
:10777000006A67EEA67AF4EEC87AF1EE10FADBD46E
:1077800006F6DC39D9ED007AF4EEC77AF1EE10FA9C
:1077900021DB96F8083C33B90623237055F088FEA8
:1077A0004C4B544ADBE7544807F054FD98B196F926
:1077B0001E3C83B9B6F90A3CD9ED007ADFED4A6A7E
:1077C00007EE103A67EEA67AB8EEC77AB4EEE77A1B
:1077D000F1EE10FAB0DCE068281AB0F5FA7F7FF617
:1077E0003EAF0323237006F6D83655F061FE96EDC2
:1077F000007AD4ED047A67EE277A054617EE900AF0
:10780000F4F782FE334B3D4ACDE9000106212846BC
:107810004EF07AFF23E7D7F83C0C7BF02BFB62F0AD
:1078200063FD62F04DFD68B155F042FE294B344ACC
:1078300006214EF069FF62F057FD62F02FFD042330
:1078400023700CE70523FBE762F04EFD62F038FD84
:10785000C8BB05232370E068DFED2A7A9FED2A7A02
:1078600006F53E66D6ED006A2D1AA6EEA77A07EE5B
:10787000905AF8EE677AF4EEC77AF1EE10FA3FF517
:10788000EEAE07232370D7F83C3C9FED207AD3ED72
:10789000C37AD3EDC66A67EE877AB6EE007A67EEF2
:1078A000A77A67EE877A87EEA67AD4ED057A77EE27
:1078B000C77A93EDD57AF4EEC77AF1EE10FA3FF677
:1078C000CEAE0823BCE762F00FFD62F003FD002896
:1078D000BFD1C4E600200D080E200D0818200D08A9
:1078E0002F200D08000000340000C842333373BF5E
:1078F00041200D085C200D08382C00208C200D083C
:10790000B4200D0800007A440000FA43CDCCCC3DF1
:10791000385C00204AF0E4FF40F29C524FF48011A2
:107920004AF096FF9BE61C4805B0BDEC028BBDE813
:10793000F043FFF7F3BBD8F80400FEF71DF894ED11
:10794000060A0121B1EE400AD7F83C0C7AF014F88F
:10795000D7F83C0C05B0BDEC028BBDE8F0437BF0E2
:107960005BBBD8F80400FEF707F89FED0C0A002176
:10797000EAE79FED0A8AD8F804008DED038AFDF747
:10798000FBFFD7F83C0C0123B0EE480A03AA04F130
:1079900014017AF0F7FDDBE7047B00200000000013
:1079A00030B590F8B83185B00446F3B168460FF0B1
:1079B00025FE414869460AF031FC50B104F13C0013
:1079C00028F062F9002384F8B83104F59A7025F0A4
:1079D000E5FA94F890310B2B2DD8DFE803F0294A13
:1079E0004E524A562C5A5E622C6600F59A7025F06B
:1079F000D5FA04F13C0590B194F84030012B0ED13A
:107A000094F89031012B0AD1284627F0ABFF50B1F2
:107A10002046FEF7D9F8294A02214EF075FE284685
:107A200027F0CEFFD5E72046FEF7CEF8244AF3E74D
:107A30002046FFF75FFB94F844303BB994F846309A
:107A400023B994F840309A1E5342534194F8B92117
:107A50007AB373BB84F8B9311A4B586803681B6852
:107A60009847014618482D2205B0BDE830404BF03C
:107A70003DBF2046FFF752FBDDE72046FFF78CFBBA
:107A8000D9E72046FFF7A0FBD5E72046FFF7A2FB8A
:107A9000D1E72046FFF7D4FBCDE72046FFF70EFCE9
:107AA000C9E70A48FFF760FDC5E72046FFF7D6FCA7
:107AB000C1E705B030BD00BF303E0020D0200D082A
:107AC000F8200D08385C0020283C00209486002017
:107AD0002DE9F0412DED028B074684B008460E4695
:107AE0000FF0BCFD032880466D4628D1FB6818685E
:107AF0007CF098F9012822D12148294607F03AFC68
:107B00000446B0B17B69DDED007A1B68F8EEE77AD8
:107B100093EDF27A77EEC77A4246FDEEE77A17EEFA
:107B2000901AC829CDED007AB8BFC82130460FF0B1
:107B30006BFD204604B0BDEC028BBDE8F081114B1B
:107B40000FCB85E80F0030460FF088FD0146284630
:107B50000FF0ECFD04460028EBD07B69DDED017AE7
:107B60001B68B8EEE78AD3EDF27A284638EE678ACA
:107B70000FF074FDBDEEC88A024618EE101AD5E764
:107B8000382C00204078002010B543699FED126A20
:107B90001B68D3EDF06A93EDF17AD3EDF27A86B0FB
:107BA00066EE866A27EE067A67EEC67A68460C4667
:107BB000CDED006A8DED017ACDED027A24F0CAFC9C
:107BC00003A920468DED030ACDED040A8DED051ABB
:107BD00010F074F806B010BD0AD7233C30B5083257
:107BE00004461D460FCA84E80F00134301BFAB686B
:107BF000A360EB68E360636885B093B920460FF03B
:107C00002DFD03AA014628460FF034FD60B103990B
:107C1000019120460FF022FD0199024620460FF007
:107C2000F3FC204605B030BD696801912846F1E7B4
:107C300030B50B6985B004460BB94B6953B30023CB
:107C4000C4F8B43108310FC96D4685E80F002946E4
:107C50002046FFF73DFF98B9124B0122D3F80C1CC8
:107C600028460FF0D1FC4CF02FFB022215214CF0DE
:107C700087FA2046FDF7A8FF0B4A02214EF044FD8B
:107C800029462046FFF71AF810B90848FBF7AAFF63
:107C900005B030BD0123C0F8B43105B0BDE83040B7
:107CA000FFF78EB8386C00202C210D08382C0020EE
:107CB00070B51A4B04460E460FCB88B06D4685E86A
:107CC0000F0020462946FFF75FFFE36818687CF045
:107CD00043FA98B1E368186803681B69984768B16C
:107CE000E368294618687CF0A9F838B94AF0F8FD2D
:107CF00040F295624FF480114AF0AAFD214604A893
:107D00002B463246FFF76AFF04A92046FEF7D6FF4E
:107D100010B90348FBF766FF08B070BD407800203B
:107D2000382C002070B5154B0C4606460FCB88B09A
:107D30006D4685E80F0029463046FFF725FF2B46A4
:107D40002246314604A8FFF749FF6288A388122A19
:107D50004FEA132305D1227ED20744BF03EB8303EE
:107D60005B00227A07EE903AC2F34002B8EE670A4F
:107D700004A93046FFF7BAF808B070BD407800207B
:107D800038B504460D46FFF793FF0023C4F894313D
:107D9000AB88A4F8923138BD7FB50D460446FFF795
:107DA00087FF05F108010FC96E4686E80F001343EF
:107DB00006D1234BD3F8102CD3F8143C0292039332
:107DC00004F5D072012130460FF054FC94F898313C
:107DD00070B923F0050343F0050384F89831204679
:107DE000FDF7F2FE174A06214EF08EFC04B070BD7E
:107DF00023F0070384F898310023C4F89C31E3682A
:107E000062691B68106893ED080A93ED0C1AD3EDB4
:107E1000070AB0EEC00A79F019FDE36862691B68D1
:107E2000106893ED080A93ED0C1AD3ED070AB0EE33
:107E3000C00A79F085FD08212046FEF78BFDD5E7C5
:107E4000386C002058210D082DE9F0438DB06D46A7
:107E500088461C46074613460A4601462846DDE981
:107E60001469FFF7BBFE95E80F0084E80F0007A830
:107E70000FF0C4FBB8F80430F3B9B8F800100131C2
:107E800005AA89B207F13C0027F018F9A0B12346F2
:107E900005AA39462846FFF7A1FE95E80F0086E8B7
:107EA0000F00BDF81630A3F152025342534189F836
:107EB00000300DB0BDE8F08394E80F0086E80F00B5
:107EC0000023F4E770B58B8892B004460D46164641
:107ED000002B47D10DA80FF091FB298801310BAA87
:107EE00089B204F13C0027F0E9F800283AD0BDF847
:107EF0002E1052291CD019D8112913D80F2913D9A3
:107F000033462A46214603A8FFF768FE03AB214605
:107F100007A80BAAFFF762FEE36807A918687CF0C0
:107F200081FC01E01329EBD012B070BD5E29FAE7A5
:107F300007AD03A80FF062FB28460FF05FFB0DF1C1
:107F40000B03CDE90053324603AB0BA92046FFF7E4
:107F50007BFFE0689DF80B3000682A4603A97CF09F
:107F600037FCE1E70120DFE770B5214B04460E4600
:107F70000FCB88B06D4685E80F0020462946FFF7F5
:107F800003FEE36818687CF0E7F898B1E3681868C6
:107F900003681B69984768B1E368294618687BF055
:107FA0004DFF38B94AF09CFC40F216624FF4801144
:107FB0004AF04EFC214604A82B463246FFF70EFE3F
:107FC00004A92046FEF77AFE20B90A48FBF70AFE0C
:107FD00008B070BD0023C4F89431B388A4F892317E
:107FE00004AA31462046FFF76DFF0028F0D1ECE7E8
:107FF00040780020382C0020F0B5324B04460E4665
:108000000FCB91B004AD85E80F0020462946FFF75D
:10801000BBFDE36818687CF09FF898B1E3681868C6
:1080200003681B69984768B1E368294618687BF0C4
:1080300005FF38B94AF054FC4FF4DF624FF4801169
:108040004AF006FC0CAF08A80FF0D8FA38460FF03B
:10805000D5FA0DF10F03CDE900732A4608AB31467E
:108060002046FFF7F1FEE0689DF80F3000683A46C1
:1080700008A97CF0F3FE20B91348FBF7B3FD11B05B
:10808000F0BD0023C4F89431B388A4F8923108AA53
:1080900031462046FFF716FF0028EDD00B4B1B683A
:1080A000022B09D0032B03D1094B93F935321BB1B5
:1080B00006480021FAF764FA01212046FEF74AFC3F
:1080C000DDE700BF40780020382C00203C860020EF
:1080D000384C002037B504460D4686F0CFFDC4F875
:1080E000A801D5ED027AF5EEC07AF1EE10FA17DDAF
:1080F0009FED137A67EE877AFCEEE77AC4ED697A32
:108100002046FDF761FDD4F8A4214FF47A73B2FB49
:10811000F3F30C4A062103B0BDE830404EF0F4BA48
:1081200062F0D2FB0023009395F90D2095F90E30F3
:1081300095F90C1062F064FBC4F8A401E0E700BFFD
:1081400000007A4470210D0810B5B1F90A30A0F88A
:10815000BC3191F90C3080F8BE31B1F90D30A0F886
:10816000C031B1F90F3007EE903AF8EEE77A0446E5
:10817000C0ED717A86F082FD0B21C4F8C80120465B
:10818000BDE81040FEF7E6BB38B504460D4686F064
:1081900075FDC4F8B001D5ED027A9FED047A67EE63
:1081A000877AFDEEE77AC4ED6B7A38BD00007A4439
:1081B0004A7C06480B46003A91F91010D3ED030AA9
:1081C00093ED020A18BF0122FAF7E4B93C860020B9
:1081D00070B51A4E04467068036886B01B680D4679
:1081E0009847042806D16B88102B0ED0732B1FD014
:1081F00000201BE0706803681B6898470328F7D1CC
:1082000094F89031062BF3D1EDE705F108010FC981
:1082100002ACDFED0B0A84E80F000023094800934D
:10822000B0EE600A1A46214602F0B4FE06B070BDF8
:1082300020462946FFF7BCFF0120F7E7385C002005
:10824000000000004C82002038B5D1F8093007EE5C
:10825000903AF5EEC07AF1EE10FA05460C4605DDCF
:108260000B7A022B03D01ED9032B0ED038BD154B31
:108270009FED150AD3F8400C27EE800A7BF002FF31
:10828000D4F80930C5F8D031F0E70E4B9FED0E0A57
:10829000D3F8400C27EE800A7BF004FFD4F80930B5
:1082A000C5F8D431E2E7074B9FED070AD3F8400C3D
:1082B00027EE800A7BF004FFD4F80930C5F8CC31F2
:1082C000D4E700BF386C00200000C84238B5114D1B
:1082D0000C4605F6D44095F84D1D59F07DFA58B17D
:1082E00095F84D1D05F6D44059F07EFA20B994ED6D
:1082F000040A0948FAF7EAF994ED041AD4ED020ADF
:1083000094ED030A95F84D1D0448BDE8384000225D
:1083100059F0A2BA386C00203C8600200C7900206D
:10832000F0B50B69214F85B005460E460BB94B6978
:1083300053B300233B7006F108030FCB6C4684E86F
:108340000F0021462846FFF7C3FB98B9184B0122BE
:10835000D3F80C1C20460FF057F94BF0B5FF022262
:1083600015214BF00DFF2846FDF72EFC114A022186
:108370004EF0CAF921462846FEF7A0FC38B90E484F
:10838000FBF730FC05B0F0BD3846FEF755FEB3886C
:1083900007EE903AF8EE677A09212846C7ED017A90
:1083A00005B0BDE8F040FEF7D5BA00BF94860020C6
:1083B000386C002080210D08382C002010B5044CAA
:1083C000237813B1034866F067FA207810BD00BF28
:1083D00050870020007A00200078072894BF0020F2
:1083E0000120704713B5094B01910446D3F8400CA6
:1083F00003681B69984730B10199204602B0BDE877
:108400001040FEF755BA02B010BD00BF386C002016
:1084100090F8983113F0010018BFC3F38000704743
:10842000094A034692F8AD0768B192F8AC27043ABE
:10843000012A07D85B6A1B6893F8A100431E5842C3
:108440005841704700207047387C002010B5044622
:1084500086F014FCD4F8B031C01AD4F8AC3123EA59
:10846000E37398424FF0000084BFC4F8AC010120D0
:1084700010BD000010B5036804461B6E9847D4F881
:10848000AC3123EAE37398424FF000003CBFC4F8DC
:10849000AC01012010BD000008B504480321FAF723
:1084A00051F8BDE808400148FAF76CB93C86002055
:1084B00070B51C4B0446D3F8400C03681B690E468C
:1084C0009847054610B90025284670BDD4F8943168
:1084D0005BB986F0D3FBB4F89231C4F8940123B1B0
:1084E000114A537843F00103537086F0C7FBD4F868
:1084F0009421B4F89231801A4FF47A72B0FBF2F002
:108500009842E0D323B9084A537843F001035370EB
:108510002046FDF759FB3388044A06214EF0F4F853
:10852000D2E700BF386C00202C8800202C1F0D08DB
:1085300010B590F89031042B0446164B0AD1D3F8AD
:10854000400C03681B69984718B12046FEF7B0FC41
:10855000002010BD0A79D3F8483CDFED0F6A93ED97
:108560000E6A07EE902A0A7E920748BF9FED0B7AAB
:10857000F8EE677A48BF67EE877A86EE267AB0EE25
:10858000C77AB4EEE77AF1EE10FAACBF0120002012
:10859000DFE700BF386C0020DB0FC9400000803BE4
:1085A00013B5094B01910446D3F8400C03681B69CD
:1085B000984730B10199204602B0BDE81040FEF75F
:1085C00077B902B010BD00BF386C002010B504466A
:1085D00086F054FBD4F8A831C01AD4F8A4319842DC
:1085E0004FF0000084BFC4F8A401012010BD0000BA
:1085F00038B505460C4686F041FBD5F8C831C01A9F
:1086000023894FF47A725343984294BF002001208B
:1086100038BD0000C368186808B190F8B808704702
:1086200010B5012104460A4804F0FEFC28B120469A
:108630000321BDE81040FEF78DB94AF051F9BDE8BD
:10864000104040F26B124FF480114AF001B900BFA4
:10865000A883002090F89031022B04D0032B04D182
:10866000034804F0B1BC012070470020704700BFF0
:10867000A883002038B50C4BD3F8A85B90F8903154
:10868000032B044605F004050AD1084804F0B4FCA5
:1086900094F8903135B110B9023B5842584138BD79
:1086A0000020F5E70120FAE7384C0020A8830020DD
:1086B00010B50F4A137843F0800313700D4B93F9F4
:1086C000F82F002A044609DBFEF740FA70B920466D
:1086D0000822BDE810400921FDF748B9BDE8104067
:1086E00001220E2103F55160F5F75CBC10BD00BFFF
:1086F0002C880020384C0020F8B5D0F8B44105464D
:108700005CB1012C1AD04AF0EBF840F643024FF46A
:1087100080114AF09DF8012407E0184BD3F8400C73
:1087200003681B69984710B900242046F8BD284605
:10873000FEF746FB0123C5F8B431F6E7104F97F971
:10874000F83F002BF0DA436A1B6893F8A160012E12
:10875000EAD13C3026F008FD04460028E5D107F5B3
:1087600080539B6A93F8CB3033B132460D2107F525
:108770005160F5F717FCD8E73446D6E7386C00208F
:10878000384C002038B56D4B5A686D4B9A42044600
:108790000D4601D0002071E04B885E2B54D8512B40
:1087A0000CD8103B9AB20F2A28D92046FDF70CFAB4
:1087B0006B88644A04214DF0A7FF58E0523B0C2B14
:1087C000F3D801A252F823F01F890108AB870108F2
:1087D000E1880108F5880108AB870108AB8701082B
:1087E000AB870108AB870108AB870108AB8701089D
:1087F000AB87010825890108FD8801080F2BD4D813
:1088000001A252F823F000BFEF8801089587010804
:10881000058901080B89010819890108F5880108F3
:10882000E1880108AB870108AB870108AB87010825
:10883000AB870108AB870108AB870108AB8701084C
:10884000AB87010811890108732B74D006D8702BEF
:108850006ED0722BA9D1FFF70DFE44E04AF2CF6231
:10886000934262D0A1D8B32B09D8B12B9DD9204611
:10887000FDF7AAF9298852F033F9012038BDBC3B35
:108880009AB2132A91D8132B8FD801A252F823F051
:108890006F8801086F880108AB870108AB87010862
:1088A000AB870108AB870108AB8701086F88010817
:1088B000AB8701086F880108AB870108AB87010807
:1088C000AB8701086F880108AB870108AB870108F7
:1088D000AB8701086F880108AB8701086F88010822
:1088E0002046FFF76BFD00283FF454AFBFE7FFF7CA
:1088F000DFFDF8E72046FFF7FFFEF4E71248FFF739
:108900006BFDF0E7FFF714FEEDE7FFF76BFDEAE71D
:10891000BDE83840FFF77CBDFFF782FDE3E7FFF7D6
:108920003FFEE0E7FFF752FEDDE7FFF761FEDAE723
:10893000FFF78CFDD7E7FFF7AFFDD4E7385C0020E9
:10894000047B0020B4210D089486002090F890311B
:10895000032B0BD0062B06D0012B0AD1C368186855
:1089600003681B681847044801F006BF034804F079
:10897000B3BB0020704700BF4C820020A8830020BA
:108980008B88012B05D00B693BB94B692BB9CB68A0
:108990001BB904480021FAF7FFB902480022083148
:1089A000FAF71CBA382C002010B54B885E2B044611
:1089B0000A464DD8512B05D8103B99B20F2921D921
:1089C00000209DE0523B0C2BFAD801A151F823F076
:1089D0003B8B0108C1890108F58A01080B8B01084E
:1089E000C1890108C1890108C1890108C18901083B
:1089F000C1890108C1890108C1890108438B0108A7
:108A00004B8B01080F2BDBD801A151F823F000BFDD
:108A1000038B0108158B01081D8B0108258B0108AC
:108A2000358B01080B8B0108F58A0108C189010803
:108A3000C1890108C1890108C1890108C1890108EA
:108A4000C1890108C1890108C18901082D8B01086C
:108A5000B32B00F0848016D8732B7DD00ED8702BEA
:108A600077D0722BACD1D1ED027A9FED447A67EECC
:108A7000877AFDEEE77AC0ED6B7A40E0B22B9FD1AA
:108A8000FFF7E2FB3BE0CD2B2CD8BB2B98D9BC3BAE
:108A9000112B95D801A151F823F000BFFF8A0108DE
:108AA000FF8A0108C1890108C1890108C18901083B
:108AB000C1890108C1890108658B0108C1890108C4
:108AC000658B0108C1890108C1890108C1890108B4
:108AD000658B0108C1890108C1890108C1890108A4
:108AE000718B01084AF2CF6293427FF469AFFFF7BE
:108AF0002BFB04E002F108012046FEF74DF80120AF
:108B000010BD1146FFF730FAF9E711462046FFF78E
:108B10008FF8F4E71146FFF7CBF8F0E71146FFF7BF
:108B200001F9ECE71146FFF72BF9E8E71146FFF7EB
:108B300033F9E4E7FFF774FDE1E71146FFF75CFA6C
:108B4000DDE71146FFF7C6FAD9E71146FFF7E8FB64
:108B5000D5E7FFF719FBD2E7FFF72AFBCFE7FFF7CF
:108B60000FFFCCE7064802F10801F9F7CFFDC6E791
:108B700011462046FFF7AAFBC1E700BF0000C8422C
:108B80003C860020704700007047000090F82800E5
:108B90007047000090F8A802704700000F2070474F
:108BA0000020704700207047002070470020704769
:108BB0000048704764220D080048704770220D0875
:108BC00008B5094800F50053D3F8F43BB3F9083071
:108BD00000EE103AB8EEC00AF5F76EFCBDE80840AA
:108BE0000248FCF727BE00BF382C0020DC7C0020A8
:108BF00010B514482DED028B1C4600F5005300F50E
:108C00008040B3F90432D0F8340C08EE103A03680F
:108C100082B09B6ECDE900219847B8EEC88AF0EE8D
:108C2000400ADDE90021B0EE480A0748FCF7A6FB40
:108C30000548FCF761FE84ED000A02B0BDEC028B32
:108C400010BD00BF382C0020DC7C0020F8B51C4D86
:108C500005F5005405F580462846D6F83C7CF5F726
:108C600019FCB4F9403201EE103AB4F93E3200EE8C
:108C7000903A434200EE103AB8EEC11AF8EEE00A1C
:108C8000B8EEC00A384678F0E1FD2846D6F83C6CCC
:108C9000F5F700FCB4F9403201EE103AB4F93E3277
:108CA00000EE903A434200EE103A3046B8EEC11A58
:108CB000BDE8F840F8EEE00AB8EEC00A78F040BE31
:108CC000382C002038B5144C04F5804504F57F6439
:108CD000D5F8340C03689B689847692100F1940229
:108CE00020464AF0DBFAD5F8340C0368DB68984775
:108CF0006A2100F1940220464AF0D0FAD5F8340CEB
:108D000003681B6998476B2100F194022046BDE877
:108D100038404AF0C3BA00BF382C0020014806F0A2
:108D2000B3BC00BF382C00203C3084F061BB000095
:108D3000F7B51D4D0646686803681B6B98470446E7
:108D400068B315F9073C002BA5F580572ADBAB6A01
:108D500093F8CB401CB397F8F83F03F0A003202B07
:108D600020D1686803681B689847052807D06868A1
:108D700003681B689847A0F110035C425C410B4AF2
:108D800002F618430193D7F80C3D0093D2F83C3C0F
:108D9000D2F8342C2146304684F0D8FA04462046D6
:108DA00003B0F0BD0024FAE7385C0020386C0020E6
:108DB0003C30FFF7BDBF000038B5114D04461148E7
:108DC000F5F7ACFF95F9F83F002B14DA236A93F816
:108DD000A120012A06D00C4B00215868BDE838407C
:108DE000FCF7EABB0D2105F55160F5F7DBF895F9C5
:108DF000F83F002BEFDB2046BDE8384084F0E2BDB1
:108E0000384C0020382C0020385C00203C30FFF724
:108E1000D3BF000001207047012070470120704738
:108E200001207047072070470120704700207047DD
:108E3000002070470120704700487047B8230D0894
:108E400000487047C0230D0870B52DED028B00253A
:108E5000C36880F83C501B68DFED488AD3ED0A0AEE
:108E600042699FED478A93ED060AF4EEE80A04464C
:108E7000F1EE10FA88B01068B8BFF0EE480A78F04A
:108E8000CBFAE36862691B681068D3ED0A0A93EDB8
:108E9000060AF4EEE80AF1EE10FAB8BFF0EE480A5E
:108EA00078F032FB636920461E68FCF791FE636828
:108EB000B3F93820B3F9363000EE903A434201EE70
:108EC000102A00EE103AB8EEC11AF8EEE00AB8EE39
:108ED000C00A304678F0BAFC636920461E68FCF789
:108EE00077FE6368274CB3F93820B3F9363000EECB
:108EF000903A434200EE103A01EE102A3046B8EEA6
:108F0000C11AF8EEE00AB8EEC00A78F019FDD4F8FC
:108F1000480C7AF0B5FDD4F8486C338B1B0723D589
:108F200004A80EF06BFB09F081FB9FED170A0446C5
:108F300006F11C0023F04AFB01AA04A920468DED8E
:108F4000010ACDED020A8DED031A09F051FB80B143
:108F50000322294604A80EF057FB0C4B186804AAFC
:108F600090F8791058F094FD09480821F9F7EAFAC9
:108F7000012008B0BDEC028B70BD00BF00000034C2
:108F800000007A43386C00200AD7233CA8910020C7
:108F90003C86002030B52DED048BC3689FED898A97
:108FA0001B684269D3ED0A7ADFED870A93ED060A62
:108FB000F4EEC87AF1EE10FA0446A8BFF0EE670AA4
:108FC000106889B078F028FA636920461D68FCF7BC
:108FD000FFFD6368B3F93820B3F9363000EE903AFC
:108FE000434200EE103A01EE102A2846774DB8EEC3
:108FF000C11AF8EEE00AB8EEC00A78F027FCD5F8FE
:10900000480C7AF07FFEA5F580535B7FD90747D4E3
:10901000D5F8483C1A8BD20742D593ED0A9AB4EEA4
:10902000C89AF1EE10FAB8BF93ED049AE36A186893
:1090300056F072F8D5F8403CD3ED067AA36B20EEDB
:10904000270AD3ED007AF0EE498AE0EE278AB0EEE7
:10905000490AF5EEC08AF1EE10FAD8BFDFED5C8A5E
:10906000F0EE680A1FF02EFF28B9D5F8480CB0EED4
:10907000680A7AF0C5FB636893F95130272B0FD04B
:10908000A36A186856F048F8F0EEC07AF4EEC87A91
:10909000F1EE10FAB0EE407A20D5002384F83C308F
:1090A000236B1B68B3F9083000EE103A2046B8EE87
:1090B000C00AFCF74FFC2046FCF7BCFB2046B0EE94
:1090C000408AFCF741FA002848D00021204609B028
:1090D000BDEC048BBDE83040FCF76EBAD5F8483CD7
:1090E0009FED3C0AD3ED0F7AD3ED0B6AA36B27EE0D
:1090F000800AF4EEC86AD3ED007AF1EE10FA67EE5A
:10910000277A10DB9FED341ADFED310A552037EE58
:10911000800A1FF0DBFF012384F83C30D5F8480CAF
:109120007AF05EFBBCE79FED2D7AF4EEC76AF1EEB4
:1091300010FA05D89FED261ADFED290A5920E6E737
:10914000F0EEE66AF4EEC86AF1EE10FAE3D594F8B0
:109150003C30002B08BFB0EE670ADCE7636A0221EF
:1091600018687FF051F81F4806F020F9B0EE480A61
:10917000D5F8480C7AF0C8FC01461B48FAF730FCD9
:109180006369186879F048FF236A1D686369186885
:1091900078F080FD05AC204614498DED020ACDED36
:1091A000030A8DED041AF9F7BDFB079B009394E8C1
:1091B0000C0002A9284675F095FF09B0BDEC048BA0
:1091C00030BD00BF0000003400007A43386C00203E
:1091D00000000000E02E65420000B442000000B430
:1091E0000000B4C2D0580020382C00203C8600205B
:1091F00008B5064BD3F8483CD868243022F032FF3B
:10920000FCEEC07A17EE900A08BD00BF386C002053
:10921000024BD3F8483CD86878F0E6BD386C0020A3
:109220000B207047012070470020704701207047D5
:1092300000207047004870475C240D0800487047C4
:1092400064240D080120704708B5DFED237AF4EEA1
:10925000E70AF1EE10FA2DED028BF0EE408AB0EE47
:10926000608A35DDDFED1D7AF4EEE70AF1EE10FAE3
:109270002ED5F6EE007A70EEE77ADFED196A9FEDF3
:10928000190ADFED190AF0EEE77A87EEA67A872051
:10929000B7EE001A30EE470A1FF018FFDFED137A21
:1092A0009FED131ADFED130A20EE270A8A2020EE25
:1092B000280A1FF00BFF30EE080ABDEC028BDFED31
:1092C0000A0ABDE808408D20B7EE001A1FF0FEBE66
:1092D0009FED050AEFE700BFAC1C5A3ED578493F29
:1092E0008FC2753E9A99993F00000000FAEDEBBAE3
:1092F0009A99993E9A9999BE70B57E4EB6F9043204
:109300002DED048B00EE903AF8EEE00A82B00446B0
:1093100001AA6946B0EE600AFCF730F8A0697CF05B
:10932000EBF8E369D0ED008AD3ED946AD3ED977A38
:1093300090ED016AA3689FED701ADFED700A27EEC9
:10934000E80A68EEA68A03F6F803E6EE278A0546E1
:109350003B20DFED6B7AB0EEE87AB4EEE77AF1EE1F
:1093600010FA58BFB0EE677ADFED667AC7EE275A7B
:10937000F7EE007A77EEE57A9DED007A67EE877A70
:1093800093ED007A67EE877A9FED5F7AA6EE260A64
:1093900087EE879A1FF09AFE3C209FED571ADFED6B
:1093A000570AB0EE408AB0EE680A1FF08FFE626B7B
:1093B000564B1268DFED567AB2F90820D3ED006AF9
:1093C0009FED541ADFED540A07EE102AB8EEC77A63
:1093D000F0EE408A27EE277ADFED507AA6EEA77AE4
:1093E0004520F4EE007AA7EE678ABAEE000A28EE6E
:1093F000000A83ED007A8DED000A1FF067FEDDEDB7
:10940000017A9FED477A474B8DED000AF0EEE77A3F
:10941000F4EEC77AF1EE10FA51D593ED007ADFED54
:10942000427A77EE277AB2EE007AF4EEC77AF1EE5E
:1094300010FA58BFF0EE477AC3ED007A67EEA87ACB
:10944000CDED017A636A186890F8CB10002939D104
:109450007EF0DAFE636A1B6893F8A110012938D008
:1094600003293FD039B9236A186876F023FB236AB1
:10947000186875F06FFD236ADDED010A18689DED2F
:10948000000A0368B0EE491ADB6A9847204695ED5A
:10949000028AFCF76FF92046F0EE400AB0EE480A67
:1094A000FFF7D2FE236A62681868D2ED020A0368E9
:1094B00001215B6E984702B0BDEC048B70BD0022A9
:1094C0001A60BFE796F9F93F002BB4BF01210221D2
:1094D000BEE7236A186876F0EDFA236A186875F01B
:1094E0004FFDC8E7D9790029C5D12046FCF766FBB6
:1094F000C1E700BF384C002000000C4400000CC441
:109500000000FA4400409C4500003442B086002030
:109510000AD7233D00A08C4500A08CC58FC2753FA3
:1095200000000034B48600208FC2F53C162070473E
:1095300000207047002070470120704700207047CE
:1095400081F001007047000001207047004870471B
:1095500000250D080048704794070D0803681BB1EB
:10956000007900F00100704718467047F0B5494D8A
:1095700095F94D6D85B00446A5F50055002E00F017
:1095800085804548FFF7EAFF064600287ED06369DC
:1095900020461F68FCF71CFB6368B3F93820B3F959
:1095A000363000EE903A434201EE102A00EE103AB7
:1095B000B8EEC11AF8EEE00AB8EEC00A384678F004
:1095C00045F9636920461F68FCF702FB6368B3F93D
:1095D0003820B3F9363000EE903A434200EE103AAC
:1095E00001EE102A3846B8EEC11AF8EEE00AB8EEDD
:1095F000C00A78F0A5F905F58043D3F83C0C78F063
:1096000039FA18B96369186879F0B8FBB5F9A4306C
:1096100004F13C001BB9B5F8A230A5F8A430B5F8A8
:10962000A43007EE903AF8EE677A04F1980203A9A5
:109630000027CDED037A4CF017FB04F15C00C4F871
:10964000A07001906CF0ACFC002384F8A530B5F953
:10965000A43001981BB9B5F8A230A5F8A430B5F82C
:10966000A43007EE903AF8EEE77AB7EE000A80EE03
:10967000270A6CF0B9FC09487BF03AFFC4F8C870BF
:10968000DFED077A20EE270A84ED310A304605B077
:10969000F0BD00BF384C00208059002050780020D9
:1096A0000AD7233C10B50446FBF7C2FB2046154BF6
:1096B00040F83C3B4CF05AFA134B2365134B9FED9B
:1096C000142A9FED141ADFED140A9FED140A636546
:1096D000F1EE041A04F15C006CF09CFC00232046BF
:1096E0000F49C4F8A830C4F8AC30C4F8B030C4F89E
:1096F000B430C4F8B830C4F8BC3041F051FF204653
:1097000010BD00BF08260D08CDCCCC3D0000404068
:109710000AD7233B00803B459A99993ECDCC4C3EDD
:10972000A0250D082DE9F0432DED028B9BB091464D
:1097300004460D4685F0A2FAB8499FEDB98A06465F
:10974000A1F1080022F0C0FB94ED161ACDED110A2C
:109750007E20F1EE410A8DED100A1FF0B7FC94ED6A
:10976000161A8DED100AF1EE410A7F209DED110AC7
:109770001FF0ACFC10A904F13C008DED110A4CF077
:1097800091FAA848CDED130A8DED120A7BF0B0FED8
:10979000D4ED327AD4ED140A94ED151AE0EE087A7D
:1097A000892004F15C074FF00008B0EE670A1FF053
:1097B0008DFC12A822F0D4FB9B4812A909F088F96D
:1097C00014A938468DED140ACDED150A6CF0C8FACF
:1097D0003846CDF85880CDF85C806CF005FB8DEDF7
:1097E000160ACDED170AB9F1000F00F0018101232F
:1097F000C4F8D06084F8CC308C4E04F1A80116A8CF
:1098000022F08AFBB6F9043200EE103A16A8B8EE40
:10981000C00A22F0A5FB16A9A6F6086009F044F9D3
:1098200018A928468DED180ACDED190A22F074FB0F
:10983000B6F9043295ED007A07EE903AF8EEE77A41
:10984000B0EEC77AB4EEE77AF1EE10FA00F3CE800C
:1098500095ED017AB0EEC77AF4EEC77AF1EE10FA20
:109860004CBF0123002384F8A530B6F9043295EDEE
:10987000000A5A4207EE903A00EE902AB8EEE71A34
:10988000F8EEE00ACA201FF021FC85ED000AB6F9C7
:10989000043295ED010A5A4200EE902A07EE903A02
:1098A000F8EEE00AB8EEE71ACB201FF00FFC85EDCA
:1098B000010A94F8A4305A1C84F8A4201422B3FBA3
:1098C000F2F102FB1133DBB2002B34D14AF0FCFC85
:1098D000064685F0DBF98046D4F8AC000F46F2F777
:1098E00013FECDE90E01D4F8A800F2F70DFECDE984
:1098F0000C01D4F8A000F2F707FECDE90A01686870
:10990000F2F702FECDE908012868F2F7FDFDCDE986
:1099100006011398F2F7F8FDCDE904011298F2F769
:10992000F3FDCDE90087CDE90201414B414A4249AF
:1099300030464AF03FFA1BB0BDEC028BBDE8F08325
:1099400012A822F08FFBDFED3D7AB4EEE70AF1EECC
:1099500010FA57D494F8CC3063B956E038466CF01E
:10996000A3FA94F8CC3084ED2A0AC4ED2B0A002B1C
:109970003FF442AFDFED325ADFED324A9FED324A1B
:10998000DFED323A12AA2B4605F10801B2EE0E5A6B
:10999000B7EE003AB2EC016A94F99D00B0EEC67AD7
:1099A00067EE256A07EE900A76EE842AF8EEE77AEB
:1099B000B0EE647AA7EE857AC3EEA27A27EE087A33
:1099C00077EE837A27EE267AB5EEC06A67EE877A5D
:1099D000F1EE10FA48BFF1EE677AE3EC017A9942B2
:1099E000D8D1CDF85C80CDF8588005E701233AE75F
:1099F00094F8CC304BB1D4F8D00040F6B833361AD6
:109A00009E429DD9002384F8CC3094F8A530002BD9
:109A1000A4D138466CF0AEFAA3E700BFAC590020E1
:109A20000AD7233C50780020303E0020384C0020DC
:109A3000C8F00C080C250D0894070D089A99993E5A
:109A40000000C8420000BE42000070420000FA431D
:109A50002DE9F04F2DED048B0446A5B0BD487BF0F9
:109A600047FDBD4BDFEDBD7A1B68DB6A93F89C3088
:109A700060EE278A33B9F1EE687AC4ED327AC4ED2C
:109A8000318A46E0B64D05F540539B6A93F8A090A5
:109A9000B9F1020FEFD185F0F1F805F58043D3F865
:109AA0004C3CC01A40F2DB539842E4D99FEDAD8A9A
:109AB00095F8DB1B8DED218A18AB21AA05F6C800AD
:109AC0008DED228A8DED238A1DF046FE08B3A6484F
:109AD00021A920F0FBFBD4ED2C7A8DED210A37EE85
:109AE000800AD4ED2D7ACDED220A77EEA00A9F48A8
:109AF00084ED2C0AC4ED2D0A8DED231AFFF72EFDFF
:109B000060B985F0BBF884ED2D8AC4F8C00084EDFF
:109B10002C8A25B0BDEC048BBDE8F08F05F5005B09
:109B2000D4F8C020DBF87C3D42B9C4F8C03084EDE5
:109B30002D8A84ED2C8A84ED328AEAE79A42E8D0B5
:109B40008B4804F1B00108F0AFFF8A498DED190A86
:109B5000F1EE607AA1F1080010EE108A17EE907A0B
:109B6000CDED1A0ACDED1B7A8DED1C0A22F0ACF971
:109B7000DBF87C3DD4F8C0208DED1D0AA3EB020A72
:109B8000BAF5FA7FCDED1E0A04F1B8051DAE0CD969
:109B900096E80300C4F8C03084ED2D8A84ED2C8A49
:109BA00085E80300C4ED318AC5E72946304622F036
:109BB0008BF996E8030085E8030094ED329ADBF810
:109BC0007C3D9FED6D6AC4F8C03039EE285A8DEDAA
:109BD0001F0ACDED200A1FA91BAA0023F0EE489A08
:109BE000F1EC017AF0EEE76AF4EEC66AF1EE10FAF3
:109BF0001FD4D2ED005AB0EEE57AB4EEC67AF1EE9B
:109C000010FA16D485EEA77AB5EEC07AF1EE10FA06
:109C10000FD907EE903AF8EEE77A37EE457A77EE0D
:109C2000A67AE7EE269AFCEEE77ACDED177A9DF854
:109C30005C30B9F1010F02F1040240F087802BB1D2
:109C400007EE903AF8EEE77AC9EEA79A4FF4EC7077
:109C5000F5EEC09AF1EE10FA48BF79EEA99AB5EE8A
:109C6000001AFDEE000AB0EE690A1FF02FFA39EE75
:109C7000009A9FED420A94ED327ADFED417A29EEA7
:109C8000009AA7EE279AD4ED147A84ED329A39EE31
:109C9000289AB4EEE79AF1EE10FA44BF77EEE87A2C
:109CA000C4ED327A94ED329A4AF00EFB054684F008
:109CB000EDFF8146D4F8C400CDF850A00E46F2F76F
:109CC00023FCCDE9120118EE900AF2F71DFCCDE954
:109CD0001001D4F8C800F2F717FCCDE90E0119EE17
:109CE000900AF2F711FC38EE899ACDE90C0119EED1
:109CF000100AF2F709FCCDE90A014046F2F704FC2C
:109D0000CDE908013846F2F7FFFBCDE906012098BE
:109D1000F2F7FAFBCDE904011F98F2F7F5FB194BB6
:109D2000194ACDE90201CDE90096184928464AF0C2
:109D300041F82046FBF748FF1549B0EE490A4CF0C0
:109D40006FFF84ED2D8A84ED2C8A98E64FF001098F
:109D500046E700BF50780020308600200AD7233C19
:109D6000382C0020000000005041002080590020C5
:109D7000303E0020AC5900200AD7233DCDCC4C3ECC
:109D8000CDCC4C3F2C250D0838250D086F250D082E
:109D900074250D082DE9F0412DED048B044688B0A3
:109DA000FFF756FE636920461D68FBF711FF6368E5
:109DB000B3F93820B3F9363000EE903A434200EE62
:109DC000103A01EE102AF8EEE00AB8EEC11AB8EE29
:109DD000C00A284677F03AFD04F13C052046FBF71F
:109DE000BFFD28464BF05AFFD4ED260A1FF06AF853
:109DF000B64BA0B9B3F9A4201AB9B3F8A220A3F8BE
:109E0000A420B3F8A43007EE903AF8EE677A04F194
:109E1000980206A92846CDED067A4BF025FFAC4DF9
:109E2000DFEDAC8AD5F8F43BB3F9083000EE103A18
:109E3000A5F50050B8EEC00AF4F73EFB2046B0EEA0
:109E4000408A8DED030AFBF7C3FEB5F93E3201EE01
:109E5000103A434200EE903AB8EEC11AF8EEE00A2A
:109E6000F820B0EE480A1FF031F920468DED030AC4
:109E7000FBF742FD2046B0EE409A9DED030AFBF74A
:109E8000F5FC074605F64850FFF768FBD8B195F892
:109E9000683D9FED917AD4ED286A07EE903AF8EE8E
:109EA000E77A67EE877A9FED8D7AE6EE877A8C4EB9
:109EB000C4ED287A042F21D8DFE817F00800BE008F
:109EC000E000E500F000F0EE687AF0E7854B002155
:109ED000986A7EF099F9D6F8340C75F03BF8D6F80C
:109EE000340C012175F0E6FDD6F83C0C9FED790AA3
:109EF00079F020F804F15C006CF052F8D5F8EC3BF6
:109F0000CDED048AB3F90880D5F8F03BCDED058A94
:109F1000B3F90870B5F9043208EE103A236A1868EC
:109F200003689B6E9847B8EEC88AF0EE400A05AA0F
:109F3000B0EE480A04A92046FBF720FA94F99C30B9
:109F400094ED287A07EE903AF8EEE77AF1EE489A27
:109F5000B4EEE77AF1EE10FA37DB84F08FFED6F834
:109F60004C3CC01A40F6B83398422ED958EA070341
:109F700006A914BF012200222046CDED068ACDEDB0
:109F8000078AFFF7CFFBF6EE007A69EEA70A28EE04
:109F9000271A4FF4A5709DED060A8DED011ACDED3F
:109FA000000A1FF093F840F24B108DED060A9DED6C
:109FB000011ADDED000A9DED070A1FF087F806A9DA
:109FC00004A88DED070A21F0A7FFB0EE481AF0EEC5
:109FD000690A9DED040A4FF4A7701FF077F8B0EE00
:109FE000481AF0EE690A8DED040A40F24F109DED1B
:109FF000050A1FF06BF8B5F904328DED050A00EE85
:10A00000103A05AA04A9B8EEC00A374862F082FEE9
:10A01000D6F8340CDDED050A03689DED040ADB6A11
:10A02000B0EE491A98476369186878F0F5FF08B0F0
:10A03000BDEC048BBDE8F0812A4B2C4F986A0221BD
:10A040007EF0E2F83B786BB963689FED291ADFED8B
:10A05000210A93ED040A4FF48C701FF037F838464C
:10A0600005F0FAFE20469DED030AFBF7E3FB1F48CF
:10A070008DED030A03A905F029FF3FE7236A0121BB
:10A08000186875F017FD236A186874F079FF636922
:10A090009FED100A186878F04DFF2FE7114F02214D
:10A0A000B86A7EF0B1F820469DED030AFBF7C2FBCB
:10A0B000A7F55A708DED030A05F078F963699DEDF7
:10A0C000030A186877F048FC18E700BF382C002016
:10A0D000384C002000000000D0CC4C3D3333733F9F
:10A0E000386C0020385C0020907900206C870020BC
:10A0F00000007A4417207047012070470020704705
:10A1000000207047012070470048704794260D08D2
:10A110000048704799070D0883689FED067A03F69B
:10A120003803D3ED187A67EE877AFCEEE77A17EEFC
:10A13000900A70470000C84283689FED067A03F6D4
:10A140003803D3ED197A67EE877AFDEEE77A17EEDA
:10A15000900A70470000C842806800F638007FF01F
:10A160005BBA000010B5836803F63803D3ED180A14
:10A1700093ED190A044B0C460FCB84E80F002046E0
:10A180000DF078FD012010BD4078002070B5836887
:10A1900093F9386804460D4696B1B3F85C28D207A7
:10A1A00008D50B4A106828B193F83A2890F879102E
:10A1B00057F050FC29462046BDE8704000F034BC02
:10A1C000FBF702FD034A04214CF09EFA304670BDB5
:10A1D000A89100209C260D082DE9F0432DED048B5D
:10A1E00099B00446FBF7B0F9074640B1002120467C
:10A1F00019B0BDEC048BBDE8F043FBF7DDB9636A31
:10A200009FEDA38A186802217DF0FEFFA0688DED06
:10A21000098A12AB0FAA0CA900F638008DED0A8A44
:10A220008DED0B8A8DED0C8A8DED0D8A8DED0E8AEC
:10A230008DED0F8A8DED108A8DED118A8DED128ACC
:10A240008DED138A8DED148A7FF0A8FC0546002859
:10A2500000F0EF80DFED8F8ADDED0F6A9DED107A63
:10A26000DDED117AA36867EEE87A66EEA86A27EE5C
:10A27000287A03F6540393ED000ACDED177A15A85A
:10A28000CDED156A8DED167A22F0A0F9DFED827A18
:10A290008DED090A8DED030A8DED050AB0EEC00AB9
:10A2A000B4EEE70AF1EE10FACDED0A0A8DED0B1AC5
:10A2B000CDED040ACDED060A06D5F0EEE00AF4EE87
:10A2C000E70AF1EE10FA02D405A821F049FF159B28
:10A2D000079307A8169B089321F0C4FE6369DFF873
:10A2E000C4911B68D9ED461AD3EDC50A6B480DF130
:10A2F0000C08B6EE009A05AAB0EE401A414693ED5E
:10A30000080A60EE890A62F063FE98E8030009AE6D
:10A3100086E8030063699DED171A1B68D9ED461A9C
:10A32000D3EDC60A93ED0E0A5C4860EE890AB0EEE2
:10A33000C11A62F031FE5A20F1EE400AB0EE401A26
:10A340009DED0B0A1EF0C2FE12A88DED0B0A9FEDCB
:10A35000510A21F0C9FD07A93046CDED080A8DED5F
:10A36000070A21F0D9FD9DED147ADDED0B7A6369C2
:10A37000E7EE687A30464FF00008CDED0B7A1B68A7
:10A3800093EDC20A21F0C0FE63699DED0B0A1B68C4
:10A39000D3EDC40A93EDC31AF0EEE00A6420F1EEA7
:10A3A000600A1EF093FE63698DED0B0A1B683B4843
:10A3B00093ED080AD3EDC50A93ED0E1AD3EDC61A34
:10A3C000A36B07AA93ED002A8DF81C80314663F039
:10A3D00091FFA06890F95038022B1CD0032B45D078
:10A3E000012B53D10CA821F033FEF7EE007AB4EE26
:10A3F000E70AF1EE10FA03DC00259FED258A18E04C
:10A400008DED078A8DED088A0CA907A81FF0B6FE0E
:10A41000B0EE408A0DE007A900F638008DED078AFE
:10A420007FF006F905460028E7D09DED078A28EE63
:10A43000288A84F023FC636CC21A632A00D80BB903
